:100000000C94EA040C9405050C9405050C94050564
:100010000C9405050C9405050C9405050C94050538
:100020000C9405050C947F170C9405050C9405059C
:100030000C94C5270C9405050C9405050C94050536
:100040000C9405050C9405050C9413160C940505E9
:100050000C94190B0C9405050C94E00A0C940505FE
:100060000C9487190C9405050C941F270C94050516
:100070000C9433630C9405050C940505351A281A65
:100080001C1A021AE819C419D619391D6D1C6A1CEC
:10009000C419571C3D1C1D1CFD1BAB1B591B411AD1
:1000A0000A0D426174743A0020332043656C6C730E
:1000B00020200020342043656C6C73202000204CED
:1000C0006F77207761726E696E67206C6576656CFC
:1000D0003A2025642E2564000A0D3D3D3D3D3D3D01
:1000E0003D3D3D3D3D3D3D3D3D3D3D3D3D3D3D3D40
:1000F0003D3D3D3D3D3D3D3D3D3D3D3D3D000A0DD0
:10010000466C69676874436F6E74726F6C0A0D4851
:10011000617264776172653A25642E25640A0D5315
:100120006F6674776172653A5625642E256425637F
:1001300020000A0D74686520757365206F66207451
:1001400068697320736F66747761726520697320C4
:100150006F6E6C79207065726D6974746564200AC5
:100160000D6F6E206F726967696E616C204D696BEF
:10017000726F4B6F707465722D4861726477617233
:1001800065000A0D7777772E4D696B726F4B6F7034
:100190007465722E64652028632920486953797339
:1001A00074656D7320476D6248000A0D3D3D3D3D0D
:1001B0003D3D3D3D3D3D3D3D3D3D3D3D3D3D3D3D6F
:1001C0003D3D3D3D3D3D3D3D3D3D3D3D3D3D3D009C
:1001D0000A0D47656E65726174696E6720646566B5
:1001E00061756C74204D69786572205461626C652C
:1001F0000025642025640A000A0D496E69742E20CA
:10020000454550524F4D003A2047656E6572617406
:10021000696E672044656661756C742D506172610A
:100220006D65746572207573696E67206F6C6420EC
:10023000537469636B2053657474696E6773000A45
:100240000D466C696768742D74696D65202575208D
:100250006D696E2020546F74616C3A2575206D694C
:100260006E000A0D414343206E6F742063616C6918
:100270006272617465642021000A0D5573696E67AE
:1002800020706172616D6574657273657420256498
:10029000000A0D43616C6962726174696E67207057
:1002A000726573737572652073656E736F722E2E2F
:1002B000004F4B0A0D000A0D436F6E74726F6C3A5B
:1002C000200048656164696E67486F6C64004E6F1A
:1002D000726D616C20284143432D4D6F6465290088
:1002E0000A0D3D3D3D3D3D3D3D3D3D3D3D3D3D3DA1
:1002F0003D3D3D3D3D3D3D3D3D3D3D3D3D3D3D3D2E
:100300003D3D3D3D3D0A0D002E000A0D2044414378
:10031000206F7220493243204552524F52212043D0
:100320006865636B204932432C2033567265662C16
:100330002044414320616E6420424C2D4374726C12
:10034000005B25695D005B25695D002B204D696BB5
:10035000726F4B6F70746572202B0048573A5625A8
:10036000642E25642053573A25642E2564256300A6
:1003700053657474696E673A2564202573004932A9
:1003800043204552524F52212121004D6973736918
:100390006E6720424C2D4374726C3A256421210013
:1003A00028632920486F6C6765722042757373005B
:1003B000486F6568653A2020202020253569005364
:1003C0006F6C6C486F6568653A20253569004C751F
:1003D0006674647275636B3A20253569004F6666F2
:1003E0002020202020203A20253569004B65696EA9
:1003F00065200048F668656E726567656C756E67A6
:1004000000616B742E204C616765004E69636B3A26
:1004100020202020202025356900526F6C6C3A2066
:100420002020202020253569004B6F6D706173738B
:100430003A202020253569004B313A2534692020A7
:100440004B323A25346920004B333A253469202059
:100450004B343A25346920004B353A253469202045
:100460004B363A25346920004B373A253469202031
:100470004B383A25346920004E693A2534692020EA
:10048000526F3A253469200047733A253469202099
:1004900047693A253469200050313A2534692020D3
:1004A00050323A253469200050333A2534692020EF
:1004B00050343A25346920004779726F202D20533B
:1004C000656E736F72004E69636B20253469202856
:1004D0002533692E25692900526F6C6C20253469FB
:1004E00020282533692E2569290047696572202552
:1004F0003469202825336929004E69636B2025342F
:100500006920282533692E25782900526F6C6C20CC
:1005100025346920282533692E2578290047696507
:100520007220253469202825336929004E69636BC0
:100530002025346920282533692928253369290095
:10054000526F6C6C202534692028253369292825B1
:1005500033692900476965722025346920282533CD
:100560006929282533692900414343202D205365FB
:100570006E736F72004E69636B20253469202825E5
:1005800033692900526F6C6C20253469202825338B
:10059000692900486F63682025346920282533695C
:1005A0002900566F6C746167653A202020253569F3
:1005B0000052432D4C6576656C3A20202535690044
:1005C00052432D4368616E6E656C733A2534690041
:1005D0004B6F6D706173732020202020202000520B
:1005E00069636874756E673A2020253569004D652A
:1005F0007373776572743A202025356900537461EE
:1006000072743A202020202025356900506F7469CB
:10061000313A202025336900506F7469323A202026
:1006200025336900506F7469333A202025336900FF
:10063000506F7469343A202025336900536572760F
:100640006F202000536574706F696E74202025330D
:1006500069005374656C6C756E673A2025336900C8
:1006600052616E67653A2533692D253369004578F7
:100670007465726E436F6E74726F6C2020004E69E9
:100680003A2534692020526F3A2534692000477397
:100690003A253469202047693A25346920004869A1
:1006A0003A253469202043663A2534692000424CBB
:1006B0002D4374726C204572726F72732000202576
:1006C0003364202025336420202533642020253303
:1006D0006420002025336420202533642020253326
:1006E0006420202533642000202533642020253316
:1006F00064202025336420202533642000424C2DC3
:100700004374726C20666F756E6420002025632030
:100710002020256320202025632020202563200021
:1007200020256320202025632020202563202020F1
:10073000256320002025632020202D2020202D202F
:1007400020202D00313000313100313200466C69FB
:100750006768742D54696D652020002020202020BA
:10076000202535756D696E00546F74616C3A2535BE
:10077000756D696E0028726573657429000A0D50E5
:100780006C6561736520636F6E6E65637420537072
:10079000656B7472756D207265636569766572202C
:1007A000666F722062696E64696E67204E4F572EC5
:1007B0002E2E006F6B2E0A0D0054696D656F7574D7
:1007C0002E0A0D0000010203040405060708090AA9
:1007D0000B0B0C0D0E0F101111121314151516170B
:1007E0001818191A1B1B1C1D1D1E1F1F202121223A
:1007F000232324242525262727282829292A2A2B8C
:100800002B2C2C2D2D2D2E2E2F2F30303031313200
:100810003232333333343434353535363636373790
:100820003737383838393939393A3A3A3A3B3B3B35
:100830003B3C3C3C3C3C3D3D3D3D3E3E3E3E3E3FE8
:100840003F3F3F3F3F4040404040404141414141A8
:100850004142424242424242434343434343434470
:10086000444444444444444545454545454545453F
:100870004646464646464646464747474747474711
:1008800047474747484848484848484848484849EB
:10089000494949494949494949494949494A4A4AC5
:1008A0004A4A4A4A4A4A4A4A4A4A4A4B4B4B4B4BA3
:1008B0004B4B4B4B4B4B4B4B4B4B4B4B4C4C4C4C84
:1008C0004C4C4C4C4C4C4C4C4C4C4C4C4C4C4C4D67
:1008D0004D4D4D4D4D4D4D4D4D4D4D4D4D4D4D4D48
:1008E0004D4D4D4D4D4E4E4E4E4E4E4E4E4E4E4E2D
:1008F0004E4E4E4E4E4E4E4E4E4E4E4E4E4E4E4F17
:100900004F4F4F4F4F4F4F4F4F4F4F4F4F4F4F4FF7
:100910004F4F4F4F4F4F4F4F4F4F4F4F4F4F000085
:100920008F001E01AD013B02CA025803E6037404A6
:1009300002058F051B06A7063307BE074808D20825
:100940005B09E3096B0AF20A780BFD0B810C040DBD
:10095000860D070E870E060F840F00107B10F51012
:100960006E11E5115B12CF124213B31323149214CC
:10097000FE146A15D3153B16A11605176717C8177D
:1009800027188318DE1837198E19E319361A871AB3
:10099000D61A231B6E1BB61BFD1B411C831CC31CDC
:1009A000001D3C1D751DAB1DE01D121E421E6F1E5D
:1009B0009A1EC31EE91E0D1F2E1F4D1F691F841F87
:1009C0009B1FB01FC31FD31FE11FEC1FF51FFB1F91
:1009D000FF1F002011241FBECFEFD0E1DEBFCDBF2F
:1009E00013E0A0E0B1E0ECEDFFEC02C005900D9249
:1009F000AC3DB107D9F71AE0ACEDB3E001C01D92F0
:100A0000AE31B107E1F70C9436060C940000282FA4
:100A1000FB018150853008F023E0842F992733278C
:100A200021503040829FD001839FB00D929FB00D26
:100A30001124AC59BF4F019724F00E94D067019256
:100A4000FACF0E948B610895863038F085E0A2E0ED
:100A5000B0E0082E0E94DD6708958823C1F708954D
:100A6000582F863048F155E0842F9927252F3327BA
:100A700021503040829FD001839FB00D929FB00DD6
:100A80001124AC59BF4FFB01019724F001900E9443
:100A9000DD67FACFA2E6B0E0042E0E94DD67A0E594
:100AA000B0E088E0FB01182E0E94E967852F0E94C4
:100AB00024050E948B6108958823B1F60895CF9391
:100AC000A2E0B0E00E94D067802DC82F8150853011
:100AD00020F0C3E08C2F0E9424058C2F9927CF9102
:100AE00008958091E608E82FFF27EE0FFF1FEC54D2
:100AF000F74F808191818D5E9F4F14F0109203011A
:100B0000808191818A5B9F4F24F480910301882327
:100B100019F02091830717C081E080930301209191
:100B20008307280F20938307253038F088EE93E061
:100B3000909301048093000406C066E970E0822F60
:100B40000E94CA2CE6CF822F992790935108809358
:100B5000500808951F93CF93DF93182F882351F4E3
:100B6000809104098233A0F080930001112309F4DD
:100B700079C038C080EA90E09F938F931F920E94C3
:100B80007E130F900F900F9080910409823360F7CD
:100B900084EF91E00E94FD16EC01112309F042C0A0
:100BA0008091270390912803823891050CF046C06C
:100BB0008091040923E0829FC001112480930001E9
:100BC0001123A1F268EC70E0822F0E94CA2C88EAFF
:100BD00090E09F938F931F920E947E130F900F902F
:100BE0000F90C4CF809100016AE00E946067892F56
:100BF00099279F938F93809100010E9460679927A6
:100C00009F938F938EEB90E09F938F931F920E9400
:100C10007E138DB79EB707960FB6F8949EBF0FBE92
:100C20008DBF20C0CE010E940617882309F0B8CFDF
:100C3000CE010E9406178823A9F3B2CF8091040940
:100C40009927880F991F880F991F809300011123FE
:100C500009F48CCF68EC70E084E00E94CA2C83EB2E
:100C600090E0B7CFDF91CF911F910895CFEFD0E102
:100C7000DEBFCDBF00E010E014B815B8C7EED3E07A
:100C8000E297D7FFFDCF189BACC2199BB5C22DE0F0
:100C90002093020181E887B93E9A8FEF88B98BE1F2
:100CA00084B981E085B98EE38AB987E48BB9469A25
:100CB00084B7877F84BF80916000886180936000E3
:100CC0001092600080ED97E09093010480930004FF
:100CD0001092DD041092DC041092B9081092B8084A
:100CE0001092DF041092DE041092E1041092E004EE
:100CF000243108F47CC288E894E0A0E0B0E080935E
:100D0000860390938703A0938803B09389032A30C6
:100D100009F4A0C2243109F49DC2289A0E946817E0
:100D20000E9439170E9453100E94B0270E94551844
:100D30000E94D1260E94C05D789488ED90E09F9338
:100D40008F931F920E947E130F900F900F9087E653
:100D500090E09F938F938CE490E09F938F931F92EA
:100D60001F92809102016AE00E946067892F992793
:100D70009F938F93809102010E94606799279F93B0
:100D80008F938EEF90E09F938F931F920E947E131C
:100D90008DB79EB70D960FB6F8949EBF0FBE8DBF50
:100DA00082E391E09F938F931F920E947E130F9096
:100DB0000F900F9082E891E09F938F931F920E9473
:100DC0007E130F900F900F908AEA91E09F938F937C
:100DD0001F920E947E138091C8000F900F900F9079
:100DE000803209F42FC2809102018C3008F0FDC1DD
:100DF000299A49E066EE78E083E00E940705C8EE94
:100E0000D3E0DE010E94D067802D813009F4F6C165
:100E100080ED91E09F938F931F920E947E130F901D
:100E20000F900F9028ED35E0F9018FE015861686BA
:100E30001786108A8150349687FFF8CF80E480931C
:100E4000E5058093E6051092E7058093E805809319
:100E5000E90590EC9093EA051092EB058093EC0580
:100E60008093ED051092EE059093EF059093F005B9
:100E70008093F1051092F2058093F3059093F405A9
:100E800081E08093D8058BE0A4E0B1E0E9EDF5E0E6
:100E90000D9001928A95E1F78DE4DE01F901182E9B
:100EA0000E94E967C0E0D0E061EFC62E61E0D62E77
:100EB00059EEE52E55E0F52EF70181917F01992736
:100EC00087FD90959F938F93DF93CF93DF92CF927F
:100ED0001F920E947E138DB79EB707960FB6F894A7
:100EE0009EBF0FBE8DBF2196CC30D1052CF3A1E063
:100EF000B0E00E94D067802D803509F065C2AEE079
:100F0000EA2EA0E0FA2ED7010E94D067802D992703
:100F1000582F442747010894811C911CD4010E943A
:100F2000D067802D480F511DECEFAE2EEFEFBE2E97
:100F3000AE0CBF1CD5010E94D067802D9927382F99
:100F400022276DEFC62E6FEFD62ECE0CDF1CD601FA
:100F50000E94D067802D280F311DEFEF2F3F3E07F5
:100F600009F4F4C2FFEF4F3F5F0709F4EFC230937B
:100F7000DD032093DC035093DF034093DE03809175
:100F8000DC039091DD039F938F938091DE0390911A
:100F9000DF039F938F938FE392E09F938F931F9232
:100FA0000E947E138DB79EB707960FB6F8949EBF2A
:100FB0000FBE8DBFA4E0B0E00E94D067802D8530C9
:100FC00008F0F3C20E945F0545E666EE78E00E94F5
:100FD00007050E945F0599279F938F9389E792E009
:100FE0009F938F931F920E947E138091EE080F9023
:100FF0000F900F900F900F9080FDB6C20E94113895
:10100000809102018A3009F4ADC2843109F4AAC288
:10101000289A80ED97E0909301048093000485E581
:101020008093850786EB92E09F938F931F920E9497
:101030007E138091EE080F900F900F9082FF8FC269
:1010400082EC92E09F938F931F920E947E130F90E9
:101050000F900F900E941C1E88E893E19093AD03BF
:101060008093AC0381E0809384070E94AA0580EE00
:1010700092E09F938F931F920E947E1380ED97E0E2
:101080000E94FD16EC010F900F900F9080910404C8
:10109000882309F49EC080911903882309F499C01C
:1010A0001092040480918307882309F408C10E94E8
:1010B00071050E94B13A209102012A3009F408C159
:1010C000243109F405C1289A8091E304882309F4A6
:1010D00005C18091E30481508093E3048091C705AA
:1010E000882369F081508093C705882341F41092CA
:1010F000C5051092C4051092C3051092C2058091D7
:10110000AC039091AD0301979093AD038093AC0332
:101110008091AC039091AD03892B29F080914B0411
:10112000882309F4E1C08091AC039091AD03892B31
:1011300009F410C180911203909113038F5F9F4FA8
:1011400009F421C180910404882321F08091D904FD
:10115000882311F40E948F100E94780DCE010E9406
:1011600006178823A1F1649680910F03882309F460
:10117000C9C0815080930F0380910001282F33272D
:101180008091270390912803821793070CF0B4C035
:101190008091B20480628093B20480911203909196
:1011A00013038F5F9F4F09F402C10E94B26084E075
:1011B0008093FF038091D904882311F40AEA15E093
:1011C0000F5F1F4F8BE00237180709F445C00E94DC
:1011D0009A618091FF03882309F058CF0E94F6603E
:1011E00055CF199B2DC024E153CD299802CE8BE019
:1011F00095E0A0E0B0E083CD2BE04ACDA1E0B0E0E7
:101200000E94D067802D8F3F09F402CE1092850393
:1012100028ED35E08DE4DE01F901182E0E94D86733
:1012200090918503F9013D962FE080813496181640
:101230000CF49F5F215027FFF8CF9093850332CEA7
:101240002AE026CD8091CA00863009F0CCCD0E94DC
:101250003A62C9CD289862CD00E010E02091DE030B
:101260003091DF032F5F3F4F3093DF032093DE0386
:101270008091DC039091DD0301969093DD038093D0
:10128000DC03832F9927D701082E0E94DD67809108
:10129000DE03D401082E0E94DD678091DD03D501B5
:1012A000082E0E94DD678091DC03D601082E0E9483
:1012B000DD6784E190E00E94FD16EC0188CF0E947A
:1012C000A83E0E94B13A209102012A3009F0F8CEDE
:1012D00028988091E304882309F0FBCE80916F0069
:1012E000806280936F00FACE2A3009F45EC0243108
:1012F00009F45BC0289A26CF8091B2048F7D809339
:10130000B20453CF80938F071092BE041092BD0495
:101310001092BC041092BB041092BA041092B9044B
:1013200080911203909113038F5F9F4F09F024CF98
:101330008091E304882309F01FCF88E99AE3909312
:1013400001048093000480E09CE090931303809359
:10135000120312CF0E94E72685E090E09093AD0340
:101360008093AC03809162089091630801969093FA
:1013700063088093620880911203909113038F5F3A
:101380009F4F09F0DFCE8091D904882309F4DACE8B
:1013900080E197E2909301048093000480E890E05C
:1013A0009093130380931203CDCE2898CBCE80E781
:1013B00097E1909301048093000480E093E0909380
:1013C000130380931203F1CE0E94512A88EF91E01B
:1013D0009F938F931F920E947E1341E0942E0F9053
:1013E0000F900F90C0E5D0E07E010894E11CF11C45
:1013F00032E0C32ED12CCC0EDD1E23E0A22EB12C68
:10140000AC0EBD1E94E0692E712C6C0E7D1E85E025
:10141000482E512C4C0E5D1EB6E02B2E312C2C0E7E
:101420003D1E92E0991609F48BC0E3E09E1609F484
:101430008AC0F3E0F91508F483C080910201843179
:1014400068F085E08093010910921F098BE1809379
:10145000FD088EE480931C0980931D09DE010E9423
:10146000D067802D8C3008F068C0D7010E94D0670B
:10147000802D8C3008F061C0D6010E94D067802D8D
:101480008C3008F05AC0D5010E94D067802D8C3076
:1014900008F053C0DE010E94D067802D8093E608DB
:1014A000D7010E94D067802D8093E708D6010E9463
:1014B000D067802D8093E808D5010E94D067802DE9
:1014C0008093E908D3010E94D067802D8093EA08B9
:1014D000D2010E94D067802D8093EB08D1010E9439
:1014E000D067802D8093EC08A7E5B0E00E94D0671C
:1014F000802D8093ED0821E0921651F487E092E070
:101500009F938F931F920E947E130F900F900F90C6
:1015100045E666EE78E0892D0E943005939495E0CB
:10152000991508F07ECF83E00E94240580E5A1E0B4
:10153000B0E0082E0E94DD67E2CC0E94382AE8CF96
:101540000E941E2B7ACF0E94E92B77CF1092DF03E7
:101550001092DE031092DD031092DC0310CD8EECAE
:1015600092E070CD289855CD81E992E09F938F93BA
:101570001F920E947E1388EE93E00E94FD16EC01FC
:101580000E945B180F900F900F90CE010E940617DB
:101590008823D9F381EB92E09F938F931F920E944F
:1015A0007E130F900F900F9029CD82E692E09F93CB
:1015B0008F931F920E947E130F900F900F9002CD79
:1015C0001F920F920FB60F9211248F939F93EF9358
:1015D000FF93809111038823A9F48091F3039091E4
:1015E000F4030196FC01EB5CF94FE081ED3079F0FA
:1015F0008639910561F09093F4038093F303E093AF
:10160000C6000EC01092F4031092F30309C01092AA
:10161000F4031092F30381E080931103E093C6007A
:10162000FF91EF919F918F910F900FBE0F901F90A0
:1016300018951F920F920FB60F9211242F933F937C
:101640004F935F938F939F93AF93BF93EF93FF93CA
:1016500090E08091C6008093EB035091F9035639D6
:1016600010F09093FA038091EB038D3091F020916C
:10167000FA03822F99278130910509F46AC08230DC
:1016800091050CF48CC0029709F47DC01092FA0306
:10169000A6C02091FA03223061F79093FA03852FB8
:1016A00099278E56984FFC01329740812091F5037F
:1016B0003091F603241B3109DC0111978C91281B12
:1016C0003109C9019F709093F6038093F5030024BC
:1016D000880F991F001C880F991F001C892F902DBF
:1016E000982F935C9093F7032F733070235C2093B3
:1016F000F8038081891709F46CC090E08091E803B9
:101700008F5F8093E8038091EA03882309F067C024
:10171000992309F464C081E08093EA03580F509341
:10172000E7035150E52FFF27EE56F84F8DE08083F9
:1017300080919407823509F052C088E190E02CE056
:101740000FB6F894A895809360000FBE20936000B8
:1017500046C02F5F2093FA03E52FFF27EE56F84F80
:101760008091EB0380835F5F5093F9032091EB033B
:101770008091F5039091F603820F911D9093F603EB
:101780008093F5032CC0E52FFF27EE56F84F80918C
:10179000EB038083563938F31092FA03E7CF892B95
:1017A00009F074CF8091EB03833259F08091EB0301
:1017B0008093920781E08093F9038091EB0399274E
:1017C000DDCF8091EA03882389F781E08093FA03D3
:1017D000EDCF8C91821709F090CF91E094CFFF91DB
:1017E000EF91BF91AF919F918F915F914F913F91F9
:1017F0002F910F900FBE0F901F901895AC01A0E095
:10180000B0E09D01A817B90748F4E5E3F6E081913F
:10181000280F311D1196A417B507C8F33F70FD01BD
:10182000EB5CF94FC9010024880F991F001C880F39
:10183000991F001C892F902D835C80831196FD01D8
:10184000EB5CF94F2F733070822F835C8083AA5C2E
:10185000B94F8DE08C9310921103809135068093DF
:10186000C6000895BF92CF92DF92EF92FF920F933E
:101870001F93CF93DF93CDB7DEB72C859D857E85F3
:10188000BB2483E2809335069F59909336062093BC
:10189000370603E010E0772309F4ADC0CF84D88881
:1018A00043E1E42EF12CEC0EFD1EA989BA8971509A
:1018B000109709F4A0C0109709F43CC0F601EB0D95
:1018C000F11DB3949081119789F47723A1F1F70169
:1018D00022E030E0E20EF31ED701C080D180E20E9C
:1018E000F31E0D90BC91A02DBB247150109719F1DF
:1018F000F601EB0DF11DB3944081119709F466C018
:101900001097D1F0F601EB0DF11DB39460811197A2
:10191000A1F4772391F0F7013296D701CD90DC90B6
:1019200032E0E32EF12CEE0EFF1EA081B181BB242C
:10193000715003C090E040E060E0F801EB5CF94FCB
:10194000892F86958695835C80830F5F1F4FF801F2
:10195000EB5CF94F892F992783709070829592954F
:10196000907F9827807F982755279A013295229556
:101970002F7023273F702327822B835C80830F5F88
:101980001F4FF801EB5CF94F4F705070440F551F1B
:10199000440F551F862F99270024880F991F001C7C
:1019A000880F991F001C892F902D842B835C8083C6
:1019B0000F5F1F4FF801EB5CF94F6F73635C60833F
:1019C0000F5F1F4F109709F076CF15C0772309F4EA
:1019D000B3CFF701A2E0B0E0EA0EFB1ED701C08052
:1019E000D18022E030E0E20EF31E0D90BC91A02DDC
:1019F000BB24715085CFC8010E94FE0BDF91CF91AF
:101A00001F910F91FF90EF90DF90CF90BF900895BE
:101A1000A3E07A2F4091E703465009F45FC0E72F17
:101A2000FF27EE56F84F80818D537F5FE72FFF270A
:101A3000EE56F84F20812D537F5FE72FFF27EE569C
:101A4000F84F30813D537F5FE72FFF27EE56F84F69
:101A500060816D537F5F9927880F991F880F991FA9
:101A6000522F52955F70582B822F99278F7090704C
:101A700082959295907F9827807F9827232F26958F
:101A80002695282B832F9927837090700024969594
:101A900087950794969587950794982F802D682BA6
:101AA00041504F3FD9F0EA2FFF27EE56F84F5083B1
:101AB000AF5F41504F3F91F0EA2FFF27EE56F84FAE
:101AC0002083AF5F41504F3F49F0EA2FFF27EE568A
:101AD000F84F6083AF5F442309F0A1CF85E997E019
:101AE0009093E6038093E503A350A093E403089545
:101AF000CF93DF93CDB7DEB722970FB6F894DEBF52
:101B00000FBECDBF8091EA03882309F4AFC20E94C3
:101B1000080D80919307823609F471C08091940773
:101B200099278436910509F457C08536910584F5C7
:101B30008136910509F44EC1823691050CF4C2C07C
:101B40008236910509F49AC183369105C1F48091DA
:101B5000E0039091E103892B09F04FC2A091E503C6
:101B6000B091E6039C91992309F03DC29C918AE0D3
:101B7000989FC00111249093E1038093E003109299
:101B8000EA031092E6031092E5031092E4036EC29A
:101B90008C36910509F410C18D3691050CF0B3C057
:101BA0008736910509F42BC18836910541F78FEFEF
:101BB00080930F03E091E503F091E603808190911B
:101BC0004404892B80934404882311F01092EC0381
:101BD00081E08093F003D3CFE091E503F091E60339
:101BE00090818AE0989FC001112490930D03809307
:101BF0000C03892B21F281E08093EF03C0CF809109
:101C0000940799278037910509F4F2C0813791052F
:101C10000CF485C08337910509F45BC184379105C5
:101C20000CF03CC18137910509F078CFA091E50314
:101C3000B091E6038C918F3F09F40CC28C918823FC
:101C400009F003C281E08C93A091E503B091E60313
:101C500045E666EE78E08C910E94070580911103BD
:101C60008823E1F3E091E503F091E6038081898325
:101C700080E58A8385E690E09F938F9386EE98E0D7
:101C80009F938F9321E030E03F932F93CE010296F4
:101C90009F938F933F932F93CE01820F931F9F9318
:101CA0008F9383E08F9381E08F9381E58F930E94E0
:101CB000320CADB7BEB71F960FB6F894BEBF0FBEBD
:101CC000ADBF2CCF8B34910509F059CFE091E503DE
:101CD000F091E603808191819093F5048093F40460
:101CE0002091F2043091F304821B930B845E9D4F8C
:101CF00068E671E00E948067845B90409093F104F5
:101D00008093F0043CCF8437910509F47CC086377A
:101D1000910509F034CF81E08093EE0330CF8D360A
:101D2000910529F18E3691050CF093C08B34910505
:101D300009F0F4CEA091E503B091E6038D919C915A
:101D40009093F5048093F4042091F2043091F3040D
:101D5000821B930B845E9D4F68E671E00E94806752
:101D6000845B90409093F1048093F004D7CE8091EF
:101D700011038823E1F3A091E503B091E6039C9160
:101D8000913009F43FC1198281E090E09F938F93D5
:101D9000CE0101969F938F9381E08F938F938DE473
:101DA0008F930E94320C8DB79EB707960FB6F894AA
:101DB0009EBF0FBE8DBFB2CE8FEF80930F03E09119
:101DC000E503F091E60380818093450481E08093F0
:101DD000F103D5CEE091E503F091E603E081E03236
:101DE00058F08FE1809310038FEF80930F03C7CEDD
:101DF00081E08093ED0392CEE0931003F5CF81E074
:101E00008093F203BCCE8091E703853108F4DAC0F9
:101E1000E091E503F091E60380E1ADE6B7E00190E3
:101E20000D928A95E1F7809111038823E1F31F92C7
:101E300080910E038F9384E58F930E94320C8AEF7A
:101E40008093E2038FEF80930F030F900F900F901A
:101E500096CE8E36910509F061CE809111038823CC
:101E6000E1F38DE490E09F938F9388ED95E09F934D
:101E70008F9381E08F938F938EE492CFA091E503AF
:101E8000B091E6038BE0E5E8F7E00D9001928A95CA
:101E9000E1F780918E0780936A08A6CF8437910579
:101EA00009F03CCE8091E703853108F4BCC0A091D5
:101EB000E503B091E60380E1EDE6F7E00D900192D5
:101EC0008A95E1F780EF8093E2038FEF80930F0311
:101ED00025CE2091E5033091E603F9018081815000
:101EE000853018F481818035E9F0198280911103E1
:101EF0008823E1F381E090E09F938F93CE010196D8
:101F00009F938F9381E08F938F9383E58F930E94AC
:101F1000320CEDB7FEB737960FB6F894FEBF0FBE82
:101F2000EDBFFCCD66EE78E085E62E5F3F4FDB012E
:101F3000F901982F01900D929A95E1F722503040C7
:101F4000482FD9018C910E94300580911C09992756
:101F5000AA27BB27BC01CD0124EC39E040E050E0CA
:101F60000E944167DC01CB018093A6039093A703F5
:101F7000A093A803B093A90380911D099927AA27CC
:101F8000BB27BC01CD010E944167DC01CB018093DE
:101F9000A2039093A303A093A403B093A503E0919D
:101FA000E503F091E60380810E9424050E945F050D
:101FB000898380E00E94AA056EE670E089810E9414
:101FC000CA2C94CFE091E503F091E60380819181E2
:101FD000A281B38180936D0790936E07A0936F07E2
:101FE000B093700720CF8AE0989FC00111240E940F
:101FF000FD169093340680933306A091E503B091CB
:10200000E603B4CD48ED55E08DE4FA01282F0D909C
:1020100001922A95E1F7A8EEB3E0FA01182E0E948A
:10202000E9679983B1CEA091E503B091E6038D9164
:102030009D910D90BC91A02D80936D0790936E079C
:10204000A0936F07B09370073DCF863008F400CEA1
:1020500085E0F9CD0E945F05E091E503F091E6038C
:102060008083A091E503B091E603E8CD22960FB6F8
:10207000F894DEBF0FBECDBFDF91CF910895CF930F
:10208000C82F8A3029F08091C00085FFFCCF04C0A2
:102090008DE00E943F10F7CFC093C60080E090E033
:1020A000CF910895089588E18093C1008091C00088
:1020B00082608093C0008091C10080688093C100DD
:1020C0008091C10080648093C1008AE28093C40043
:1020D00080910C0390910D030E94FD16909362076E
:1020E000809361078CED90E00E94FD16909391071C
:1020F00080939007109263078CE48093640786E0D6
:10210000809367078AE08093650781E08093660784
:102110001092E6031092E5031092E4030895EF9203
:10212000FF920F931F9380911103882309F478C2C3
:102130008091F003882309F082C08091F103882305
:1021400029F080911103882309F07FC18091EE036B
:10215000882329F080911103882309F05BC18091C5
:10216000F203882329F080911103882309F036C1F6
:1021700080919007909191070E940617882329F07B
:1021800080911103882309F0C8C080910C039091BD
:102190000D03892B09F084C18091EF03882329F076
:1021A00080911103882309F00FC28091E003909180
:1021B000E103892B09F07EC1209110032F3F59F1D3
:1021C00080E190E09F938F93822F9927829592953B
:1021D000907F9827807F9827845F9E4F9F938F934F
:1021E00081E090E09F938F9380E193E09F938F93A2
:1021F00082E08F9381E08F9381E48F930E94320C71
:102200008FEF809310038DB79EB70B960FB6F8949F
:102210009EBF0FBE8DBF80916A08882329F08091F0
:102220001103882309F05EC08091ED03882309F42F
:10223000F7C180911103882309F4F2C139C080915C
:102240001103882309F479CF0E94251E84E190E0D0
:102250009F938F939091EC0384E1989FC001112488
:10226000865D9C4F9F938F9381E090E09F938F9327
:102270008CEE93E09F938F9382E08F9381E08F9316
:1022800088E48F930E94320C8091EC038F5F2DB70E
:102290003EB7255F3F4F0FB6F8943EBF0FBE2DBF30
:1022A000843008F4B8C11092EC031092F00345CFCB
:1022B00086E190E09F938F9384EB98E09F938F93B8
:1022C00081E08F938F9380E58F930E94320C109260
:1022D000ED038DB79EB707960FB6F8949EBF0FBE5D
:1022E0008DBF9EC181E090E09F938F938AE698E036
:1022F0009F938F9381E08F938F9382E48F930E94BB
:10230000320C10926A082DB73EB7295F3F4F0FB6C7
:10231000F8943EBF0FBE2DBF87CF8091FD0899274F
:10232000880F991F880F991F7C010027F7FC0095E3
:10233000102F80912E0590912F05A0913005B0911E
:102340003105BC01CD01A80197010E94B56730930A
:102350007E0720937D078091260590912705A09107
:102360002805B0912905BC01CD01A80197010E9463
:10237000B5673093800720937F078091C6048093D0
:1023800081078091C5048093820788E090E09F9345
:102390008F938DE797E09F938F9381E08F9383E0F6
:1023A0008F9387E78F930E94320C809183072DB71C
:1023B0003EB7295F3F4F0FB6F8943EBF0FBE2DBF0B
:1023C000853018F086E08093830783E690E00E94D2
:1023D000FD169093910780939007D7CE8BE090E005
:1023E0009F938F9385E897E09F938F9381E08F93DE
:1023F00080910E038F9387E48F930E94320C10928A
:10240000F2038DB79EB707960FB6F8949EBF0FBE26
:102410008DBFAECE8AE090E09F938F9383E697E0E6
:102420009F938F9381E08F938F9386E58F930E9484
:10243000320C1092EE032DB73EB7295F3F4F0FB617
:10244000F8943EBF0FBE2DBF8ACE0E94251E80E5A8
:1024500090E09F938F938AE293E09F938F9321E084
:1024600030E03F932F9389E293E09F938F933F93C4
:102470002F9385E494E09F938F9383E08F9381E083
:102480008F938CE48F930E94320C1092F1038DB7DE
:102490009EB70F960FB6F8949EBF0FBE8DBF56CE57
:1024A00080916107909162070E940617882309F0C6
:1024B00077CE72CE80913306909134060E94061733
:1024C000882309F479CE80911103882309F474CE0E
:1024D0008091FD089927880F991F880F991F7C010B
:1024E0000027F7FC0095102F80912E0590912F0565
:1024F000A0913005B0913105BC01CD01A801970133
:102500000E94B56730932606209325068091260504
:1025100090912705A0912805B0912905BC01CD0116
:10252000A80197010E94B5673093280620932706DB
:102530002091B0093091B1094091B2095091B3098D
:10254000DA01C90103E0880F991FAA1FBB1F0A9572
:10255000D1F7820F931FA41FB51F820F931FA41FD3
:10256000B51F2091860330918703409188035091D5
:102570008903BC01CD010E94B56730932A062093E0
:1025800029068EE090E09F938F9385E296E09F93DB
:102590008F9381E08F938F9383E48F930E94320C0B
:1025A0008091E0039091E1030E94FD169093340620
:1025B000809333062DB73EB7295F3F4F0FB6F8948F
:1025C0003EBF0FBE2DBFF8CD82E490E09F938F9366
:1025D00088E298E09F938F9381E08F938F9384E4B8
:1025E0008F930E94320C1092EF038DB79EB707961F
:1025F0000FB6F8949EBF0FBE8DBF80910C039091D3
:102600000D03009709F4D1CD0E94FD169093620747
:1026100080936107CACD8093EC031092F0038DCDB7
:102620001F910F91FF90EF900895982F80916B0864
:10263000813031F0892F0E943F10282F33270CC0A2
:1026400080914604E82FFF27E65DFC4F90838F5F63
:102650008093460421E030E0C90108950F931F9351
:10266000CF93DF938C01EB01672B71F0F80181911F
:102670008F010E941513219739F0F80181918F0184
:102680000E941513219791F7DF91CF911F910F9120
:1026900008950F931F93CF93DF938C01EB01672B6A
:1026A00081F0F8010F5F1F4F84910E94151321974D
:1026B00041F0F8010F5F1F4F84910E94151321977D
:1026C00081F7DF91CF911F910F910895CF93C82F7C
:1026D000181634F480E20E941513C1501C16D4F36E
:1026E000CF910895CF93C82F181634F480E30E9439
:1026F0001513C1501C16D4F3CF9108952F923F9219
:102700004F925F926F927F928F929F92AF92BF9201
:10271000CF92DF92EF92FF920F931F93CF93DF93AD
:10272000CDB7DEB7E0970FB6F894DEBF0FBECDBFD2
:1027300026968FAD26972896EEADFFAD2897882474
:102740009924540180936B0848E4C42ED12CCC0EFC
:10275000DD1E7F01C701F7011491112331F01532FD
:1027600021F00894E11CF11CF6CFB701681B790B2E
:1027700009F095C0112309F43DC20894E11CF11C35
:102780001FA63FA4232C0FEF39A6F7010894E11CE4
:10279000F11C14911537C9F1812F80628837A9F196
:1027A000103209F440C0133209F48DC01A3209F412
:1027B00079C01D3209F476C01B32C9F11E32C9F14D
:1027C000103309F48AC0812F8153893008F07EC00C
:1027D00060E070E0CB01880F991F880F991F880F68
:1027E000991F860F971F680F791F610F711D605326
:1027F0007040F7010894E11CF11C1491812F805363
:102800008A3040F3262E153739F630FE3DC0F601EA
:1028100084E090E0C80ED91E80809180A280B380B1
:10282000103209F0C0CF89A5882309F0AECF19A7CF
:10283000ACCFF7010894E11CF11C14911A3209F491
:1028400051C060E070E014C0CB01880F991F880F61
:10285000991F880F991F860F971F680F791F610FA7
:10286000711D60537040F7010894E11CF11C149134
:10287000812F80538A3040F3EFEF6F3F7E0714F4CF
:102880006FEF7FEF062F86CFF60182E090E0C80E53
:10289000D91E808191814C01AA24BB2481CF0E9442
:1028A000491368CF1A3251F4F60182E090E0C80E65
:1028B000D91E208022200CF068CF219490E1392A83
:1028C000EFED3E2262CF98E0392A5FCF1836C9F08B
:1028D0001C36D1F481E0382A58CF34FC56CFF0E2D0
:1028E0003F2A53CFF60182E090E0C80ED91E6081E6
:1028F00071819FEF6F3F790714F46FEF7FEF062F21
:1029000044CF24E0322A41CF133609F44DC11434A8
:1029100009F41FC1143609F41CC1193609F419C190
:102920001F3409F40FC11F3609F40CC1103709F424
:10293000F9C0133709F4B2C0153509F4ECC01537E6
:1029400009F4E9C0183509F444C0183709F441C046
:10295000112309F44FC1CE0101969DA78CA71983BD
:1029600081E0482E19A6632C7724042D5FA4541807
:1029700057FC2DC029A5222331F10F5F050DC3019E
:1029800080739070892B09F42FC1222309F027C18D
:1029900066FC1BC1C30180739070809709F410C15D
:1029A000852D0E947213842D992787FD9095BC0177
:1029B0008CA59DA50E942E1364FECCCE822D801B7B
:1029C0000E946613C7CE66FED9CF0E5FD7CF5524BF
:1029D000D1CFE0E1EEA733FE07C081149104A1043A
:1029E000B10411F0F0E43F2A19A60FA707FD02C0B9
:1029F0002FED3222CE0189969DA78CA781149104D8
:102A0000A104B10419F49FA5992361F1EEA54E2EFE
:102A100055246624772418AA84149504A604B704C0
:102A200010F0F1E0F8ABC501B401A30192010E94DE
:102A30009367DC01CB01082F8A30F0F4005DECA530
:102A4000FDA50293FDA7ECA7C501B401A301920166
:102A50000E94936749015A01F8A9FF23E1F62EA5C8
:102A6000283079F0632C7724CE010196482EFCA5FE
:102A70004F1A28E2420E79CF095A183501F70F7D17
:102A8000DECF632C772463FEEFCF003369F380E35E
:102A9000ECA5FDA58293FDA7ECA7E6CFF60182E0A9
:102AA00090E0C80ED91E0190F081E02DFDA7ECA7A3
:102AB000EF2B81F4FE013196FDA7ECA788E2898314
:102AC0008EE6818385E78B838CE68C838D8389E218
:102AD0008E831F8207FD15C0802F992787FD909553
:102AE000AC0160E070E08CA59DA50E945A6600973D
:102AF00031F0482EFCA54F1A04150CF033CF402EB0
:102B000031CFECA5FDA501900020E9F731974E2EBD
:102B10002CA5421A27CF153511F481E0382A9AE006
:102B20009EA762CFF60182E090E0C80ED91E808198
:102B300091814C01AA24BB2490E19EA7E0E43E2AA7
:102B400018E752CF1F3411F4E1E03E2AF8E0FEA767
:102B50004BCF143411F491E0392A30FE18C0F6013D
:102B600084E090E0C80ED91E80809180A280B3805E
:102B7000B7FE0AC0B094A09490948094811C911CDC
:102B8000A11CB11C8DE289A79AE09EA72ECFF60169
:102B900082E090E0C80ED91E808191814C01AA2468
:102BA00097FCA094BA2CE4CFFE013196FDA7ECA7C8
:102BB000F60182E090E0C80ED91E80818983D0CED4
:102BC000822D801B0E947213EBCE80E38AA71BA785
:102BD00062E070E0CE018A960E942E13DBCE61E0A7
:102BE00070E0CE018996F8CF822D801B0E9466137B
:102BF00029A5CBCEE0960FB6F894DEBF0FBECDBFB1
:102C0000DF91CF911F910F91FF90EF90DF90CF90C8
:102C1000BF90AF909F908F907F906F905F904F90FC
:102C20003F902F9008951F920F920FB60F9211248C
:102C30002F933F935F936F937F938F939F93AF9364
:102C4000BF93EF93FF938091FF03882329F0809136
:102C5000FF0381508093FF038091D305882319F0EF
:102C600081508093D3058091070481508F3F09F4F0
:102C700093C0809307048091000490910104892BF4
:102C800001F1809100049091010401979093010457
:102C9000809300048091000490910104209112031C
:102CA0003091130382239323892B89F080910201B1
:102CB0008A3009F48BC0479A8091EE0883FF8DC05B
:102CC00010C08FEF9FEF90931303809312038091B6
:102CD00002018A3009F478C047988091EE0883FF9A
:102CE0007CC086B19927FC01E071F07084FF0AC0B6
:102CF00080910204909103040196909303048093C1
:102D000002046BC08091020490910304892B49F165
:102D100080910204909103048A56914010F58091AD
:102D200002049091030469E270E00E946C67809154
:102D3000020490910304860F971F909303048093DD
:102D4000020480910204909103040B9708F440C0A0
:102D500080910204909103040A979093F504809364
:102D6000F4048091F4049091F5042091F2043091E0
:102D7000F304821B930B845E9D4F68E671E00E9412
:102D80008067845B90409093F1048093F0041092EC
:102D900003041092020421C089E08093070480910B
:102DA00014038F5F817080931403882319F481E0EA
:102DB00080930404809105049091060401969093F9
:102DC00006048093050457CF5A9887CF5A9A85CF27
:102DD000F093F504E093F404C4CFFF91EF91BF9119
:102DE000AF919F918F917F916F915F913F912F91C3
:102DF0000F900FBE0F901F901895209105043091F1
:102E00000604280F391FC901019608952091050471
:102E100030910604821B930B892F99278695807425
:102E200090700895CF93DF930E94FD16EC01CE01C0
:102E30000E9406178823D9F3DF91CF9108951F933D
:102E4000CF93DF930E94FD16EC011FEC08C0809128
:102E50001903882321F09093190310937A00CE016F
:102E60000E940617982F882391F3DF91CF911F912D
:102E700008959FB7F8945F983E9A469A8091B00063
:102E80008F708093B0008091B00083608093B00019
:102E90008091B1008B738093B1008091B1008B6001
:102EA0008093B1001092B2008FEF8093B3008091B5
:102EB000B00080688093B000809170008A7F80931A
:102EC0007000809170008260809370009FBF0895B1
:102ED0008AE090E00E94FD1690930F0480930E0408
:102EE00082E085BD83EA84BD17BC88E788BD86E0A3
:102EF00086BD80916E00816080936E0008951F9260
:102F00000F920FB60F9211242F933F934F935F931D
:102F10008F939F93EF93FF93209108042223C9F589
:102F20008091B00086FF63C08091B0008F7B80935A
:102F3000B000E0910D04EE2309F479C0FF27EB52B5
:102F4000FC4F80819927880F991F87559C4F55E02A
:102F50008D3D950708F494C08CED95E090930A049C
:102F6000809309042091090430910A042C5B3040BD
:102F700030930A042093090480910B0490910C046F
:102F8000820F931F90930C0480930B0481E0809335
:102F900008042091090430910A0441E02F373407D6
:102FA00050F08FEF8093B3002F5F304030930A04CE
:102FB000209309046DC02F3F310571F068F0A9011D
:102FC0004F5F50404F37510508F052C080E8809362
:102FD000B30020583040EACF809109048093B300B9
:102FE00010920A04109209041092080451C08091B2
:102FF000B00080648093B0008CEB90E090930A0462
:103000008093090480910B0490910C0484549F4F89
:1030100090930C0480930B04469890910D049F5F4D
:1030200080911509891708F520930D04AFCF809181
:103030001509282F33278DED96E0289FA001299FA1
:10304000500D389F500D1124CA0120910B0430916E
:103050000C04821B930B90930A0480930904109232
:103060000C0410920B04469A91CF90930D048ECFCE
:103070008FEF8093B30050930A044093090408C073
:1030800021E08737920708F069CF87E791E066CFA4
:10309000FF91EF919F918F915F914F913F912F9170
:1030A0000F900FBE0F901F90189510927C008FEC20
:1030B00080937A000895EF92FF920F931F93CF931E
:1030C000DF9303E010E0D8010E94D067802DC82F65
:1030D000DD27C531D10508F02A97C7BD1092170426
:1030E00084E690E00E941F1780911D0390911E03BB
:1030F0008052934010F4C0E0D0E0CA3FD105E0F424
:1031000088E0E82E83E0F82EC7BD82E390E00E94BD
:103110001F17FF92EF921F920E947E1380911D0352
:1031200090911E030F900F900F908052934020F0CB
:103130002196CA3FD10540F3D8010C2E0E94DD67CD
:10314000C09378088CE291E00E941F17DF91CF9125
:103150001F910F91FF90EF900895EF92FF920F93C0
:103160001F93CF93DF9300E00093120400931104A8
:103170000093100480ED97E00E94FD16EC011CE81E
:1031800021E0F22E95EFE92E033009F4ABC000E008
:1031900080912704909128048C5F93400CF091C09B
:1031A00080911C03815080931C0380912504909191
:1031B00026048C5F93400CF079C080911B038150F2
:1031C00080931B0380912304909124048C5F93408F
:1031D0000CF04AC080911A03815080931A0388E052
:1031E00080934E040E94D72680911C038A3008F0F9
:1031F00055C0F09212048AE080931C0380911B0357
:103200008A3008F043C0F09211048AE080931B03D7
:1032100080911A038A3098F5F09210048AE0809326
:103220001A0380914E04882379F0CE010E9406177C
:103230008823B9F38AE093E09F938F931F920E94B3
:103240007E130F900F900F90109219038FEC8093C4
:103250007A00809119038823E1F31A3008F447C0FB
:10326000115009F091CF48C080912304909124041B
:10327000875094408CF180911A038F5FAECF863FC8
:1032800080F2F0921004E0921A03CBCF863F08F44C
:10329000BFCFF0921104E0921B03BACF863F08F42F
:1032A000ADCFF0921204E0921C03A8CF80912504C8
:1032B00090912604875094408CF080911B038F5F7F
:1032C0007FCF80912704909128048750944044F048
:1032D00080911C038F5F67CF0F5F81CF0F5F72CF2D
:1032E00001E063CF1B3008F452CF19E050CF8AE0E1
:1032F00090E00E941F17B4CF86E490E00E941F1751
:10330000DF91CF911F910F91FF90EF9008951F9241
:103310000F920FB60F921124AF92BF92CF92DF920D
:10332000EF92FF920F931F932F933F934F935F93CF
:103330006F937F938F939F93AF93BF93EF93FF937D
:1033400020913004822F9927AA27BB272F5FFC01E9
:10335000429740F4E25CFF4FEE0FFF1F0590F4919F
:10336000E02D09941092300482E080932F04809124
:103370002F0480937C0080913004882309F443C497
:103380008FEC80937A003FC42093300480917800C2
:10339000909179002091350430913604820F931F6B
:1033A000909336048093350481E0DFCF209330047E
:1033B0008091780090917900209133043091340409
:1033C000820F931F909334048093330484E0CDCF15
:1033D00020933004809178009091790020913C05F1
:1033E00030913D05821B930B90937708809376086C
:1033F000809176089091770890933E0480933D04E5
:1034000082E0B3CF2093300480913A0590913B0540
:103410002091780030917900821B930B90936D0876
:1034200080936C0880916C0890916D0890933C0497
:1034300080933B0487E099CF2093300480917800FB
:1034400090917900909332048093310486E08DCF7F
:103450002093300420917800309179003093340427
:103460002093330410922F0482CF209330042091B4
:10347000780030917900309336042093350481E050
:1034800074CF1092300481E080931903809113046B
:1034900090911404019690931404809313048091E6
:1034A00078009091790090931E0380931D03809182
:1034B0001D0390911E035C01CC24DD2480913F0408
:1034C00090914004A0914104B0914204A80EB91E0D
:1034D000CA1EDB1E809143048F5F823108F4E8C26C
:1034E00080911F0390912003A0912103B0912203AA
:1034F0007C018D0123E0EE0CFF1C001F111F2A959B
:10350000D1F7E81AF90A0A0B1B0BEA0CFB1C0C1D7D
:103510001D1D80911704992787FD9095A92FB92F1C
:10352000BC01CD0126EC34E240E050E00E9441674E
:10353000DC01CB01E81AF90A0A0B1B0BD801C70101
:103540000496A11DB11DB7FD23C313E0B595A79542
:10355000979587951A95D1F780931F039093200331
:10356000A0932103B0932203809170089091710879
:103570007C010027F7FC0095102F80911F0390918C
:103580002003A0912103B0912203E81AF90A0A0B43
:103590001B0BE092D504F092D6040093D70410934D
:1035A000D804209118043091190440911A045091C4
:1035B0001B0457FDFDC2A4E0559547953795279507
:1035C000AA95D1F78091180490911904A0911A043A
:1035D000B0911B04821B930BA40BB50B80931804B2
:1035E00090931904A0931A04B0931B0480911804BB
:1035F00090911904A0911A04B0911B048E0D9F1D87
:10360000A01FB11F8093180490931904A0931A046B
:10361000B0931B048091150490911604BC0162952F
:103620007295707F7627607F7627681B790B2091D3
:1036300018043091190440911A0450911B0457FD4D
:10364000B2C2E4E05595479537952795EA95D1F7AD
:103650008091D5049091D604821B930B880F991FFB
:10366000880F991F880F991F860F971F97FDA9C272
:103670009595879595958795959587959595879532
:103680009093160480931504D601C501D7FC95C20A
:10369000B595A7959795879580933F04909340049F
:1036A000A0934104B093420489E08093430482E0F4
:1036B0005CCE209330042091780030917900809185
:1036C000330490913404280F391F809102018A300D
:1036D00009F448C2220F331F220F331F30933404E2
:1036E00020933304C90137FD73C29595879595954D
:1036F00087959595879590932604809325048091CE
:10370000390490913A04820F931F97FD66C29595F4
:10371000879590933A048093390420914405309121
:103720004505821B930B90932403809323032091E0
:103730002B0430912C048091230390912403280FB3
:10374000391F37FD47C23595279530932C042093B8
:103750002B0483E00ACE209330042091780030912E
:1037600079008091350490913604280F391F80919B
:1037700002018A3009F407C2220F331F220F331FC0
:103780003093360420933504C90137FDFFC1959568
:10379000879595958795959587959093280480931F
:1037A00027048091370490913804820F931F97FD6E
:1037B0000DC2959587959093380480933704209196
:1037C000460530914705821B930B90932603809307
:1037D000250320912D0430912E0480912503909192
:1037E0002603280F391F37FDEEC1359527953093F5
:1037F0002E0420932D0481E0B8CD209330048091D5
:1038000078009091790020913C0530913D05821B14
:10381000930B909377088093760880917608909127
:10382000770820913D0430913E04820F931F9093BE
:10383000200480931F0482E098CD2093300480916F
:103840003A0590913B052091780030917900821BD8
:10385000930B90936D0880936C0880916C08909105
:103860006D0820913B0430913C04820F931F90938C
:1038700022048093210487E078CD20933004809146
:1038800002018A3009F471C1843109F4A8C1809120
:103890007800909179002091310430913204820FA8
:1038A000931F909324048093230486E05ECD20939D
:1038B0003004809178009091790020913304309108
:1038C0003404820F931F9093340480933304109236
:1038D0002F044DCD20933004E2CD2093300480910D
:1038E000780090917900AA2797FDA095BA2FBC0186
:1038F000CD010E94C7667B018C01809134059091B7
:103900003505A0913605B09137059C01AD01C80180
:10391000B7010E946766DC01CB01BC01CD010E94AA
:10392000AA66DC01CB0190931E0480931D04809154
:103930001D0490911E0402970CF4C6C080913405BA
:1039400090913505A0913605B091370520E030E81B
:103950004BE354E4BC01CD010E94D1668823DCF521
:103960008091340590913505A0913605B0913705C9
:103970002AE037ED43EA5CE3BC01CD010E946866B2
:10398000DC01CB018093340590933505A093360577
:10399000B09337058091B3049091B404845F914053
:1039A000D0F48091340590913505A0913605B09101
:1039B00037052DEC3CEC4CEC5DE3BC01CD010E94E5
:1039C0006866DC01CB018093340590933505A093A4
:1039D0003605B093370581E080931C048091780010
:1039E0009091790090936F0880936E0880911D04E8
:1039F00090911E04AA2797FDA095BA2F2091F60456
:103A00003091F7044091F8045091F904820F931F0C
:103A1000A41FB51F8093F6049093F704A093F804B5
:103A2000B093F9042091F6043091F7044091F80422
:103A30005091F90457FDB2C00AE055954795379566
:103A400027950A95D1F78091F6049091F704A091FB
:103A5000F804B091F904821B930BA40BB50B80936F
:103A6000F6049093F704A093F804B093F90483E06C
:103A70007CCC2093300480912703909128039C01F3
:103A8000220F331F280F391F809178009091790001
:103A900063E070E00E946C67260F371F369527950C
:103AA00036952795309328032093270385E05DCC36
:103AB00080934304A0923F04B0924004C09241041A
:103AC000D092420482E051CC80911D0490911E045A
:103AD0008F5F9F4F0CF07FCF80913405909135051B
:103AE000A0913605B091370520E030E849E054E474
:103AF000BC01CD010E94D46618160CF06CCF8091E9
:103B0000340590913505A0913605B09137052AE02E
:103B100037ED43EA5CE3BC01CD010E946766DC013E
:103B2000CB018093340590933505A0933605B0936F
:103B300037058091B3049091B404845F914008F0FC
:103B40004ACF8091340590913505A0913605B0910A
:103B500037052DEC3CEC4CEC5DE3BC01CD010E9443
:103B600067662FCF220F331FB9CD809178009091D7
:103B700079002091310430913204820F931F019615
:103B8000969587958ECE220F331FFACD0796FFCDDF
:103B9000D801C7010B96A11DB11DD7CC21503C4FB8
:103BA0004F4F5F4F49CF215F3F4F4F4F5F4F49CD41
:103BB000215F3F4F4F4F5F4FFECC0196A11DB11DBE
:103BC00067CD0F9655CD2F5F3F4F0FCE0196F1CDAC
:103BD00007968BCD2F5F3F4FB6CD019698CD809144
:103BE0007800909179002091310430913204820F55
:103BF000931F2FEF37E0281B390B309324042093B9
:103C0000230486E0B2CBFF91EF91BF91AF919F91DA
:103C10008F917F916F915F914F913F912F911F9164
:103C20000F91FF90EF90DF90CF90BF90AF900F90EB
:103C30000FBE0F901F90189590E2EAE2F3E08FE438
:103C40009193815087FFFCCF08951F93CF93DF930B
:103C50008091450420912903281710F420934504EE
:103C60009091440490FF08C080914504882309F492
:103C70001EC181508093450491FF08C08091450486
:103C8000821709F4E4C18F5F80934504892F992737
:103C900080FF02C081FD08C10E941C1E9091450456
:103CA0009A3008F0A2C081E180934604892F9927B9
:103CB0009F938F9381E493E09F938F9381E08F9301
:103CC0000E947E130F900F900F900F900F90809195
:103CD0004504C82FDD27C730D10509F4BBC1C83062
:103CE000D1050CF08CC0C330D10509F455C2C430E5
:103CF000D1050CF0DFC0C130D10509F4BBC2C23020
:103D0000D1050CF438C31092460481E094E09F93EF
:103D10008F93C1E0CF930E947E1384E18093460489
:103D20000F900F900F9080912E0590912F05A091EC
:103D30003005B0913105B7FD58C63AE0B595A79565
:103D4000979587953A95D1F7BF93AF939F938F93AC
:103D50008BE094E09F938F93CF930E947E1388E231
:103D6000809346048DB79EB707960FB6F8949EBF12
:103D70000FBE8DBF8091260590912705A091280543
:103D8000B0912905B7FD2CC62AE0B595A795979562
:103D900087952A95D1F7BF93AF939F938F938AE12D
:103DA00094E09F938F93CF930E947E138CE3809334
:103DB00046042DB73EB7295F3F4F0FB6F8943EBF7C
:103DC0000FBE2DBF8091F4049091F5049F938F93C3
:103DD00089E294E09F938F93CF930E947E130F907C
:103DE0000F900F900F900F90D6C780E180934604FC
:103DF000892F99279F938F9386E493E05DCFCB30F3
:103E0000D10509F45DC1CC30D1050CF00FC1C9302A
:103E1000D10509F40BC52A970CF01CC31092460477
:103E200080ED95E09F938F9311E01F930E947E1386
:103E300084E1809346040F900F900F908091F004DE
:103E40009091F1049F938F938FED95E09F938F93C3
:103E50001F930E947E1388E2809346040F900F9078
:103E60000F900F900F908091F4049091F5049F9320
:103E70008F938EEE95E09F938F931F930E947E13F6
:103E80008CE3809346040F900F900F900F900F904B
:103E90008091F2049091F3049F938F938DEF95E0BE
:103EA0009F938F931F9399CF10924504F5CE209343
:103EB0004504E2CEC530D10509F403C426970CF0C1
:103EC0008CC3109246048091E708E82FFF27EE0F7D
:103ED000FF1FEC54F74F808191819F938F938091C6
:103EE000E608E82FFF27EE0FFF1FEC54F74F808105
:103EF00091819F938F9388E794E09F938F9311E034
:103F00001F930E947E1384E1809346048DB79EB771
:103F100007960FB6F8949EBF0FBE8DBF8091E9083B
:103F2000E82FFF27EE0FFF1FEC54F74F80819181A0
:103F30009F938F938091E808E82FFF27EE0FFF1FD4
:103F4000EC54F74F8081918188589F4F9F938F93B6
:103F500088E894E09F938F931F930E947E1388E2DA
:103F6000809346042DB73EB7295F3F4F0FB6F894B4
:103F70003EBF0FBE2DBF8091EB08E82FFF27EE0F4D
:103F8000FF1FEC54F74F8081918182599F4F9F937F
:103F90008F938091EA08E82FFF27EE0FFF1FEC5464
:103FA000F74F8081918182599F4F9F938F9388E92A
:103FB00094E09F938F931F930E947E138CE38093D2
:103FC00046046DB77EB7695F7F4F0FB6F8947EBF2A
:103FD0000FBE6DBF8091ED08E82FFF27EE0FFF1F8A
:103FE000EC54F74F8081918182599F4F9F938F931B
:103FF0008091EC08E82FFF27EE0FFF1FEC54F74FDE
:104000008081918182599F4F9F938F9388EA94E09A
:104010009F938F931F930E947E138DB79EB7079631
:104020000FB6F8949EBF0FBE8DBFB5C6CD30D1057B
:1040300009F447C4CD30D1050CF452C22E9709F4CF
:10404000D9C481508093290310924504A4C61092CC
:1040500045041CCE84E1809346048091270390910F
:1040600028039F938F9382EA95E09F938F9311E0AB
:104070001F930E947E1388E2809346040F900F9056
:104080000F900F900F908091E30499279F938F9347
:1040900081EB95E09F938F931F930E947E138CE397
:1040A000809346040F900F900F900F900F90809187
:1040B000B308992701979F938F9380EC95E0F0CEFA
:1040C000109246048EE696E09F938F9311E01F9323
:1040D0000E947E1384E1809346040F900F900F900E
:1040E00080918907992787FD90959F938F93809161
:1040F0008807992787FD90959F938F938EE796E089
:104100009F938F931F930E947E1388E280934604AF
:104110008DB79EB707960FB6F8949EBF0FBE8DBFA2
:1041200080918A07992787FD90959F938F9380911F
:104130008B0799279F938F938EE896E09F938F9399
:104140001F930E947E138CE3809346042DB73EB7E5
:10415000295F3F4F0FB6F8943EBF0FBE2DBF809131
:104160008F0799279F938F9380918C07992787FDBD
:1041700090959F938F938EE996E09F938F931F93D3
:104180000E947E136DB77EB7695F7F4F0FB6F894BC
:104190007EBF0FBE6DBFFFC5109246048091B80868
:1041A0009091B9089F938F938091B6089091B7082A
:1041B0009F938F9388E394E09F938F9311E01F93D5
:1041C0000E947E1384E1809346046DB77EB7695FD9
:1041D0007F4F0FB6F8947EBF0FBE6DBF8091BC08B5
:1041E0009091BD089F938F938091BA089091BB08DE
:1041F0009F938F9388E494E09F938F931F930E94E3
:104200007E1388E2809346048DB79EB707960FB65B
:10421000F8949EBF0FBE8DBF8091C0089091C108D9
:104220009F938F938091BE089091BF089F938F9327
:1042300088E594E09F938F931F930E947E138CE3F5
:10424000809346042DB73EB7295F3F4F0FB6F894D1
:104250003EBF0FBE2DBF8091C4089091C5089F93AB
:104260008F938091C2089091C3089F938F9388E6A3
:1042700094E083CF8091EE0880FD1CC084E18093A0
:1042800046048CEE93E09F938F9311E01F930E945E
:104290007E1388E2809346040F900F900F9083EF77
:1042A00093E09F938F931F930E947E130F900F9024
:1042B0000F9071C5109246048091D5049091D60458
:1042C000A091D704B091D804BC01CD0125E030E025
:1042D00040E050E00E94B5673F932F9380EB93E05E
:1042E0009F938F9311E01F930E947E1384E180932C
:1042F00046040F900F900F900F900F908091D10473
:104300009091D204A091D304B091D404BC01CD010A
:1043100025E030E040E050E00E94B5673F932F93E6
:104320008FEB93E09F938F931F930E947E1388E2FD
:10433000809346040F900F900F900F900F908091F4
:104340001D0390911E039F938F938EEC93E09F9398
:104350008F931F930E947E138CE3809346040F90EB
:104360000F900F900F900F9087B599279F938F9381
:104370008DED93E095CD209709F063CE1092460421
:104380008BE493E09F938F9311E01F930E947E1321
:1043900084E1809346040F900F900F9087E690E0A1
:1043A0009F938F938CE490E09F938F93DF93CF93B1
:1043B000809102016AE00E946067892F99279F938C
:1043C0008F93809102010E94606799279F938F933A
:1043D0008BE593E09F938F931F930E947E1388E257
:1043E000809346042DB73EB7235F3F4F0FB6F89436
:1043F0003EBF0FBE2DBF89ED95E09F938F930E9426
:104400005F0599279F938F9380E793E09F938F9306
:104410001F930E947E138091AC039091AD036DB702
:104420007EB7695F7F4F0FB6F8947EBF0FBE6DBF3A
:10443000069708F488C490914B04992309F47DC42D
:104440008CE380934604892F99279F938F938BE861
:1044500093E026CD109246048CE396E09F938F93D1
:1044600011E01F930E947E1384E1809346040F9015
:104470000F900F908091920399279F938F9384E4DC
:1044800096E09F938F931F930E947E1388E2809300
:1044900046040F900F900F900F900F908091FD03A6
:1044A0009091FE039F938F9382E596E09F938F9365
:1044B0001F930E947E138CE3809346040F900F900D
:1044C0000F900F900F908091100999279F938F93D1
:1044D00080910F0999279F938F9380E696E04DCEA8
:1044E000109246048EEA96E09F938F9311E01F93FB
:1044F0000E947E1384E1809346040F900F900F90EA
:1045000080918E0899279F938F9380918D0899278A
:104510009F938F9380918C0899279F938F9380917D
:104520008B0899279F938F938EEB96E09F938F93A1
:104530001F930E947E1388E2809346048DB79EB736
:104540000B960FB6F8949EBF0FBE8DBF8091920858
:1045500099279F938F938091910899279F938F9389
:104560008091900899279F938F9380918F08992726
:104570009F938F9383ED96E09F938F931F930E9459
:104580007E138CE3809346042DB73EB7255F3F4FE3
:104590000FB6F8943EBF0FBE2DBF809196089927A5
:1045A0009F938F938091950899279F938F938091E4
:1045B000940899279F938F938091930899279F93AD
:1045C0008F9388EE96E09F938F931F930E947E13A4
:1045D0006DB77EB7655F7F4FD9CD1092460488E6F0
:1045E00095E09F938F9311E01F930E947E1384E1C7
:1045F000809346040F900F900F9080913C0590910E
:104600003D059F938F9380911F04909120049F9369
:104610008F9385E795E09F938F931F930E947E135E
:1046200088E2809346046DB77EB7695F7F4F0FB60F
:10463000F8947EBF0FBE6DBF80913A0590913B0507
:104640009F938F9380912104909122049F938F9345
:1046500084E895E09F938F931F930E947E138CE3D1
:10466000809346048DB79EB707960FB6F8949EBF09
:104670000FBE8DBF8091340590913505A091360510
:10468000B0913705BC01CD010E94AA66DC01CB01C7
:104690009F938F9380916709909168099F938F935F
:1046A00083E995E09F938F931F930E947E132DB70C
:1046B0003EB7295F3F4F0FB6F8943EBF0FBE2DBFE8
:1046C0006AC31092460488EB94E09F938F93C1E0F5
:1046D000CF930E947E13809102010F900F900F9054
:1046E0008A3009F4A5C28B3009F4DEC1843109F4A3
:1046F000DBC18D3009F04FC384E180934604809183
:104700001C0399279F938F9340914605509147052D
:10471000CA0157FD39C395958795959587959595C8
:104720008795959587959F938F939A0157FD29C3F8
:1047300035952795359527953595279580912704AB
:1047400090912804821B930B9F938F938CE295E0AA
:104750009F938F93CF930E947E1388E280934604A9
:104760006DB77EB7675F7F4F0FB6F8947EBF0FBE01
:104770006DBF80911B0399279F938F9340914405B0
:1047800050914505CA0157FD04C3959587959595A8
:10479000879595958795959587959F938F939A0182
:1047A00057FDF4C23595279535952795359527956D
:1047B0008091250490912604821B930B9F938F93E5
:1047C00080E495E09F938F93CF930E947E138CE3B8
:1047D000809346048DB79EB709960FB6F8949EBF96
:1047E0000FBE8DBF80911A0399279F938F932091BD
:1047F000420530914305C90137FDC1C295958795A2
:104800009F938F938091230490912404281B390B4C
:104810003F932F9384E595E09F938F93CF930E94CE
:104820007E132DB73EB7275F3F4F45CF109246040A
:104830008091EA049091EB049F938F938CE096E033
:104840009F938F9311E01F930E947E1384E18093C6
:1048500046040F900F900F900F900F908091E804F6
:104860009091E9049F938F9388E196E09F938F93B3
:104870001F930E947E1388E2809346040F900F904E
:104880000F900F900F908091E6049091E7049F9312
:104890008F9384E296E09F938F931F930E947E13E1
:1048A0008CE3809346040F900F900F900F900F9021
:1048B0008091E4049091E5049F938F9380E396E0C8
:1048C000EFCA109246048DEF96E09F938F93C1E05C
:1048D000CF930E947E1384E1809346040F900F9043
:1048E0000F908091AA0899278D969F938F9380911E
:1048F000A90899278D969F938F938091A80899274F
:104900008D969F938F938091A70899278D969F935B
:104910008F938CE097E09F938F93CF930E947E13A9
:1049200088E2809346048DB79EB70B960FB6F89435
:104930009EBF0FBE8DBF8091AE0899278D969F9325
:104940008F938091AD0899278D969F938F93809137
:10495000AC0899278D969F938F938091AB089927E8
:104960008D969F938F9380E297E09F938F93CF9341
:104970000E947E138CE3809346042DB73EB7255FDB
:104980003F4F0FB6F8943EBF0FBE2DBF8091AF08CA
:1049900099278D969F938F9384E397E09F938F93AE
:1049A000CF930E947E130F900F900F900F900F9057
:1049B0008091B008882309F02DC18091B108882327
:1049C00009F01AC18091B208882309F4E4C188E48F
:1049D000809346048AE497E09F938F93CF9364CCAF
:1049E00081509C4FAF4FBF4FCFC981509C4FAF4FAD
:1049F000BF4FA3C9109246048DE497E09F938F9315
:104A000011E01F930E947E1384E1809346040F906F
:104A10000F900F908091DE039091DF039F938F930F
:104A20008BE597E09F938F931F930E947E1388E2FC
:104A3000809346040F900F900F900F900F908091ED
:104A4000DC039091DD039F938F9388E697E09F931B
:104A50008F931F930E947E1389E4809346040F90E6
:104A60000F900F900F900F9085E797E09F938F9393
:104A70001F930E947E13809144040F900F900F901B
:104A800083FF89C11092DF031092DE03AEE0B0E035
:104A900080E0082E0E94DD67AFE0B0E08091DE0389
:104AA000082E0E94DD6777C184E18093460440911F
:104AB000460550914705CA0157FD57C19C013595E0
:104AC0002795359527953595279535952795C901CE
:104AD00082959295907F9827807F9827BA01681BCE
:104AE000790BCB0177FD3FC1959587959F938F9368
:104AF0003F932F939A0157FD33C1359527953595EF
:104B00002795359527958091270490912804821B3D
:104B1000930B9F938F9389EF94E09F938F93CF9301
:104B20000E947E1388E2809346048DB79EB7099653
:104B30000FB6F8949EBF0FBE8DBF409144055091B3
:104B40004505CA0157FD0AC19C0135952795359544
:104B500027953595279535952795C9018295929585
:104B6000907F9827807F9827BA01681B790BCB012B
:104B700077FDF2C0959587959F938F933F932F93E1
:104B80009A0157FDE6C035952795359527953595BA
:104B900027958091250490912604821B930B9F9367
:104BA0008F938BE095E09F938F93CF930E947E131A
:104BB0008CE3809346048DB79EB709960FB6F894A0
:104BC0009EBF0FBE8DBF2091420530914305C901A4
:104BD00037FDCDC0959587959F938F938091230442
:104BE00090912404281B390B3F932F938DE195E07E
:104BF0009F938F93CF9359CD84E48093460487E4A9
:104C000097E09F938F93CF930E947E130F900F9006
:104C10000F90D8CE80E48093460484E497E09F937D
:104C20008F93CF930E947E130F900F900F90C5CE5D
:104C300084E18093460440914605509147059A01CE
:104C400057FD9AC035952795359527953595279524
:104C5000C901880F991F880F991F880F991F481B3A
:104C6000590B5F934F933F932F938091270490911B
:104C70002804821B930B9F938F9386EC94E09F9361
:104C80008F93CF930E947E1388E2809346042DB7C2
:104C90003EB7275F3F4F0FB6F8943EBF0FBE2DBF04
:104CA00040914405509145059A0157FD62C03595E4
:104CB00027953595279535952795C901880F991F13
:104CC000880F991F880F991F481B590B5F934F93AB
:104CD0003F932F938091250490912604821B930B80
:104CE0009F938F9388ED94E09F938F93CF930E942F
:104CF0007E138CE3809346046DB77EB7675F7F4F6A
:104D00000FB6F8947EBF0FBE6DBF809142059091A3
:104D100043059F938F938091420590914305209185
:104D2000230430912404821B930B9F938F938AEE6C
:104D300094E09F938F93CF936EC98CE38093460446
:104D400080EA93E0AECA8CE3809346048EE793E05A
:104D5000A8CA295F3F4F17CF01960CCF0F96F4CE0C
:104D6000295F3F4FCACE0196BFCE0F96A7CE0196C0
:104D700031CF295F3F4F9BCF295F3F4F63CF0196D4
:104D80003DCD295F3F4FD4CC0F96C5CC295F3F4F17
:104D900009CD0F96FACC10924404DF91CF911F9168
:104DA00008951092B9008AE28093B800089585EAC8
:104DB0008093BC00089584E98093BC00089510920C
:104DC000B9008093BB0085E88093BC0008950E94E1
:104DD000DB2610924E048091BB0010924D0480E8B7
:104DE0008093BC001092BD001092BA001092BB00DC
:104DF0001092B9001092B8000E94D1260E94D726C6
:104E000080E00E94DF2608958093BB0085E88093B0
:104E1000BC00089585EC8093BC00089585E88093DC
:104E2000BC0008953FEF20E0261730F4FC0181918B
:104E300038272F5F2617D8F3832F992708951F92BD
:104E40000F920FB60F9211242F933F934F935F93BE
:104E50006F937F938F939F93AF93BF93EF93FF9342
:104E600080914E04282F33278F5F80934E042E307D
:104E7000310509F448C02F3031059CF42A30310542
:104E800009F443C02B3031054CF528303105C9F108
:104E9000293031050CF047C0232BA9F010924E04A5
:104EA00049C02231310569F1233131050CF124313A
:104EB0003105E9F124313105C4F125313105A1F085
:104EC0002631310559F70E94DB268AE090E0909365
:104ED000AD038093AC0310924E042CC02C303105EE
:104EE000B9F02D3031056CF480E80E94DF2622C035
:104EF00020313105C9F32131310554F480911B0370
:104F0000F4CF88E9F2CF82E1F0CF80911C03EDCF9E
:104F10000E94DB268AE090E09093AD038093AC037F
:104F20000E94D72607C080E1E0CF84E1DECF8091E8
:104F30001A03DBCF8091BC0080688093BC00FF9196
:104F4000EF91BF91AF919F918F917F916F915F9101
:104F50004F913F912F910F900FBE0F901F9018957A
:104F600083EC8093810080916F00806280936F005A
:104F70001092430510924205109245051092440587
:104F8000109247051092460508951F920F920FB692
:104F90000F921124EF92FF920F931F932F933F9341
:104FA0004F935F936F937F938F939F93AF93BF9331
:104FB000CF93DF93EF93FF9380913E0982FD2CC046
:104FC0002091860030918700809151049091520485
:104FD000281B390B80918600909187009093520492
:104FE00080935104C9018D549440835F9A4108F025
:104FF000B5C0809153048093B3088091530490917D
:105000005404049714F010928403C1E0D0E0D093CC
:105010005404C093530415C24091860050918700F8
:105020008091550490915604481B590B809186003D
:10503000909187009093560480935504CA018D5433
:105040009440835F9A4138F58091AF048093500477
:1050500080915004843008F00EC18091B0048536F0
:1050600008F47BC18AE08093B004809102018A3009
:1050700009F476C1843109F473C1289881E08093E2
:10508000AF048091D904882309F0DBC180915004DA
:105090008093B308D6C10091AF040A3008F0E4C091
:1050A000CA018B5F9040845B914008F05BC1425D18
:1050B0005140E02FFF27EE0FFF1FE95AFB4F808181
:1050C0009181FA01E81BF90BCF0105960B9708F4C3
:1050D0005CC1E02FFF27EE0FFF1FE95AFB4F8081D5
:1050E00091819C01220F331F280F391F240F351F78
:1050F00037FDA4C1E901D595C795D595C795CA01D6
:1051000001968C179D070CF071C121978091E304E3
:105110008E3B08F462C1E02FFF27EE0FFF1FDF0177
:10512000A95ABB4F8D919C919E01281B390BC90137
:1051300063E070E00E948067CB01880F991F860FA3
:10514000971FE359FB4F91838083E02FFF27EE0FDA
:10515000FF1FE95AFB4FD183C0830BC1C091530499
:10516000D0915404CA30D1050CF06BC1C9018B5FDA
:105170009040845B914008F060C0225D3140FE01A8
:10518000EC0FFD1FEC54F74F80819181D901A81BD2
:10519000B90BCD01B7FD0EC1069754F48091E3041D
:1051A000883C08F046C18091E304865F8093E30465
:1051B000FE01EC0FFD1FEC54F74F80819181AC0193
:1051C000440F551F480F591F420F531F57FD33C13E
:1051D0007A01F594E794F594E794C90101968E1548
:1051E0009F050CF013C10894E108F1088091E304D5
:1051F000833C08F403C18E010C0F1D1FF801EC5411
:10520000F74F80819181F701E81BF90BCF0163E033
:1052100070E00E948067CB01880F991F860F971F4F
:105220000653174FD80111969C938E93FE01EC0FF5
:10523000FD1FEC54F74FF182E082FE013196F093AE
:105240005404E0935304E530F10509F4B9C05D98C6
:10525000E630F10509F4BFC05C98379709F4B9C08E
:105260005B98EFC05C9A5B98043108F054C00F5F04
:105270000093AF04E6C09091B30880915004981752
:1052800009F0EBCE4091B0044B3008F49BC0109273
:1052900084031092AF043AC00091AF04E02FFF27BF
:1052A000EE0FFF1F9F012D573B4FDF01AC54B74F4F
:1052B0008D919C91D9018D939C93DF01A653B74F9B
:1052C0008D919C91E756FB4F91838083E02FFF27C0
:1052D000EE0FFF1F9F012C54374FDF01A95ABB4F20
:1052E0008D919C91D90111969C938E93DF01A359C6
:1052F000BB4F8D919C91E653F74F91838083E02FB4
:10530000EF5FEB3008F05EC0E093AF044F3120F662
:105310000091AF04DBCF043109F093C0809102010A
:105320008A3009F47DC0843109F47AC028988EE16E
:105330008093AF042AE0CAECD8E0A3E8B4E0E4EB41
:10534000F8E08D919D919183808332961982188225
:105350002296215027FFF5CF74C01092B00485CE5D
:10536000289A8CCE809102018A3011F1843101F1AA
:105370002898053019F15D98063009F473CF5C98D0
:10538000073009F070CF5B9A72CF8091B0048A31F8
:1053900008F448C08091E304865F8093E304809121
:1053A000E304893C08F495CE88EC8093E30491CE25
:1053B000289ADFCF909581959F4FEECE5D9ADFCFF3
:1053C0005D9A46CF4F3F09F459CE4F5F4093B004EA
:1053D00055CE5B9A36C05C9A40CFE02FFF27EE0F88
:1053E000FF1FE359FB4F11821082AFCE4150504056
:1053F000C417D5070CF08ACE219688CEFE01EC0F9B
:10540000FD1FE653F74F1182108210CF215030401C
:10541000E216F3060CF0EACE0894E11CF11CE6CE8D
:10542000289A85CF8B3008F4BACF8091E3048E5F41
:10543000B4CF88ECBBCE4D5F5F4FCACE2D5F3F4FE0
:1054400059CEFF91EF91DF91CF91BF91AF919F9195
:105450008F917F916F915F914F913F912F911F910C
:105460000F91FF90EF900F900FBE0F901F90189527
:1054700081E08093E80882E08093E70883E08093EE
:10548000E60884E08093E90885E08093EA0886E0F6
:105490008093EB0887E08093EC0888E08093ED0828
:1054A00008951F938AE68093EE0851E050933E09D9
:1054B0004EE14093EF088BEF8093F1088AE08093F0
:1054C000F2084093F0084093F40885E08093F508D3
:1054D00080E48093F6081092F70884E18093F30843
:1054E0008EE08093F808E0E1E093F9081CE0109367
:1054F000FA08F8E0F093FB0886EE8093FC084093EE
:10550000FD0880E88093FE0830E53093FF0896E9B7
:105510009093000983E080930109309302099093EE
:10552000030981E28093040983E280930509409393
:1055300006091092070960E26093080910920909B0
:1055400010920A0910920B0910920C09109221096D
:1055500010922209109223091092240924E6209324
:105560000D0998E290930E0950933D0910920F098E
:105570008AEF8093100976E0709315092093110942
:1055800090931209109213098093140982E3809377
:1055900016099AE5909317098093180910923C090F
:1055A0009093190930931A0950931B0985E580934C
:1055B0001C0980931D09E0931E0960931F09209325
:1055C00020098FE58093250983EF809327098AEAD4
:1055D0008093290980932A098FE08093260980937C
:1055E00028098CEF80932B0920932C0990932D0987
:1055F00090932E0990932F098BE480933009809328
:105600003109809332091092330970933409F09371
:105610003509909336094093370920933809209330
:10562000390984E080933A09AEEAB3E0EFE3F9E0A8
:105630000D9001921A95E1F71F9108958AE68093E3
:10564000EE0871E070933E095EE15093EF088BEF36
:105650008093F1089AE09093F2085093F0085093E9
:10566000F40885E08093F50880E48093F6081092B2
:10567000F7088FE08093F3089093F80880E1809317
:10568000F90866E06093FA08E8E0E093FB0886EE2C
:105690008093FC085093FD0880E88093FE082AE57B
:1056A0002093FF0898E79093000983E08093010915
:1056B000209302099093030981E28093040983E215
:1056C00080930509509306091092070940E2409320
:1056D00008091092090910920A0910920B091092F8
:1056E0000C0910922109109222091092230910929C
:1056F000240934E630930D0998E290930E097093D3
:105700003D0910920F098AEF8093100960931509E3
:105710003093110990931209109213098093140980
:1057200082E3809316092093170980931809109239
:105730003C092093190980E580931A098CE3809332
:105740001B0985E580931C0980931D0940931E0960
:1057500040931F099BE4909320098FE580932509CE
:1057600083EF809327098AEA8093290980932A0985
:1057700084E180932609809328098CEF80932B097C
:1057800030932C0920932D0920932E0920932F0963
:105790009093300990933109909332091092330914
:1057A00060933409E0933509209336095093370903
:1057B000309338093093390984E080933A098CE0BA
:1057C000A5EBB3E0EFE3F9E00D9001928A95E1F7E4
:1057D00008958AE68093EE0871E070933E094EE1E9
:1057E0004093EF088BEF8093F1088AE08093F208F2
:1057F0004093F0084093F40885E08093F50880E436
:105800008093F6081092F7088FE08093F30868E021
:105810006093F80820E12093F90856E05093FA08C5
:105820006093FB0886EE8093FC084093FD0880E8B7
:105830008093FE0834E63093FF0898E790930009C0
:1058400083E080930109309302099093030981E278
:105850008093040983E28093050984E1809306091B
:1058600010920709209308091092090910920A0959
:1058700010920B0910920C09109221091092220922
:10588000109223091092240930930D0998E2909305
:105890000E0970933D0910920F098AEF8093100949
:1058A000509315093093110990931209109213091E
:1058B0008093140992E3909316092AE5209317091F
:1058C0009093180910923C092093190980E5809360
:1058D0001A0986E480931B0985E580931C0980934F
:1058E0001D0980E280931E0980931F09909320096F
:1058F0008FE58093250983EF809327098AEA8093B7
:10590000290980932A0940932609409328098CEF9E
:1059100080932B0930932C0920932D0920932E0975
:1059200020932F098BE48093300980933109809371
:10593000320910923309509334096093350920934A
:10594000360940933709309338093093390984E098
:1059500080933A098CE0ADEBB3E0EFE3F9E00D9012
:1059600001928A95E1F708956817790744F4680F62
:10597000791F77FD09C0CB01959587950895681B20
:10598000790B861B970B08956F5F7F4FCB01959521
:1059900087950895EF92FF920F931F93CF93C82F8F
:1059A0008B018091D9048823A9F4C150CF3F91F095
:1059B0007B01E60EF71E1093010400930004809112
:1059C000000490910104892BD1F7C7010E9412179E
:1059D000C15088F7CF911F910F91FF90EF900895DC
:1059E0002F923F924F925F926F927F928F929F92EF
:1059F000AF92BF92CF92DF92EF92FF920F931F93DD
:105A0000CF93DF93CDB7DEB7ED970FB6F894DEBF37
:105A10000FBECDBF209142053091430580912304F4
:105A200090912404281B390B3A8729873093AA09BF
:105A30002093A90920912D0430912E0437FDD4C75D
:105A40003595279535952795359527953AA729A713
:105A50003C872B87790120912B0430912C0437FD52
:105A6000C0C73595279535952795359527953CA73A
:105A70002BA73E872D87F0926A09E092690930933F
:105A8000600920935F098091980990919909AA274C
:105A900097FDA095BA2F7C018D01EE0CFF1C001F15
:105AA000111FE80EF91E0A1F1B1F80911F04909101
:105AB00020049C01442737FD4095542FDA01C90189
:105AC000880F991FAA1FBB1F880F991FAA1FBB1FF2
:105AD000820F931FA41FB51F820F931FA41FB51F12
:105AE000E80EF91E0A1F1B1F17FD9CC71595079589
:105AF000F794E79415950795F794E794F092990930
:105B0000E09298098091B4099091B509AA2797FD70
:105B1000A095BA2F7C018D01EE0CFF1C001F111FF8
:105B2000E80EF91E0A1F1B1F809121049091220488
:105B30009C01442737FD4095542FDA01C901880F95
:105B4000991FAA1FBB1F880F991FAA1FBB1F820F77
:105B5000931FA41FB51F820F931FA41FB51FE80E2C
:105B6000F91E0A1F1B1F17FD54C715950795F794BB
:105B7000E79415950795F794E794F092B509E092AC
:105B8000B4098091670990916809AA2797FDA095AB
:105B9000BA2F9C01AD01220F331F441F551F280F40
:105BA000391F4A1F5B1F80911D0490911E04AA2774
:105BB00097FDA095BA2F280F391F4A1F5B1F57FD6D
:105BC00016C7559547953795279555954795379518
:105BD0002795309368092093670920911F0430911D
:105BE0002004C901880F991F880F991F820F931FE6
:105BF000820F931FAA2797FDA095BA2F20911E050B
:105C000030911F054091200550912105820F931F6F
:105C1000A41FB51F80931E0590931F05A093200518
:105C2000B09321052091210430912204C901880FED
:105C3000991F880F991F820F931F820F931FAA2706
:105C400097FDA095BA2F20911A0530911B05409120
:105C50001C0550911D05820F931FA41FB51F809333
:105C60001A0590931B05A0931C05B0931D05809108
:105C700072099091730920911F0430912004820FC2
:105C8000931F90937309809372098091AC0990914E
:105C9000AD092091210430912204820F931F90932B
:105CA000AD098093AC098091380590913905019632
:105CB00090933905809338058091160590911705CA
:105CC000A0911805B0911905BC01CD010E94C766CD
:105CD0005B016C0180916E0890916F08AA2797FD77
:105CE000A095BA2FBC01CD010E94C7667B018C0133
:105CF0008091340590913505A0913605B091370516
:105D00009C01AD01C801B7010E946766DC01CB01AF
:105D10009C01AD01C601B5010E946866DC01CB01A2
:105D2000BC01CD010E94AA66DC01CB01809316055F
:105D300090931705A0931805B09319058FEC8093E5
:105D40007A001092190320900605309007054090C4
:105D500008055090090539E423163BE6330631E087
:105D6000430630E053060CF414C188E49BE6A1E03E
:105D7000B0E08D839E83AF83B88760900E057090EE
:105D80000F05809010059090110539E463163BE6ED
:105D9000730631E0830630E093060CF4DCC488E43B
:105DA0009BE6A1E0B0E089839A83AB83BC834985FD
:105DB0005A85CA01AA2797FDA095BA2F2091FE0403
:105DC0003091FF044091000550910105280F391FC3
:105DD0004A1F5B1F2DA33EA34FA358A7A090B00955
:105DE000B090B109C090B209D090B309A80EB91E05
:105DF000CA1EDB1E860175013091CC043BA3332300
:105E000009F0DAC08091CB04882309F0C2C4409124
:105E1000EE084CA346FF13C6EBA5FCA5CF01AA27AD
:105E200097FDA095BA2FBC01CD0129813A814B8104
:105E30005C810E9441679B01AC0197FD2CC7BBE0D0
:105E40005595479537952795BA95D1F780918E034B
:105E5000E82EFF2400271127C801B7010E944167DF
:105E600097FD14C7ACE09595879577956795AA95AA
:105E7000D1F76F87788B898B9A8B609352057093DB
:105E80005305809354059093550529A53AA5C9015A
:105E9000AA2797FDA095BA2FBC01CD012D813E8187
:105EA0004F8158850E9441679B01AC0197FD01C756
:105EB000FBE05595479537952795FA95D1F7C80199
:105EC000B7010E94416797FDEFC6DC01CB01ECE012
:105ED000B595A79597958795EA95D1F7809356053F
:105EE00090935705A0935805B093590520915205FA
:105EF000309153053093E1082093E0082091560536
:105F0000309157053093E5082093E4082F853889B0
:105F100049895A89821B930BA40BB50B8AAF9BAF9F
:105F2000ACAFBDAF8093560590935705A09358052D
:105F3000B0935905A80EB91ECA1EDB1E8601750155
:105F400030918D033DA7332309F0A3C58EA79FA7EA
:105F5000A8ABB9ABB7FD61C62EA53FA548A959A905
:105F600055954795379527958DA19EA1AFA1B8A5C9
:105F7000821B930BA40BB50B8DA39EA3AFA3B8A755
:105F80008093FE049093FF04A0930005B093010555
:105F90008CC598EB291694E939069EEF49069FEFC8
:105FA00059060CF0F1C328EB34E94EEF5FEF2D8377
:105FB0003E834F835887E1CE2DA13EA14FA158A526
:105FC0002093FE043093FF04409300055093010595
:105FD0003091EE083CA31092E5081092E40810926C
:105FE000E1081092E00810924E0510924F051092B1
:105FF00050051092510510924A0510924B051092CF
:106000004C0510924D0530918D033DA780914E05B2
:1060100090914F05A0915005B0915105BC01CD0163
:1060200024E630E040E050E00E94B567DA01C901A3
:1060300040914A0550914B05481B590B58A34F8F6F
:1060400080914A0590914B05A0914C05B0914D056A
:10605000BC01CD0124E630E040E050E00E94B5678D
:10606000DA01C90120914E0530914F05821B930B37
:106070009AA389A38091860390918703A0918803B6
:10608000B0918903BC01CD0128E631E040E050E049
:106090000E944167E616F7060807190744F0570102
:1060A0006801A61AB70AC80AD90A8601750117FD40
:1060B000A3C4A092B009B092B109C092B209D09223
:1060C000B3092BA53CA58F8D98A1280F391F790105
:1060D0000027F7FC0095102F809102059091030591
:1060E000A0910405B0910505E80EF91E0A1F1B1FBB
:1060F000570168018091CF049091D004281B390B7F
:10610000C901AA2797FDA095BA2F280E391E4A1E4D
:106110005B1E2091A2033091A3034091A4035091F0
:10612000A503221533054405550574F4A8EAEA2EA3
:10613000A1E6FA2E012D112DE21AF30A040B150B1C
:10614000170128015701680188279927DC01821B64
:10615000930BA40BB50B281639064A065B060CF008
:10616000E9C2F8E52F2EFEE93F2EFFEF4F2EFFEF9D
:106170005F2E220E331E441E551E209206053092BD
:10618000070540920805509209058201710120928D
:10619000020530920305409204055092050529A599
:1061A0003AA5A9A1BAA12A0F3B1FA901662757FD4D
:1061B0006095762F80910A0590910B05A0910C05B2
:1061C000B0910D05480F591F6A1F7B1F5A016B01C3
:1061D0008091CD049091CE04281B390BC901AA27C8
:1061E00097FDA095BA2F680E791E8A1E9B1E80917E
:1061F000A6039091A703A091A803B091A9038EAB29
:106200009FABA8AFB9AF86159705A805B90564F48B
:1062100048EA51E660E070E0481B590B6A0B7B0BC3
:106220003A014B015A016B018EA99FA9A8ADB9ADE6
:10623000B095A095909581959F4FAF4FBF4F681631
:1062400079068A069B060CF064C2E8E56E2EEEE93C
:106250007E2EEFEF8E2EEFEF9E2E2EA93FA948AD9A
:1062600059AD620E731E841E951E60920E057092CB
:106270000F058092100590921105B401A301609260
:106280000A0570920B0580920C0590920D058DA168
:106290009EA1AFA1B8A58093120590931305A0937A
:1062A0001405B093150560922E0570922F0580920B
:1062B00030059092310520922605309227054092B4
:1062C00028055092290540932A0550932B05609389
:1062D0002C0570932D05E0922205F0922305009382
:1062E000240510932505809125039091260397FDA1
:1062F000A4C37C01F594E794F594E794F594E794AE
:10630000FAA6E9A6809123039091240397FD93C3F5
:106310008C011595079515950795159507951CA75B
:106320000BA780912704909128040F9734F458E12B
:10633000E52E5CEFF52EFAA6E9A680912704909150
:106340002804079734F440E3E42E48EFF42EFAA62D
:10635000E9A6209102012A3009F46BC2809127043A
:1063600090912804815D97400CF007C2809127042A
:1063700090912804805E974034F080EDE82E87E00D
:10638000F82EFAA6E9A680912504909126040F978D
:1063900024F408E11CEF1CA70BA780912504909121
:1063A0002604079724F400E318EF1CA70BA72A3054
:1063B00009F455C28091250490912604815D97408F
:1063C00024F008EE13E01CA70BA780912504909100
:1063D0002604805E974024F000ED17E01CA70BA771
:1063E000A0919903AA2309F497C0609125037091A5
:1063F000260380915A0590915B05681B790B2091CB
:10640000250330912603280F391F37FD3FC33595EB
:10641000279530935B0520935A05613871050CF47C
:106420003AC260E870E070936105609360058A2F5E
:106430009927869FF001879FF00D969FF00D1124FC
:10644000CF01F7FD21C37C01F594E794F594E7941F
:10645000F594E794F594E79429A53AA5E20EF31E86
:10646000FAA6E9A6409123035091240380915C058C
:1064700090915D05481B590B209123033091240313
:10648000280F391F37FDFDC23595279530935D05DF
:1064900020935C05413851050CF4F5C140E850E00B
:1064A00050935F0540935E058A2F9927849FD00102
:1064B000859FB00D949FB00D1124AD019D01B7FDD6
:1064C000DDC28901159507951595079515950795D1
:1064D00015950795EBA5FCA50E0F1F1F1CA70BA775
:1064E000869F9001879F300D969F300D1124C90122
:1064F0002091250330912603820F931F909326034A
:10650000809325038091230390912403480F591F02
:1065100050932403409323034D855E85141615067E
:106520000CF0C1C18091E0089091E10897FDA2C2F2
:10653000AA2797FDA095BA2F6DA5262F33274427AC
:106540005527BC01CD010E94416797FD8EC2E6E050
:106550009595879577956795EA95D1F7AF8DB8A111
:10656000A60FB71FB0935B09A0935A094B855C85B2
:10657000141615060CF0C1C18091E4089091E5084D
:1065800097FD6FC2AA2797FDA095BA2F6DA5262F5C
:10659000332744275527BC01CD010E94416797FD51
:1065A0005BC246E095958795779567954A95D1F7B3
:1065B000A9A1BAA1A60FB71FB0935009A0934F0984
:1065C0003CA137FDC1C110934E0900934D09F092D3
:1065D0005D09E0925C098091EA08E82FFF27EE0F41
:1065E000FF1FEC54F74F8081918182599F4FA091FA
:1065F000EA04B091EB04A817B9070CF0EEC0CD0186
:1066000001969093EB048093EA04DC018091EB08FF
:10661000E82FFF27EE0FFF1FEC54F74F8081918189
:1066200082599F4F6091E8047091E90468177907D7
:106630000CF0C4C0CB0101969093E9048093E80468
:10664000BC018091EC08E82FFF27EE0FFF1FEC54F0
:10665000F74F8081918182599F4F4091E60450917C
:10666000E704481759070CF0D5C0CA01019690936A
:10667000E7048093E604AC018091ED08E82FFF2742
:10668000EE0FFF1FEC54F74F8081918182599F4F8D
:106690002091E4043091E504281739070CF0ABC0D1
:1066A000C90101969093E5048093E4049C01B7FD31
:1066B00093C1AF3FB10539F034F08FEF90E0909384
:1066C000EB048093EA0477FD76C16F3F710539F0E2
:1066D00034F08FEF90E09093E9048093E80457FD45
:1066E00070C14F3F510539F034F08FEF90E0909337
:1066F000E7048093E60437FD6AC12F3F310509F0B6
:106700000CF4EEC28FEF90E09093E5048093E404E4
:10671000E7C260920E0570920F058092100590926C
:106720001105A0920A05B0920B05C0920C05D092FB
:106730000D05ADCD20920605309207054092080563
:1067400050920905A0920205B0920305C09204057B
:10675000D092050524CD98EB691694E979069EEF51
:1067600089069FEF99062CF528EB34E94EEF5FEF91
:1067700029833A834B835C831ACB98EEE92E93E00E
:10678000F92EFAA6E9A6F2CD2D823E824F825886D6
:10679000F4CA8DA19EA1AFA1B8A58093FE049093E9
:1067A000FF04A0930005B09301059091EE089CA30F
:1067B00012CC69827A828B829C82F9CA8081918113
:1067C00082599F4F861797070CF03BCF61157105D3
:1067D00009F437CFCB0101972FCF80819181825966
:1067E0009F4F8A179B070CF011CF109709F40ECF1B
:1067F000CD01019706CF8081918182599F4F8217E9
:1068000093070CF054CF2115310509F450CFC9017D
:10681000019748CF8081918182599F4F84179507B6
:106820000CF02ACF4115510509F426CFCA01019772
:106830001ECF8091270490912804835F934034F009
:1068400038EEE32E33E0F32EFAA6E9A68091270472
:10685000909128048A5F93400CF495CD8ECD809161
:10686000250490912604835F934024F008EE13E002
:106870001CA70BA780912504909126048A5F934062
:106880000CF4AECDA9CD3FEF403853070CF008CE45
:1068900040E85FEF05CE8FEF603878070CF0C3CD8E
:1068A00060E87FEFC0CD8091E0089091E10897FD0E
:1068B0009BC1AA2797FDA095BA2FEDA52E2F3327B0
:1068C00044275527BC01CD010E94416797FDADC10A
:1068D00056E095958795779567955A95D1F72F8DC1
:1068E00038A1261B370B30935B0920935A094B853F
:1068F0005C85141615060CF43FCE8091E408909147
:10690000E50897FD6DC1AA2797FDA095BA2FEDA5C3
:106910002E2F332744275527BC01CD010E94416704
:1069200097FD88C136E095958795779567953A9557
:10693000D1F729A13AA1261B370B30935009209398
:106940004F093CA137FF3FCE4BA1442309F03BCE7A
:106950008091CB04882309F036CE8B859C85A1E0FD
:1069600081309A070CF044C12B853C854FEF2030D5
:1069700034070CF0A3C189A59AA5280F391F3C87BD
:106980002B8720503F4F30935D0920935C09AD85E4
:10699000BE85E1E0A130BE070CF465C12BA53CA586
:1069A000A20FB31FBE87AD87A050B140B0934E0970
:1069B000A0934D0910CE1092E9041092E80457FFFD
:1069C00090CE1092E7041092E60437FF96CE109214
:1069D000E5041092E40484C11092EB041092EA04DE
:1069E00072CE295F3F4F3DC8295F3F4F29C82D5FB9
:1069F0003F4F4F4F5F4FE5C8E60EF71E081F191FA8
:106A0000E092B009F092B1090093B2091093B30972
:106A100058CB23E030E040E050E0E20EF31E041FCC
:106A2000151FA3C883E090E0A0E0B0E0E80EF91ED7
:106A30000A1F1B1F5BC807966BCC07965ACC2DA16B
:106A40003EA14FA158A52093FE043093FF0440932C
:106A5000000550930105BFCA615C7F4F8F4F9F4F68
:106A6000A0CD909581959F4F8DCD615C7F4F8F4FCD
:106A70009F4F6DCD909581959F4F5ACD215F3F4F90
:106A800020CD2F5F3F4F00CD0F96DDCC2F5F3F4FC6
:106A9000BECC2DA13EA14FA158A52093FE0430935A
:106AA000FF04409300055093010589859A85AA2724
:106AB00097FDA095BA2F2AAD3BAD4CAD5DAD820FD1
:106AC000931FA41FB51F8B8B9C8BAD8BBE8BBC0102
:106AD000CD0129813A814B815C810E9441679B01F4
:106AE000AC0197FDBBC06BE0559547953795279551
:106AF0006A95D1F760918F03862F9927AA27BB2724
:106B00008F8B988FA98FBA8FBC01CD010E944167EE
:106B100097FD9FC02CE095958795779567952A9569
:106B2000D1F76B8F7C8F8D8F9E8F60934A0570930A
:106B30004B0580934C0590934D056B897C898D891D
:106B40009E892D813E814F8158850E9441679B011E
:106B5000AC0197FD79C08BE0559547953795279502
:106B60008A95D1F76F89788D898D9A8D0E944167BA
:106B700097FD65C0BCE09595879577956795BA9523
:106B8000D1F76AAB7BAB8CAB9DAB60934E0570933A
:106B90004F05809350059093510529853A8537FD1F
:106BA0007FC0213431050CF431CA6B8D7C8D8D8D05
:106BB0009E8D97FD2AC0613871058105910564F4A9
:106BC0006AA97BA98CA99DA997FD82C0613871052E
:106BD000810591050CF41ACA81E08093EE0416CA6F
:106BE000909581959F4F8FCE909581959F4F61CEC7
:106BF000E9A5FAA58E0F9F1F9C878B878050914037
:106C000090935D0980935C09C2CE909580957095B4
:106C100061957F4F8F4F9F4FCECF0196A11DB11D24
:106C20008EA79FA7A8ABB9AB97C9615C7F4F8F4F69
:106C30009F4F4ECE615C7F4F8F4F9F4F73CE615001
:106C4000704F8F4F9F4F96CF2150384F4F4F5F4F10
:106C500082CF6150704F8F4F9F4F5CCF2150384F84
:106C60004F4F5F4F40CF4D855E856FEF40305607E9
:106C700054F58BA59CA5480F591F5E874D87405042
:106C80005F4F50934E0940934D09A5CC6150704F12
:106C90008F4F9F4FE7C82150384F4F4F5F4FCFC89E
:106CA000309521953F4F7DCF6150704F8F4F9F4F53
:106CB0000CC92150384F4F4F5F4FFAC8F0925D0911
:106CC000E0925C0964CE10934E0900934D0983CC89
:106CD00090958095709561957F4F8F4F9F4F76CFA0
:106CE000ED960FB6F894DEBF0FBECDBFDF91CF910A
:106CF0001F910F91FF90EF90DF90CF90BF90AF90DA
:106D00009F908F907F906F905F904F903F902F90CB
:106D10000895809102018D3009F455C110927A00D6
:106D2000809127049091280490935D0980935C09D9
:106D3000809125049091260490934E0980934D09EB
:106D400080912304909124049093AA098093A90927
:106D500080911F04909120049C01442737FD4095A9
:106D6000542FDA01C901880F991FAA1FBB1F880F72
:106D7000991FAA1FBB1F820F931FA41FB51F820F4D
:106D8000931FA41FB51F9093990980939809809130
:106D90002104909122049C01442737FD4095542FF3
:106DA000DA01C901880F991FAA1FBB1F880F991FFD
:106DB000AA1FBB1F820F931FA41FB51F820F931F13
:106DC000A41FB51F9093B5098093B40980911D0449
:106DD00090911E0490936809809367098FEC8093CB
:106DE0007A008091EA08E82FFF27EE0FFF1FEC548E
:106DF000F74F8081918182599F4FA091EA04B09111
:106E0000EB04A817B9070CF085C0CD01019690934B
:106E1000EB048093EA04DC018091EB08E82FFF2764
:106E2000EE0FFF1FEC54F74F8081918182599F4FE5
:106E30006091E8047091E904681779070CF096C036
:106E4000CB0101969093E9048093E804BC01809102
:106E5000EC08E82FFF27EE0FFF1FEC54F74F80815F
:106E6000918182599F4F4091E6045091E704481761
:106E700059070CF06CC0CA0101969093E704809307
:106E8000E604AC018091ED08E82FFF27EE0FFF1F0D
:106E9000EC54F74F8081918182599F4F2091E404F7
:106EA0003091E504281739070CF042C0C90101965A
:106EB0009093E5048093E4049C01B7FD7FC0AF3F4D
:106EC000B10511F00CF061C077FD67C06F3F71052F
:106ED00039F034F08FEF90E09093E9048093E80468
:106EE00057FD61C04F3F510539F034F08FEF90E00E
:106EF0009093E7048093E60437FD5BC02F3F310594
:106F000009F00CF463C08FEF90E09093E504809358
:106F1000E4045CC08081918182599F4F8A179B074E
:106F20000CF07ACF109709F477CFCD0101976FCF8E
:106F30008081918182599F4F821793070CF0BDCFBA
:106F40002115310509F4B9CFC9010197B1CF80816D
:106F5000918182599F4F841795070CF093CF41156B
:106F6000510509F48FCFCA01019787CF80819181A4
:106F700082599F4F861797070CF069CF61157105ED
:106F800009F465CFCB0101975DCF8FEF90E090932F
:106F9000EB048093EA0477FF99CF1092E9041092F2
:106FA000E80457FF9FCF1092E7041092E60437FFE2
:106FB000A5CF1092E5041092E40408C01092EB04EF
:106FC0001092EA0481CF0E94AD18A8CE80911C09CE
:106FD0009927AA27BB27BC01CD0124EC39E040E06A
:106FE00050E00E944167DC01CB018093A60390939F
:106FF000A703A093A803B093A90380911D09992723
:10700000AA27BB27BC01CD010E944167DC01CB014F
:107010008093A2039093A303A093A403B093A5032A
:1070200008956F927F928F929F92AF92BF92CF926C
:10703000DF92EF92FF920F931F93CF9300E010E047
:1070400078016801469A10933D0500933C05109322
:107050003B0500933A0580E090E0A0E0B0E080932B
:10706000340590933505A0933605B09337051093FA
:10707000470500934605109345050093440510937A
:1070800043050093420510937A0900937909109201
:107090008F0310928E03109217040E94893684E6A3
:1070A00090E00E941F170E9489368091EE0880FFB1
:1070B00010C080911D0390911E03875B934008F0E0
:1070C0007BC080911D0390911E038E5E924008F458
:1070D00073C0CFE18AE090E00E941F1780912304E3
:1070E00090912404080F191F80912704909128047F
:1070F000E80EF91E8091250490912604C80ED91E31
:10710000C150C7FFE7CFA701405F5F4F5695479536
:107110005695479550934705409346059601205F45
:107120003F4F369527953695279530934505209303
:107130004405C801409696958795929582958F70E3
:1071400089279F70892790934305809342059093E8
:107150007A09809379093093410520934005509333
:107160003F0540933E0544E050E0DA010E94D067BD
:10717000802D853020F18091B4099091B50997FD5B
:1071800053C06CE070E00E94806770933B05609391
:107190003A05809198099091990997FD56C06CE045
:1071A00070E00E94806770933D0560933C0580917C
:1071B0006E0890916F084DC00E945B188ACFDA016B
:1071C0000E94D067802D9927982F8827DA01119681
:1071D0000E94D067202D820F911D90933D058093D2
:1071E0003C05DA0112960E94D067802D9927982FCE
:1071F0008827DA0113960E94D067202D820F911DF7
:1072000090933B0580933A05DA0114960E94D0676B
:10721000802D9927982F8827DA0115960E94D0672C
:10722000202D820F911D15C0909581959F4F6CE088
:1072300070E00E94806770933B0560933A058091EF
:1072400098099091990997FFAACF909581959F4FA2
:10725000A6CFAA2797FDA095BA2FBC01CD010E9409
:10726000C766DC01CB018093340590933505A0936C
:107270003605B093370510925D0910925C091092A3
:107280004E0910924D091092AA091092A90984E69C
:1072900090E00E941F1780911F0490912004AA275C
:1072A00097FDA095BA2F9C01AD01220F331F441FFB
:1072B000551F220F331F441F551F280F391F4A1F08
:1072C0005B1F280F391F4A1F5B1F309399092093BA
:1072D00098098091210490912204AA2797FDA095F6
:1072E000BA2F7C018D01EE0CFF1C001F111FEE0C4C
:1072F000FF1C001F111FE80EF91E0A1F1B1FE80EBE
:10730000F91E0A1F1B1FF092B509E092B409809183
:10731000FD08682E772488249924C9019C014427FC
:1073200037FD4095542FC401B3010E9441675B01B2
:107330006C0160932E0570932F0580933005909318
:1073400031059701442737FD4095542FC401B301FF
:107350000E944167DC01CB018093260590932705AD
:10736000A0932805B0932905A0920A05B0920B05B9
:10737000C0920C05D0920D058093020590930305F1
:10738000A0930405B09305051092FE041092FF042B
:10739000109200051092010580911F039091200327
:1073A000A0912103B09122039093710880937008FB
:1073B00010921604109215041092F6041092F7041D
:1073C0001092F8041092F9048091F4049091F5045D
:1073D0009093F3048093F2040E94965D82E390E020
:1073E000909301048093000480911C099927AA2797
:1073F000BB27BC01CD0124EC39E040E050E00E9405
:107400004167DC01CB018856954CAF4FBF4F80934D
:10741000A6039093A703A093A803B093A903809118
:107420001D099927AA27BB27BC01CD010E944167EE
:10743000DC01CB018856954CAF4FBF4F8093A20320
:107440009093A303A093A403B093A50310928B037E
:1074500010928A038091F4049091F504AA2797FD75
:10746000A095BA2F2091860330918703409188031D
:1074700050918903BC01CD010E944167DC01CB0121
:107480008093B0099093B109A093B209B093B30966
:107490001092ED041092EC0481E0809301010E94AF
:1074A0008B618091B20484608093B2048FEF8093EB
:1074B000190A10921A0A80E280931B0A8091EA0846
:1074C000E82FFF27EE0FFF1FEC54F74F80819181CB
:1074D00082599F4F9093EB048093EA048091EB08CC
:1074E000E82FFF27EE0FFF1FEC54F74F80819181AB
:1074F00082599F4F9093E9048093E8048091EC08AF
:10750000E82FFF27EE0FFF1FEC54F74F808191818A
:1075100082599F4F9093E7048093E6048091ED0891
:10752000E82FFF27EE0FFF1FEC54F74F808191816A
:1075300082599F4F9093E5048093E40484E68093FE
:10754000E304469A579ACF911F910F91FF90EF90C5
:10755000DF90CF90BF90AF909F908F907F906F9073
:1075600008959091D904992381F58091B2048C7F7C
:107570008093B20410C0A92FBB27FD01E359F84F37
:107580008083FD01E359F84F8081A556B64F8C9357
:107590009F5F9C3080F48091E203882361F3A92FE0
:1075A000BB27FD01E359F84F8081A556B64F8C9358
:1075B0009F5F9C3080F38091E203882359F0809193
:1075C000E20381508093E20308958091B2048160C8
:1075D0008093B20408958091F1088B3F68F08B3F4F
:1075E00009F4D5C28C3F09F474C38D3F09F4F6C287
:1075F0008E3F21F48091E40480939E038091F008F3
:107600008B3F08F439C28B3F09F434C28C3F09F434
:1076100048C38D3F09F4D9C28E3F09F478C38091E5
:107620009F03882309F02DC280939F038091F20865
:107630008B3F08F42DC28B3F09F428C28C3F09F41C
:1076400042C38D3F09F4C4C28E3F09F45AC38091EE
:107650009D03882309F021C280939D038091F40843
:107660008B3F68F08B3F09F495C28C3F09F42EC321
:107670008D3F09F4B0C28E3F21F48091E4048093E1
:107680009C038091F6088B3F68F08B3F09F479C228
:107690008C3F09F4E2C28D3F09F4BEC28E3F21F453
:1076A0008091E40480939A038091FE088B3F68F0F8
:1076B0008B3F09F469C28C3F09F4FCC28D3F09F489
:1076C00090C28E3F21F48091E40480939B038091CB
:1076D000FF088B3F08F4E8C18B3F09F4E3C18C3FFE
:1076E00009F4EEC28D3F09F494C28E3F09F412C32F
:1076F000809198038B3008F4DCC18F3F11F48093A4
:107700009803809100098B3F68F08B3F09F427C2F2
:107710008C3F09F4D2C28D3F09F466C28E3F21F43A
:107720008091E40480939703809101098B3F68F076
:107730008B3F09F417C28C3F09F489C28D3F09F4CD
:107740006EC28E3F21F48091E4048093990380916E
:1077500002098B3F68F08B3F09F407C28C3F09F4A4
:1077600079C28D3F09F452C28E3F21F48091E40426
:1077700080939603809103098B3F68F08B3F09F457
:10778000F7C18C3F09F4ABC28D3F09F43CC28E3F78
:1077900021F48091E40480939503209108092B3F04
:1077A00008F48BC12B3F09F486C12C3F09F47CC23D
:1077B0002D3F09F404C22E3F09F4A6C22091930381
:1077C000809109098B3F08F07FC18093C6048091A6
:1077D0000A098B3F68F08B3F09F4D0C18C3F09F454
:1077E00066C28D3F09F4EEC18E3F21F48091E4041E
:1077F0008093C50480910B098B3F68F08B3F09F49F
:1078000084C18C3F09F471C28D3F09F4D2C18E3F0F
:1078100021F48091E4048093C40480910C098B3F8F
:1078200068F08B3F09F474C18C3F09F461C28D3F4D
:1078300009F4C2C18E3F21F48091E4048093C30413
:10784000809121098B3F68F08B3F09F464C18C3F24
:1078500009F454C28D3F09F4A3C18E3F21F48091F5
:10786000E4048093C204809122098B3F68F08B3F2F
:1078700009F454C18C3F09F42FC28D3F09F493C120
:107880008E3F21F48091E4048093C1048091230908
:107890008B3F68F08B3F09F444C18C3F09F4ECC185
:1078A0008D3F09F4C5C18E3F21F48091E40480939B
:1078B000C004809124098B3F68F08B3F09F434C1E8
:1078C0008C3F09F4DCC18D3F09F4B5C18E3F21F432
:1078D0008091E4048093BF0480910D098B3F68F090
:1078E0008B3F09F424C18C3F09F4CFC18D3F09F4CB
:1078F00084C18E3F21F48091E404809392038091AF
:1079000011098B3F68F08B3F09F414C18C3F09F4D7
:10791000BFC18D3F09F474C18E3F21F48091E4040E
:1079200080939103809116098B3F68F08B3F09F497
:1079300004C18C3F09F4AFC18D3F09F458C18E3F9B
:1079400021F48091E40480939003809119098B3F86
:1079500068F08B3F09F4F4C08C3F09F49FC18D3F60
:1079600009F448C18E3F21F48091E40480938F0391
:1079700080911A098B3F68F08B3F09F4E4C08C3F7B
:1079800009F46EC18D3F09F44DC18E3F21F4809101
:10799000E40480938E0380911B098B3F68F08B3F3A
:1079A00009F4D4C08C3F09F464C18D3F09F43DC192
:1079B0008E3F21F48091E40480938D03809120090F
:1079C0008B3F68F08B3F09F4C4C08C3F09F45AC167
:1079D0008D3F09F433C18E3F21F48091E4048093FC
:1079E0008C03809126098B3F08F47FC08B3F09F4FC
:1079F0007AC08C3F09F437C18D3F09F422C18E3F14
:107A000009F48BC180917409823008F473C08F3FF0
:107A100011F480937409809128098B3F08F46EC09B
:107A20008B3F09F469C08C3F09F420C18D3F09F4F4
:107A30000BC18E3F09F474C18091A709823008F40C
:107A400062C08F3F11F48093A70980913B098B3F5F
:107A500070F08B3F09F480C08C3F09F44CC18D3F1E
:107A600009F49BC08E3F09F05EC18091E4048093CD
:107A7000B70959C18091EA0480939F03882309F4D0
:107A8000D3CD843608F4D2CD84E6CECD8091EA04FD
:107A900080939D03882309F4DFCD843608F4DECD7E
:107AA00084E6DACD8091EA04809398038B3008F065
:107AB00024CE8AE024CE2091EA042093930380917F
:107AC00009098B3F08F481CE8B3F09F454C08C3FE9
:107AD00009F408C18D3F09F469C08E3F09F077CEE3
:107AE0008091E40472CE8091EA048093740982301C
:107AF00008F08DCF81E08DCF8091EA048093A709B3
:107B0000823008F09ECF81E09ECF8091EA0483CE40
:107B10008091EA0493CE8091EA04A3CE8091EA0496
:107B2000B3CE8091EA04C3CE8091EA04D3CE809193
:107B3000EA04E3CE8091EA04F3CE8091EA0403CF15
:107B40008091EA0413CF8091EA0423CF8091EA0464
:107B500033CF8091EA0443CF8091EA0488CF8091AB
:107B6000EA04E0CD8091EA04F0CD8091EA0400CEF1
:107B70008091EA0410CE8091EA0427CE8091EA0435
:107B800037CE8091EA048ECD8091EA049ECD80911B
:107B9000EA0432CD8091EA0472CD8091E60467CF89
:107BA0008091E6045ECE8091E6046ECE8091E6047C
:107BB0000CCE8091E6042FCE8091E6043FCE20913A
:107BC000E6047BCF8091E60413CE8091E60454CF87
:107BD0008091E6045DCF8091E60451CD8091E6046A
:107BE0000BCD8091E60471CD8091E6049BCD809110
:107BF000E604A9CE8091E604B9CE8091E6047DCE5C
:107C00008091E6048DCE8091E604C5CD8091E60496
:107C1000AFCD8091E60448CF8091E60443CD8091BA
:107C2000E60493CD8091E604B4CE8091E604C4CE00
:107C30008091E6043CCE8091E6044CCE8091E6042F
:107C4000CECE8091E60451CF8091E60457CF80914B
:107C5000E8047BCD8091E8048BCD8091E80422CDAF
:107C60008091E80496CE8091E8043FCF8091E804AB
:107C700045CF8091E804A0CE8091E80418CE809191
:107C8000E80428CE8091E804AACE8091E80435CE9D
:107C90008091E80445CE8091E80455CE8091E804B7
:107CA00065CE8091E804E8CE2091E80406CF80916B
:107CB000E8049ECD8091E80408CD8091E80432CD9F
:107CC0008091E804F1CE8091E804E2CE8091E8044E
:107CD000D6CC8091E80490CC8091E804D5CD8091F9
:107CE000E80459CD8091E80470CD8091E80493CDEB
:107CF0008091E804A3CD8091E804B9CE8091E80496
:107D0000B0CD8091E404C4CE2091E404D6CE80911D
:107D1000E404B2CE8091E404C7CE8091E404E5CEC1
:107D20008091E404EBCE33272F5F3F4F8CE398E242
:107D3000B9010E9480677093A1036093A0038091B2
:107D4000FC088093A8098091FB088093610908953D
:107D50002F923F924F925F926F927F928F929F925B
:107D6000AF92BF92CF92DF92EF92FF920F931F9349
:107D7000CF93DF93CDB7DEB7C954D0400FB6F89498
:107D8000DEBF0FBECDBF8091B104815009F485E004
:107D90008093B1040E94F02C209102012C3008F055
:107DA000B8C2299AA090DA04B090DB04BE86AD86F2
:107DB0008091610999270A96A816B90614F49E873E
:107DC0008D878091E304843608F0A5C280917E05FA
:107DD00090917F05009709F085C41092D904809195
:107DE000B2048F7E8093B2042A3009F483C4243114
:107DF00009F480C428988091B3049091B404895EFA
:107E0000934008F480C480910509282F33273E87CA
:107E10002D878091B20480618093B2048091E6083E
:107E2000A82FBB27AA0FBB1FFD01E653F74F1182F6
:107E300010828091E708282F3327220F331FC901B2
:107E40008653974FFC0111821082AC54B74F1196A4
:107E50001C921E922C54374FD90111961C921E92DF
:107E60008091E908E82FFF27EE0FFF1FEC54F74F32
:107E700011821082809184038150809384038091C9
:107E800084038F3F21F08091B20484FF3FC40E949D
:107E9000EB3A80918D0590918E05AC01440F551FF2
:107EA000480F591FE090E608AE2DBB27AA0FBB1F55
:107EB000FD01EC54F74FC090F8080C2D112780817C
:107EC0009181809F5001819FB00C909FB00C112434
:107ED0004A0D5B1D57FF02C00C947E535595479584
:107EE00055954795A653B74F8091F908682F772786
:107EF0008D919C91869F9001879F300D969F300DAC
:107F00001124240F351F30938E0520938D05809109
:107F1000C4059091C5054091C0055091C105840FDD
:107F2000951F281B390B3093E1042093E0048091C6
:107F30008F0590919005AC01440F551F480F591FB4
:107F4000F090E708AF2DBB27AA0FBB1FFD01EC5433
:107F5000F74F80819181809F9001819F300D909F8C
:107F6000300D1124420F531F57FF02C00C947A5357
:107F70005595479555954795A653B74F8D919C912B
:107F8000869F9001879F300D969F300D1124240FFE
:107F9000351F3093900520938F058091C2059091F5
:107FA000C3054091BE055091BF05840F951F281B46
:107FB000390B3093DF042093DE048091E908E82F29
:107FC000FF27EE0FFF1FEC54F74F808191819095B2
:107FD00081959F4F8330910514F40C947E4A02974B
:107FE0009093DD048093DC048091E808E82FFF275C
:107FF000EE0FFF1FEC54F74F0081118108581F4FFF
:10800000809198039927AA2797FDA095BA2FBC01C4
:10801000CD010E94C766DC01CB0120E030E040E2E8
:1080200051E4BC01CD010E946866DC01CB01BC01BA
:10803000CD010E94AA66DC01CB018093AE09D090ED
:108040009703809196039927AA2797FDA095BA2FA9
:10805000BC01CD010E94C766DC01CB0120E030E00D
:1080600040E251E4BC01CD010E946866DC01CB0115
:10807000BC01CD010E94AA66DC01CB0180935409AA
:108080004091950340936B0980918F0780FF06C054
:108090008091B709813810F00C94E14A1093DB0409
:1080A0000093DA048091DA049091DB0497FF02C018
:1080B0000C948253F091EE08FBA3F2FD02C00C94E5
:1080C000C84A10927B094091E0045091E104CA0132
:1080D00057FF02C00C94D34A95958795959587953F
:1080E00097FF02C00C94DC4A2091B7043091B80489
:1080F0002817390714F00C94864ACA0157FF02C0AA
:108100000C94665797FF02C00C946357BC01759599
:108110006795759567956536710514F40C94894AD1
:1081200064E670E04091DE045091DF04CA0157FD1F
:1081300002C00C94924A03969595879595958795DC
:1081400097FD02C00C949A4A909581959F4F20917B
:10815000B5043091B6042817390714F40C94A34AD7
:10816000215030408091B20484FD02C00C94BE4A7C
:108170001092B8041092B7041092B6041092B5048D
:10818000EF2DFF27EE0FFF1FEC54F74F409117091B
:10819000242F3327808191812817390734F4809167
:1081A0003C0982FF02C00C94554BEF2DFF27EE0FC8
:1081B000FF1FEC54F74F842F992720911809821B39
:1081C0009109208131812817390714F41092CA04CB
:1081D000EF2DFF27EE0FFF1FEC54F74F842F992749
:1081E00022273327281B390B80819181821793071F
:1081F00034F480913C0983FF02C00C94504B809171
:10820000C904882391F0EF2DFF27EE0FFF1FEC54D8
:10821000F74F809118099927841B9109208131819A
:108220008217930714F40C94854BEE2DFF27EE0F65
:10823000FF1FEC54F74F242F33278081918128179B
:10824000390734F480913C0980FF02C00C944A4BFA
:108250005091C704552399F0EE2DFF27EE0FFF1F15
:10826000EC54F74F842F992720911809821B91090C
:10827000208131812817390714F40C94804BEE2D9E
:10828000FF27EE0FFF1FEC54F74F842F992722276B
:108290003327281B390B808191818217930734F48F
:1082A00080913C0981FF02C00C94454B8091C80429
:1082B000882391F0EE2DFF27EE0FFF1FEC54F74FB0
:1082C000809118099927841B910920813181821797
:1082D000930714F40C947C4B8091CA04882331F4E6
:1082E0008091C904882311F40C94424B91E05523EA
:1082F00031F48091C804882311F40C94604B81E020
:108300008093CC041092CB041092CA041092C9043A
:1083100000C2299847CD8091E3048D3808F4AACD96
:108320008091B2048F7E8093B2049091060982E31B
:10833000989FC001112490937F0580937E05ED8561
:10834000FE85B99714F00C94654B8091B30490911D
:10835000B4048F3F910519F010F00C9473531092F0
:1083600062051092630510926405109265051092E3
:1083700066051092670510926805109269058A3F9C
:10838000910511F40C94DA583091E808E32FFF2797
:10839000EE0FFF1FEC54F74F8081918181359105DD
:1083A0000CF4E9C04091D904442309F0E4C0809161
:1083B000E908E82FFF27EE0FFF1FEC54F74F8081ED
:1083C00091818C34910514F40C94F35780918005BD
:1083D0008F5F893C10F40C9460592C3010F00C9491
:1083E000195A29981092D904109280051092B40459
:1083F0001092B304E090E608EE2DFF27EE0FFF1F6A
:10840000EC54F74F808191818734910514F00C94DE
:108410001C5AF090E708EF2DFF27EE0FFF1FEC54DA
:10842000F74F808191810190F081E02DF7FF02C02C
:108430000C94AF5CE734F1050CF470C021E0AF2D73
:10844000BB27AA0FBB1FAC54B74F8D919C911197BE
:108450008734910544F0EE2DFF27EE0FFF1FEC54FB
:10846000F74F808191818D919C918734910564F0C3
:10847000EE2DFF27EE0FFF1FEC54F74F8081918107
:10848000873491050CF022E0EF2DFF27EE0FFF1F40
:10849000EC54F74F808191818634910564F4EE2D80
:1084A000FF27EE0FFF1FEC54F74F80819181873437
:1084B00091050CF023E0EF2DFF27EE0FFF1FEC548A
:1084C000F74F808191818A5B9F4F64F4EE2DFF27E7
:1084D000EE0FFF1FEC54F74F808191818734910597
:1084E0000CF024E0EF2DFF27EE0FFF1FEC54F74FA9
:1084F000808191818A5B9F4F64F4EE2DFF27EE0F00
:10850000FF1FEC54F74F80819181863491050CF464
:1085100025E0822F0E942405F090E708EF2DFF2729
:10852000EE0FFF1FEC54F74F808191810190F08195
:10853000E02DF7FF02C00C94445C7E9714F00C947D
:10854000CB598091E608E82FFF27EE0FFF1FEC5470
:10855000F74F808191818A5B9F4F14F00C94CB5927
:1085600081E08093830788EE93E0909301048093E9
:1085700000043091E808E32FFF27EE0FFF1FEC54B3
:10858000F74F808191818B5A9F4F0CF073CCD09024
:10859000E908ED2DFF27EE0FFF1FEC54F74F808108
:1085A0009181855B9F4F14F00C94945480918105C8
:1085B0008F5F893C10F40C94CA5788EE93E0909337
:1085C00001048093000488EC8093810581E090E0B1
:1085D0009093B4048093B30481E08093D904109203
:1085E0006A0510926B0510926C0510926D05109241
:1085F000FE041092FF0410920005109201051092E3
:10860000FA041092FB041092FC041092FD04809175
:10861000FD08E82EFF2400271127809198099091EA
:1086200099099C01442737FD4095542FC801B70193
:108630000E944167DC01CB0180930E0590930F05EA
:10864000A0931005B09311058091B4099091B509DC
:108650009C01442737FD4095542FC801B7010E9463
:108660004167DC01CB018093060590930705A09339
:108670000805B093090580912E0590912F05A091D2
:108680003005B091310580930A0590930B05A093B6
:108690000C05B0930D058091260590912705A091BA
:1086A0002805B09129058093020590930305A093B6
:1086B0000405B093050510926205109263051092AF
:1086C0006405109265051092660510926705109278
:1086D0006805109269058091B20488608093B204A5
:1086E0000C949654019790937F0580937E052A30D1
:1086F00009F07DCB289A8091B3049091B404895EEF
:10870000934008F080CB1092D904B4CBA090EE082F
:10871000ABA20091CB040AA3002321F48091CC04E6
:10872000882369F08091160999272D853E85821747
:10873000930714F49E878D8781E08093EE048091E7
:10874000B20484FFD7C61092DD041092DC041092AC
:10875000E1041092E0041092DF041092DE049AE526
:108760009093AE0988E780937B099093540989A37D
:1087700080936B091092CB041092CC041AA2209122
:108780006E0930916F0940917009509171096091A3
:108790002E0570912F0580913005909131056CA7C1
:1087A0007DA78EA79FA7260F371F481F591F8091AF
:1087B000750990917609A0917709B0917809A090F8
:1087C0002605B0902705C0902805D0902905A9AEB0
:1087D000BAAECBAEDCAE8A0D9B1DAC1DBD1DC090EC
:1087E0006309D0906409E0906509F09066092A96C3
:1087F000CCAEDDAEEEAEFFAE2A97E0902A05F0904B
:108800002B0500912C0510912D05ECAAFDAA0EABAD
:108810001FAB2A96ACACBDACCEACDFAC2A97AE0C8D
:10882000BF1CC01ED11E2A96ACAEBDAECEAEDFAE12
:108830002A97C0905509D0905609E0905709F090BA
:1088400058092696CCAEDDAEEEAEFFAE2697E09090
:108850002205F09023050091240510912505EEA234
:10886000FFA208A719A72696ACACBDACCEACDFAC76
:108870002697AE0CBF1CC01ED11E2696ACAEBDAE58
:10888000CEAEDFAE2697B090CC04BDAEBB2009F0D3
:10889000CCC50AA1002309F0C8C58093750990933F
:1088A0007609A0937709B093780920936E093093E5
:1088B0006F09409370095093710980916E089091EF
:1088C0006F08815092400CF074C48091D9048823C1
:1088D00009F06FC480911304909114048F3F9105A7
:1088E00009F008F477C5BDADBB2309F012C7EAA1B2
:1088F000EE2309F00EC7F091EE04F8AFFF2309F064
:1089000008C7A0901F09ADA2AA2009F402C72A96A1
:10891000CCACDDACEEACFFAC2A97C0926309D09230
:108920006409E0926509F09266092696ECACFDAC0C
:108930000EAD1FAD2697E0925509F09256090093AF
:1089400057091093580980916E0990916F09A09171
:108950007009B0917109B7FF02C00C94725B292EA7
:108960003A2E4B2E552447FC5A9420926E09309291
:108970006F09409270095092710980917509909128
:108980007609A0917709B0917809B7FF02C00C94DD
:108990006C5B892F9A2FAB2FBB27A7FDBA958F87CA
:1089A000988BA98BBA8B8093750990937609A093C5
:1089B0007709B09378098091FD08E82EFF240027FD
:1089C000112720911E0530911F05409120055091DF
:1089D0002105C801B7010E94416797FF02C00C94AE
:1089E000665B672E782E892E992487FC9A942091B5
:1089F0001A0530911B0540911C0550911D05C801B9
:108A0000B7010E94416797FF02C00C94605BA72EDC
:108A1000B82EC92EDD24C7FCDA94D201C101861913
:108A20009709A809B90920911E09E22EFF24002701
:108A30001127BC01CD01A80197010E94B56739013A
:108A40004A0122962CAF3DAF4EAF5FAF22978F8584
:108A50009889A989BA898A199B09AC09BD09BC0101
:108A6000CD01A80197010E94B567D401C30197FE0B
:108A700002C00C944D5B892F9A2FAB2FBB27A7FD0B
:108A8000BA95BC01DA01C90157FF02C00C94475BDB
:108A9000892F9A2FAB2FBB27A7FDBA952C01809168
:108AA000B7049091B80481349105D4F48091B50451
:108AB0009091B604813491059CF48091E908E82FE7
:108AC000FF27EE0FFF1FEC54F74F8081918101903B
:108AD000F081E02DF7FF02C00C94B45C7A9734F07B
:108AE0008091190A8F3F11F40C94205AECA8FDA82C
:108AF0000EA91FA92CA53DA54EA55FA5E21AF30A54
:108B0000040B150BE0926E05F0926F050093700553
:108B1000109371058EA19FA1A8A5B9A5A9ACBAAC67
:108B2000CBACDCAC8A199B09AC09BD098B8B9C8B47
:108B3000AD8BBE8B8093720590937305A0937405E3
:108B4000B0937505E0927605F0927705009378056D
:108B50001093790580937A0590937B05A0937C050B
:108B6000B0937D0580910A0590910B05A0910C05AD
:108B7000B0910D058E199F09A00BB10B80930A05CA
:108B800090930B05A0930C05B0930D058091020501
:108B900090910305A0910405B09105052B893C89AE
:108BA0004D895E89821B930BA40BB50B8093020544
:108BB00090930305A0930405B09305053DA13323CD
:108BC00071F12091EC043091ED042138310594F0DD
:108BD00080914205909143050196909343058093BF
:108BE00042058091790990917A09019690937A09CA
:108BF0008093790920583F4F94F4809142059091D9
:108C0000430501979093430580934205809179092C
:108C100090917A09019790937A098093790910923B
:108C2000ED041092EC0491E0292E312CD801C701FB
:108C300017FF02C00C94575B81509240A040B04097
:108C40001CF084E0282E312C809197059091980596
:108C5000A0919905B0919A05A0906E09B0906F0906
:108C6000C0907009D09071098A199B09AC09BD099F
:108C7000815E914BAF4FBF4F8F539C49A040B04096
:108C800010F40C945759F0911A0AFCA3F93114F41A
:108C90000C94ED59309292052092910531E0E31643
:108CA00030E1F30630E0030730E0130714F40C94CE
:108CB000755980919305882311F40C948A5B709305
:108CC000CE046093CD04D801C70117FF02C00C94F5
:108CD000045D9C01AD01B7FF02C00C94135DB9E0C7
:108CE0005595479537952795BA95D1F78091910578
:108CF00090919205820F931F909392058093910516
:108D0000A801970117FF02C00C940D5D39014A01BB
:108D1000A3E09594879477946794AA95D1F72296C7
:108D20006CAE7DAE8EAE9FAE229749E8641643E1ED
:108D3000740640E0840640E0940664F0F8E86F2E84
:108D4000F3E17F2E812C912C22966CAE7DAE8EAEFF
:108D50009FAE2297D401C30197FE02C00C94F25C2F
:108D6000892F9A2FAB2FBB27A7FDBA95680F791FC4
:108D700050E0E51650EFF5065FEF05075FEF1507CA
:108D800014F00C94855980919405882311F40C9467
:108D90008F5B7093CE046093CD04D801C70117FF99
:108DA00002C00C94195D9C01AD01B7FF02C00C9488
:108DB000EC5C69E055954795379527956A95D1F70D
:108DC0008091910590919205820F931F9093920547
:108DD00080939105A801970117FF02C00C94E65CEF
:108DE00039014A0143E095948794779467944A95B2
:108DF000D1F768E766166CEE76066FEF86066FEFC2
:108E0000960644F438E7632E3CEE732E3FEF832E34
:108E10003FEF932E609285057092860580928705BC
:108E200090928805D401C30197FE02C00C94D75CD0
:108E3000892F9A2FAB2FBB27A7FDBA956091CD0440
:108E40007091CE04680F791F4DA1242F3327809194
:108E50009105909192052817390724F430939205D3
:108E6000209391055CA1552379F0252F332727FD09
:108E7000309580919105909192052817390724F437
:108E8000309392052093910581E8E816F1040105DD
:108E9000110574F080914605909147052091910548
:108EA00030919205820F931F90934705809346055A
:108EB00090E8E9169FEFF9069FEF09079FEF190762
:108EC00074F4809146059091470520919105309169
:108ED0009205821B930B9093470580934605B1E062
:108EE0002B2E312C8B899C89AD89BE89B7FF02C09E
:108EF0000C943E5B81509240A040B0401CF0A4E036
:108F00002A2E312C20E030E040E050E080919B059B
:108F100090919C05A0919D05B0919E05E0907509EA
:108F2000F090760900917709109178098E199F09C0
:108F3000A00BB10B815E914BAF4FBF4F8F539C493C
:108F4000A040B04028F08CA1893114F40C94035A4D
:108F500030929205209291058B899C89AD89BE89BA
:108F600081509041A040B04014F40C947959809104
:108F70009505882311F40C94785B5092D0044092AC
:108F8000CF048B899C89AD89BE89B7FF02C00C9440
:108F9000DD5CB7FF02C00C94CB5CF9E0B595A795FA
:108FA00097958795FA95D1F7280E391E309292053C
:108FB000209291052B893C894D895E8957FF02C01B
:108FC0000C94C55CE3E05595479537952795EA9550
:108FD000D1F72938F3E13F07F0E04F07F0E05F07F2
:108FE00014F40C94535C88E893E1A0E0B0E0809323
:108FF000890590938A05A0938B05B0938C05809189
:10900000890590918A05A0918B05B0918C05B7FFD9
:1090100002C00C94F85C892F9A2FAB2FBB27A7FDB9
:10902000BA954090CF045090D004480E591E2B8919
:109030003C894D895E89203080EF38078FEF4807E3
:109040008FEF580714F00C949F5980919605882350
:1090500011F40C94855B5092D0044092CF04DA0155
:10906000C90157FF02C00C94285D9C01AD01B7FFF8
:1090700002C00C94225DF9E05595479537952795E8
:10908000FA95D1F78091910590919205820F931FE7
:1090900090939205809391052B893C894D895E8937
:1090A00057FF02C00C94D15CE3E055954795379586
:1090B0002795EA95D1F728379CEE39079FEF4907A6
:1090C0009FEF590714F00C94495C88E79CEEAFEFD2
:1090D000BFEF8093890590938A05A0938B05B09389
:1090E0008C058091890590918A05A0918B05B0919E
:1090F0008C05B7FF02C00C94FE5C892F9A2FAB2F12
:10910000BB27A7FDBA954090CF045090D004480EDD
:10911000591EADA12A2F3327809191059091920578
:109120002817390724F43093920520939105BCA1A8
:10913000BB2379F02B2F332727FD309580919105A4
:10914000909192052817390724F4309392052093C3
:1091500091052B893C894D895E892138310541056E
:10916000510574F080914405909145052091910539
:1091700030919205820F931F90934505809344058B
:109180008B899C89AD89BE8980589F4FAF4FBF4F57
:109190000CF0D5C280914405909145052091910530
:1091A00030919205821B930B909345058093440563
:1091B000C6C29090190A6FEF961611F40C9488535A
:1091C0008091FD08A82EBB24CC24DD246CA57DA5B0
:1091D0008EA59FA5A60195010E94B56779018A0118
:1091E0008091980990919909AA2797FDA095BA2F87
:1091F000E81AF90A0A0B1B0B69AD7AAD8BAD9CAD71
:10920000A60195010E94B56759016A018091B409D0
:109210009091B509AA2797FDA095BA2FA81AB90A67
:10922000CA0ADB0A292C332427FC3094432C532C04
:10923000C201B101A80197010E94416797FF02C0D6
:109240000C949E573B014C01F9E0959487947794D8
:109250006794FA95D1F7C201B101A60195010E9468
:10926000416797FF02C00C94BF585B016C01E9E0B5
:10927000D594C794B794A794EA95D1F78091B70491
:109280009091B804813491053CF48091B50490919B
:10929000B60481349105C4F0D401C30197FE02C025
:1092A0000C94D0583C014D01959487947794679421
:1092B000D601C501D7FE02C00C94D5585C016D01E2
:1092C000D594C794B794A7948091E908E82FFF2715
:1092D000EE0FFF1FEC54F74F808191810190F081D8
:1092E000E02DF7FF02C00C94B1587A97A4F0C401A6
:1092F000B30123E030E040E050E00E94B56739015F
:109300004A01C601B50123E030E040E050E00E9490
:10931000B56759016A0180911B0A282F332727FD61
:109320003095432F532F261537054805590514F45A
:1093300039014A01992787FD9095909581959F4F16
:10934000AA2797FDA095BA2F681679068A069B066C
:1093500014F43C014D012A153B054C055D0514F440
:1093600059016A01A816B906CA06DB0614F45C01A5
:109370006D0180910E0590910F05A0911005B0919F
:10938000110586199709A809B90980930E059093CC
:109390000F05A0931005B0931105809106059091DB
:1093A0000705A0910805B09109058A199B09AC0928
:1093B000BD098093060590930705A0930805B09317
:1093C000090580911304909114048F3F910511F0C9
:1093D00008F089CA2A96ACACBDACCEACDFAC2A97FB
:1093E000A0926309B0926409C0926509D09266099F
:1093F0002696CCACDDACEEACFFAC2697C0925509FE
:10940000D0925609E0925709F09258090091EE0463
:1094100008AF0091DC041091DD04C80117FFEFC113
:1094200088279927801B910BEAC110921E05109284
:109430001F05109220051092210510921A05109216
:109440001B0510921C0510921D0510926E091092BA
:109450006F0910927009109271091092750910929B
:109460007609109277091092780926961CAE1DAEE7
:109470001EAE1FAE269720E030E040E050E02A9676
:109480002CAF3DAF4EAF5FAF2A9780910E05909104
:109490000F05A0911005B091110580930A059093D6
:1094A0000B05A0930C05B0930D05809106059091D6
:1094B0000705A0910805B0910905809302059093D6
:1094C0000305A0930405B0930505109214041092AF
:1094D00013041092CE041092CD041092D004109276
:1094E000CF043DAD332309F0F5C94AA1442309F067
:1094F000F1C9E3C930916B0939A341C93FEF8E3FF0
:1095000093070CF0D7C002960C94F03FB90161505C
:1095100070404091DE045091DF04CA0157FF02C041
:109520000C949B40959587959595879597FF02C0DC
:109530000C94A4402091B5043091B6042817390743
:1095400014F00C94B040CA0157FF02C00C946E573F
:1095500097FF02C00C946B579C0135952795359564
:1095600027952536310514F40C94B24024E630E0FA
:109570008091B20484FF02C00C94B8403093B604CA
:109580002093B5047093B8046093B7040C94C04062
:10959000D0927B094091E0045091E104CA0157FD4B
:1095A00002C00C946C400396959587959595879588
:1095B00097FD02C00C947440909581959F4F0C9438
:1095C000744080918807992787FD90954C2D5527E9
:1095D000849FB001859F700D949F700D1124CB0165
:1095E0002091E0043091E104820F931F9093E104F5
:1095F0008093E00480918907992787FD9095849F47
:10960000D001859FB00D949FB00D1124CD01209104
:10961000DE043091DF04820F931F9093DF04809368
:10962000DE0480918A07992787FD90952091DC04BC
:109630003091DD04820F931F9093DD048093DC044E
:1096400080918C07282F332727FD30958091F308D0
:109650009927289FF001299FF00D389FF00D1124C4
:10966000F0938B03E0938A0380918B0799278017EF
:10967000910714F00C944E409093DB048093DA042D
:109680000C945240982F0C94774181E08093C80449
:109690000C946C4181E08093C704582F0C943F4197
:1096A00081E08093C9040C94154181E08093CA0441
:1096B0000C94E8401092DD041092DC040C94F43F0A
:1096C0009093CB048093CC0424C88091D904882340
:1096D00011F40C94A5418091B3049091B404FFEF70
:1096E0008F3F9F0711F40C94A94101969093B40405
:1096F0008093B3040C94A9411092C8040C946C415B
:109700001092C70450E00C943F411092C9040C948D
:10971000154160E070E02B011092EE0418AEA090AD
:109720006E09B0906F09C0907009D0907109E090F7
:109730007509F09076090091770910917809809168
:109740007B09882309F0A7C71092D0041092CF0498
:109750001092CE041092CD04A0929705B092980575
:10976000C0929905D0929A05E0929B05F0929C05D3
:1097700000939D0510939E0510921E0510921F05E3
:10978000109220051092210510921A0510921B05C7
:1097900010921C0510921D051092160510921705C7
:1097A000109218051092190510926E0910926F0907
:1097B0001092700910927109109275091092760931
:1097C0001092770910927809109263091092640937
:1097D0001092650910926609109255091092560967
:1097E0001092570910925809109214041092130401
:1097F0000091DC041091DD04C80117FD11CE4097E3
:1098000074F0F8EE2F2EF3E03F2E3092AB0320924F
:10981000AA032BA124FD03C081E080938405B090AE
:10982000FA08CB2CDD24EE24FF24B801882777FD2D
:109830008095982F980117FD3CC7442737FD409528
:10984000542F0E9441679B01AC01C701B6010E94E1
:10985000416797FD29C7E9E09595879577956795C5
:10986000EA95D1F79B018B2D9927809FA001819FBD
:10987000500D909F500D1124CA0157FD32C7959588
:10988000879595958795280F391FC901AA2797FDB8
:10989000A095BA2F80936A0590936B05A0936C05F1
:1098A000B0936D052091FE043091FF0440910005B6
:1098B00050910105281B390B4A0B5B0B213563ECDA
:1098C000360760E0460760E056070CF424C680E5E2
:1098D00093ECA0E0B0E08093FE049093FF04A0938B
:1098E0000005B09301058091FE049091FF04A091C2
:1098F0000005B0910105805B9C43AF4FBF4F64F4FE
:1099000080EB9CE3AFEFBFEF8093FE049093FF04E6
:10991000A0930005B09301056090F4047090F504E5
:109920006114710409F44BC18BA183FFADC68CA5F2
:109930009DA5AEA5BFA5B7FF02C00C94985759E0EE
:10994000B595A795979587955A95D1F76C0197FF8F
:1099500002C00C94925789AD9AADABADBCADB7FFC8
:1099600002C00C948C5749E0B595A79597958795BB
:109970004A95D1F7BC0197FF02C00C948757C616D1
:10998000D7060CF46B01B601D7FE02C00C947857D1
:109990002B015594479455944794559447940894B3
:1099A000411C511CACE1B2E06A0E7B1E7301002722
:1099B000F7FC0095102FE4EEFDEF6E0E7F1E8090F9
:1099C000B0099090B109A090B209B090B30920916C
:1099D000860330918703409188035091890328AB17
:1099E00039AB4AAB5BABC501B4010E94B567E21A63
:1099F000F30A040B150BC801B70128E631E040E07B
:109A000050E00E94B567DC01CB018C01045B104083
:109A10004091A9095091AA095BA74AA7CA0157FF1B
:109A200002C00C9473578138910514F000E010E0E7
:109A30002090AA033090AB0321143104A1F459E122
:109A4000C516D10484F48091EC049091ED04800F4C
:109A5000911F9093ED048093EC04809184058823FA
:109A600011F00C94DA57C801880F991F880F991FBD
:109A7000880F991FB2010E9480679B01442737FD20
:109A80004095542F280D391D4A1D5B1D2093B009A8
:109A90003093B1094093B2095093B309F0909B03FE
:109AA0006F2D77276C9DC0016D9D900D7C9D900D55
:109AB000112497FF02C00C9484576C01D594C7946D
:109AC000D594C794D594C794D594C794D594C79486
:109AD0006C197D096B0177FF02C00C947C5721142F
:109AE000310411F00C94B6580091B7041091B804E9
:109AF0008091B5049091B604080F191F17FF02C09A
:109B00000C94135915950795159507951595079577
:109B1000005C1F4FCA01B90128A939A94AA95BA94C
:109B20000E94B567DA01C9012091F2043091F30473
:109B3000442737FD4095542F821B930BA40BB50B84
:109B4000845E9D4FAF4FBF4FBC01CD0128E631E091
:109B500040E050E00E94B567DC01CB01845B90409F
:109B60008C9DB0018D9D700D9C9D700D1124CB01BD
:109B7000B8010E94806783E0F89E60011124C61638
:109B8000D70614F00C94A558B601CB01AA2797FD6F
:109B9000A095BA2F2091FE043091FF04409100055A
:109BA00050910105820F931FA41FB51F8093FE04DF
:109BB0009093FF04A0930005B093010506C0809127
:109BC000A9099091AA099BA78AA780918305815032
:109BD0008F3F09F4A9C480938305F8ADFF2381F07A
:109BE000109266051092670510926805109269053B
:109BF000109262051092630510926405109265053B
:109C0000ADACAA2009F084C480917B099927AA27CA
:109C1000BB27BC01CD012CA53DA54EA55FA50E948B
:109C20004167DC01CB01BC01CD0128EF3AE240E005
:109C300050E00E94B56729010AA1002309F065C41C
:109C400080917B099927AA27BB27BC01CD0129ADAB
:109C50003AAD4BAD5CAD0E944167DC01CB01BC016C
:109C6000CD0128EF3AE240E050E00E94B5671901CB
:109C700000914F0910915009093C11050CF43DC4A5
:109C800008EC10E01093500900934F09E0905A0936
:109C9000F0905B0939ECE316F1040CF423C4E8EC12
:109CA000EE2EF12CF0925B09E0925A0980915C094A
:109CB00090915D09AA2797FDA095BA2F2091AE0932
:109CC000A22EBB24CC24DD24BC01CD01A60195012C
:109CD0000E9441679B01AC01C801AA2797FDA0958E
:109CE000BA2F67E0880F991FAA1FBB1F6A95D1F78B
:109CF000280F391F4A1F5B1F57FDEEC406E055951C
:109D00004795379527950A95D1F74201820E931E04
:109D1000340180914D0990914E09AA2797FDA09595
:109D2000BA2FBC01CD01A60195010E9441679B019C
:109D3000AC01C701AA2797FDA095BA2F17E0880F9D
:109D4000991FAA1FBB1F1A95D1F7280F391F4A1F49
:109D50005B1F57FDBCC4B6E05595479537952795D1
:109D6000BA95D1F76101C20ED31E56016AA57BA533
:109D7000660F771FCB01AA2797FDA095BA2F2091D8
:109D80005409332744275527BC01CD010E94416760
:109D90007B018C0197FD92C4A6E015950795F79479
:109DA000E794AA95D1F7E9A18E2F9927AA27BB2777
:109DB000209112053091130540911405509115051D
:109DC000BC01CD010E944167DC01CB01BC01CD018A
:109DD00020EF35E540E050E00E94B567E20EF31E4B
:109DE000FBA6EAA6C701F1E08F16F0E49F0624F077
:109DF000812CF0E49F2E340100E0801600EC9006E8
:109E00000CF06BC3812CE0EC9E2E90925D09809249
:109E10005C0911E0C11610E4D10624F0C12C70E4F5
:109E2000D72E560120E0C21620ECD2060CF050C30B
:109E3000C12C60ECD62ED0924E09C0924D094AA595
:109E40005BA54150504424F080E090E49BA78AA792
:109E5000AAA5BBA5A050B04C0CF035C300E010EC97
:109E60001BA70AA71093AA090093A90980910001D2
:109E7000482F5527809127039091280348175907A9
:109E800094F420912703309128036D857E85469FA9
:109E9000C001479F900D569F900D1124B9010E945B
:109EA0006C677E876D878D859E85880F991F880FCB
:109EB000991F9E878D879BA190FF51C0AAA1AA23BD
:109EC00009F04DC0BDADBB2309F049C08091A30589
:109ED0009091A4059093550880935408809115049F
:109EE0009091160490934F0880934E082091480556
:109EF000309149052115310509F0D3C480911D0326
:109F000090911E038959934010F00C94CD57809185
:109F10001D0390911E038436910510F00C94325964
:109F200087B58B3010F40C94F45A809117048F5F2E
:109F3000809317049AE08902900111248091780897
:109F4000821B87BD8CE291E0909301048093000412
:109F50008EE591E09093490580934805C3C4B09085
:109F6000A809809161099927880F991F880F991F67
:109F70008896ED85FE85E817F90714F49E878D878E
:109F80008B2D9927880F991F880F991F8055904016
:109F9000AD84BE848A159B0514F49E878D878091BD
:109FA0004B04882391F08091B3049091B4040297FC
:109FB000C09758F4ED84FE841E141F0434F481E02D
:109FC00090E09093B4048093B3048091E004909166
:109FD000E104B401681B790B70936D0960936C09FF
:109FE000E0917B09EE2309F468C2481A590AC201BC
:109FF000AA2797FDA095BA2F20916205309163059D
:10A000004091640550916505820F931FA41FB51FF1
:10A010008093620590936305A0936405B0936505F2
:10A020008091620590916305A0916405B0916505EA
:10A0300081300AEF900700E0A00700E0B00764F06D
:10A0400080E09AEFA0E0B0E0809362059093630512
:10A05000A0936405B093650580509640AF4FBF4F05
:10A0600064F480E096E0AFEFBFEF809362059093D9
:10A070006305A0936405B09365058091DE0490911B
:10A08000DF04B601681B790B70934C0960934B0990
:10A09000EE2309F40CC2281A390AC101AA2797FD38
:10A0A000A095BA2F2091660530916705409168050B
:10A0B00050916905820F931FA41FB51F80936605F9
:10A0C00090936705A0936805B09369058091660534
:10A0D00090916705A0916805B091690581302AEFDC
:10A0E000920720E0A20720E0B20764F080E09AEF38
:10A0F000A0E0B0E08093660590936705A0936805A3
:10A10000B093690580509640AF4FBF4F64F480E034
:10A1100096E0AFEFBFEF8093660590936705A0933D
:10A120006805B09369058091E808E82FFF27EE0FD6
:10A13000FF1FEC54F74F8091EA05992787FD909512
:10A140000190F081E02DE80FF91FE530F10514F4DE
:10A15000E0E0F0E0CF01880F991F880F991F880F6A
:10A16000991F8E0F9F1F2091EE05332727FD3095F5
:10A170008E0F9F1FB9010E9480678B018091F205AD
:10A18000992787FD9095880F991F861797070CF4DC
:10A190008C0110933908009338088091D9048823E2
:10A1A00009F482C18091B20484FD7EC11A870987B7
:10A1B000AF01440F551F440F551F8091F605282FFE
:10A1C000332727FD3095CA018E0F9F1FB9010E94CA
:10A1D00080678091FA05992787FD9095680F791F10
:10A1E000788F6F8B8091FE05992787FD9095861754
:10A1F000970714F4988F8F8B80910006282E3324B4
:10A2000027FC30944F89588D249EC001259E900DC7
:10A21000349E900D11246FE770E0681B790B7E8FE0
:10A220006D8F80910406482E552447FC5094449E1F
:10A23000C001459E900D549E900D112481589F4F52
:10A2400098A38F8F80910806A82FBB27A7FDB095F4
:10A25000BA8FA98FA49FF001A59FF00DB49FF00DB8
:10A260001124E158FF4FFC8FEB8F8091FD08992757
:10A27000880F991F880F991F7C010027F7FC009514
:10A28000102F6CA57DA58EA59FA5A80197010E9402
:10A29000B56759016A0169AD7AAD8BAD9CADA80176
:10A2A00097010E94B56739014A0180910A06282F5B
:10A2B000332727FD3095C501B9010E9480678B01C6
:10A2C0008091E608E82FFF27EE0FFF1FEC54F74FB1
:10A2D00020813181C901880F991F880F991F880F2C
:10A2E000991F820F931F40910206552747FD5095F5
:10A2F000820F931FBA010E948067061B170B209ED6
:10A30000C001219E900D309E900D1124AD8CBE8C0D
:10A31000A81AB90A409EC001419E900D509E900D12
:10A320001124CF8CD8A0C80ED91EE98CFA8CE09EDF
:10A33000C001E19E900DF09E900D11240B8D1C8D9F
:10A34000081B190B1C8F0B8F1E830D8380910E062B
:10A35000282F332727FD3095C301B9010E9480675C
:10A360008B018091E708E82FFF27EE0FFF1FEC54C9
:10A37000F74F20813181C901880F991F880F991FDC
:10A38000880F991F820F931F40910606552747FD9E
:10A390005095820F931FBA010E948067061B170B0E
:10A3A000209EC001219E900D309E900D1124A80E7C
:10A3B000B91EBE8EAD8EBA82A982409EC001419E5A
:10A3C000900D509E900D1124C80ED91ED8A2CF8E8C
:10A3D000DC82CB828091E705282F332727FD30953B
:10A3E0008AA59BA5B9010E9480678B018091E9082D
:10A3F000E82FFF27EE0FFF1FEC54F74F40815181EC
:10A4000080911206282F332727FD3095CA01880F27
:10A41000991F880F991FB9010E94806780910C06CF
:10A42000992787FD9095689FA001699F500D789F9F
:10A43000500D11249A01200F311F21583F4F3887AA
:10A440002F836FE770E07C876B87A6EDB3E0BE01DA
:10A450006F5F7F4F08EE15E00EC04F3F510519F0BA
:10A4600014F04FEF50E04D93F3E0AB3DBF0719F010
:10A4700014F00C94605DF80180810C5F1F4F9927E8
:10A4800087FD9095FB0141915191BF01480F591FE4
:10A4900057FFE3CF40E050E04D93F3E0AB3DBF0703
:10A4A00051F34CF30C94605D00E010E07FCECB01E3
:10A4B000AA2797FDA095BA2FF5CDCB01AA2797FD26
:10A4C000A095BA2F99CD9093AA098093A909CECCD3
:10A4D000B0924E09A0924D09B2CC70925D09609283
:10A4E0005C0997CC48E3E4164FEFF4060CF0DECBA2
:10A4F00078E3E72E7FEFF72ED5CB2FEF0833120747
:10A500000CF0C4CB08E31FEFBDCB22243324B0CB27
:10A510004424552491CB2093FE043093FF044093B0
:10A52000000550930105DFC988E180938305809180
:10A53000FD089927880F991F880F991F7C01002714
:10A54000F7FC0095102F6CA57DA58EA59FA5A801F1
:10A5500097010E94B56730932B0820932A0869ADB4
:10A560007AAD8BAD9CADA80197010E94B567309381
:10A570002D0820932C08809198099091990997FDB6
:10A58000A0C4959587959595879590932F0880936E
:10A590002E088091B4099091B50997FD90C49595C6
:10A5A0008795959587959093310880933008EAA513
:10A5B000FBA5F0933308E09332088091D504909185
:10A5C000D604A091D704B091D804BC01CD0125E0F8
:10A5D00030E040E050E00E94B567309335082093AA
:10A5E000340870923B0860923A088091270390915A
:10A5F000280390933D0880933C088091E3049927B9
:10A6000090933F0880933E088091B0099091B109E2
:10A61000A091B209B091B3092091860330918703CC
:10A620004091880350918903BC01CD010E94B56718
:10A6300030934108209340088091150490911604AE
:10A6400090934F0880934E088091830799279093A9
:10A650005108809350088091FD039091FE039093E0
:10A660005308809352088091C4059091C50590933A
:10A670006708809366088091C2059091C305909306
:10A68000690880936808A9CAA091A909B091AA098C
:10A69000BBA7AAA79ACA5092D0044092CF04709345
:10A6A000CE046093CD0458C861507E4F8F4F9F4FAA
:10A6B000D2C822273327201B310BBFC88FE390E07D
:10A6C000A0E0B0E0E80EF91E0A1F1B1F65CB215C5D
:10A6D0003F4F4F4F5F4F3FCB215C3F4F4F4F5F4F3F
:10A6E0000DCB0396CCC88091B20482608093B204F3
:10A6F0000C94C4414D5F5F4F0C94B83F4D5F5F4F6A
:10A700000C946E3F1092DB041092DA040C945A40C1
:10A710008091FD08E82EFF24002711276CA57DA558
:10A720008EA59FA5A80197010E94B56739014A012E
:10A730008091980990919909AA2797FDA095BA2F21
:10A74000681A790A8A0A9B0A69AD7AAD8BAD9CAD0D
:10A75000A80197010E94B56759016A018091B40967
:10A760009091B509AA2797FDA095BA2FA81AB90A02
:10A77000CA0ADB0AD401C30197FC5DC53C014D0147
:10A7800054E095948794779467945A95D1F7D601BD
:10A79000C501D7FC4CC55C016D0144E0D594C7945C
:10A7A000B794A7944A95D1F78091B7049091B804D3
:10A7B000813491050CF4C8C3C401B30123E030E037
:10A7C00040E050E00E94B56739014A01C601B50179
:10A7D00023E030E040E050E00E94B56759016A0193
:10A7E0008091E908E82FFF27EE0FFF1FEC54F74F89
:10A7F000808191810190F081E02DF7FD20C57A974D
:10A80000A4F0C401B30123E030E040E050E00E9436
:10A81000B56739014A01C601B50123E030E040E0E7
:10A8200050E00E94B56759016A0171E26716710430
:10A83000810491042CF030E2632E712C812C912C38
:10A8400080EE68168FEF78068FEF88068FEF9806F8
:10A8500044F420EE622E2FEF722E2FEF822E2FEF78
:10A86000922E91E2A916B104C104D1042CF090E219
:10A87000A92EB12CC12CD12CA0EEAA16AFEFBA068E
:10A88000AFEFCA06AFEFDA0614F00C94B94980EEC8
:10A89000A82E8FEFB82E8FEFC82E8FEFD82E0C94E6
:10A8A000B9498091D5049091D604A091D704B09174
:10A8B000D80444E0880F991FAA1FBB1F4A95D1F7FF
:10A8C0008093180490931904A0931A04B0931B0466
:10A8D000109216041092150421503040309349050F
:10A8E00020934805ABA0A1FE44C080919E03823313
:10A8F00008F003C48091CB03815098F41092EF04C8
:10A900008091D5049091D604A091D704B091D80439
:10A910008093D1049093D204A093D304B093D40431
:10A9200081E08093CB0347C010928105ED2DFF2776
:10A93000EE0FFF1FEC54F74F808191818C3491050D
:10A940000CF4B9C2809182058F5F893C08F42EC354
:10A9500088EE93E090930104809300041092D90450
:10A9600088EC809382051092B4041092B3040C9486
:10A970003A3F20919E0380918A0390918B03820F2E
:10A98000911D2091F3083327829F6001839FD00C93
:10A99000929FD00C1124C601AA2797FDA095BA2F2B
:10A9A0008093D1049093D204A093D304B093D404A1
:10A9B00081E08093EF04E0908603F090870300919C
:10A9C0008803109189036CA57DA58EA59FA5A8017C
:10A9D00097010E94B56759016A0169AD7AAD8BADE7
:10A9E0009CADA80197010E94B567B901C5010E94FD
:10A9F00030664C01CD971CF09CE3892E912CC4014C
:10AA00000E94D6644C018091EF04882309F469C147
:10AA10008091B20499279C012071307084FD61C13E
:10AA200070903E0970FC04C08091EE0881FD1EC547
:10AA3000CD84DE843093A00520939F05E090D5045B
:10AA4000F090D6040091D7041091D8048091D104DD
:10AA50009091D204A091D304B091D4048E159F0597
:10AA6000A007B10714F070FC52C1A090D504B090BB
:10AA7000D6048091D1049091D204A81AB90A809189
:10AA80009D0399278A9DF0018B9DF00D9A9DF00DF5
:10AA90001124CF01F7FD74C69595879595958795F7
:10AAA0009595879595958795C81AD90A209115048B
:10AAB0003091160437FD61C6359527953595279554
:10AAC00035952795293031050CF44DC428E030E048
:10AAD000229F7001239FF00C329FF00C11249701EC
:10AAE000F7FC6AC63595279535952795809115040D
:10AAF00090911604280F391F80919F039927AA2748
:10AB0000BB27442737FD4095542FBC01CD010E943F
:10AB1000416797FD2DC6E7E09595879577956795F1
:10AB2000EA95D1F79B010FEF613870070CF013C461
:10AB300021E83FEFC21AD30AE090F604F090F70440
:10AB40000091F8041091F90417FD04C657E015951B
:10AB50000795F794E7945A95D1F780919C03282F95
:10AB6000332744275527C801B7010E94416797FD45
:10AB7000ECC545E095958795779567954A95D1F70A
:10AB80009B014FEF613874070CF0D1C321E83FEF10
:10AB9000C21AD30A65E970E0A60EB71E7BE2A716BB
:10ABA00071E0B706E8F480919F059091A005892B8C
:10ABB000B9F48091A3059091A4051816190684F4A0
:10ABC0008091A5059091A605C816D9060CF49CC2E3
:10ABD0008091C9039091CA038C159D050CF494C211
:10ABE0008091480590914905892B21F0C090A305DB
:10ABF000D090A40580919A039927AA27BB2720917A
:10AC00001D0A332727FD3095432F532FBC01CD015B
:10AC10000E94416797FDA7C537E095958795779581
:10AC200067953A95D1F79B018FEF213838070CF0E3
:10AC30008AC321E83FEFC21AD30AC601AA2797FDAB
:10AC4000A095BA2F2DE0880F991FAA1FBB1F2A9528
:10AC5000D1F79401442737FD4095542FBC01CD0115
:10AC60000E94B56720937205309373054093740575
:10AC700050937505C0907205D09073058091A10521
:10AC80009091A2059C01220F331F280F391F2C0D14
:10AC90003D1D37FD57C5A9015595479555954795D4
:10ACA000BA018091EF08282F3327220F331F220F7C
:10ACB000331F421753070CF007C3A901B901B09025
:10ACC000A80970FEC0C2AD85BE85A417B5070CF0FB
:10ACD000BAC2AD01B093A205A093A1055E874D87CE
:10ACE00018C06091F708662309F437C177276634E6
:10ACF00071050CF04AC226E430E03093C80320937B
:10AD0000C703AD84BE84B092A205A092A105B09005
:10AD1000A8098091B20481FFF9C18091B20484FD39
:10AD20005EC2E090A705F090A8050091A9051091DA
:10AD3000AA05E114F10401051105B1F4CD84DE8406
:10AD400076010027F7FC0095102FECE0EE0CFF1CBD
:10AD5000001F111FEA95D1F7E092A705F092A80510
:10AD60000093A9051093AA058091150490911604EB
:10AD7000809115049091160497FD95C48436910531
:10AD80000CF076C26D857E859B01442737FD40958A
:10AD9000542FC401AA2797FDA095BA2FBC01CD015D
:10ADA0000E94416797FD31C59B01AC017DE055953F
:10ADB0004795379527957A95D1F72093720530936B
:10ADC000730540937405509375058091B304909179
:10ADD000B40477E0803D970708F00AC4D801C701A2
:10ADE00069E0B695A795979587956A95D1F7E81A82
:10ADF000F90A0A0B1B0BDA01C90123E0880F991F1E
:10AE0000AA1FBB1F2A95D1F7E80EF91E0A1F1B1FA8
:10AE1000E092A705F092A8050093A9051093AA0552
:10AE2000D801C7012CE0B695A795979587952A95E7
:10AE3000D1F79093A4058093A3054091F50844238E
:10AE400009F4F3C355279C01BA010E948067C90128
:10AE5000861B970B9093A6058093A505260F371F99
:10AE60003093CA032093C903C0902E05D0902F05BC
:10AE7000E0903005F0903105CCA6DDA6EEA6FFA649
:10AE8000E0902605F09027050091280510912905EE
:10AE9000E9AEFAAE0BAF1CAF0091A9091091AA0957
:10AEA0001BA70AA780905C0990905D09C0904D098E
:10AEB000D0904E0956C8109282050C943A3F0396E2
:10AEC0006ECB03965ECB03960C948640909581954D
:10AED0009F4F0C94824003960C94AC4A90958195B8
:10AEE0009F4F0C94A84A909581959F4F0C94134DB9
:10AEF000695F7F4F0C94C84C84EF91E09093AB0353
:10AF00008093AA030C94E54D4F960C945D4D70957B
:10AF100061957F4F0C94BF4C81509E4FAF4FBF4FF8
:10AF20000C94B34CD094C194D108D3940C94AB4CF2
:10AF300081509E4FAF4FBF4F0C949F4C61507E4F3E
:10AF40008F4F9F4F0C9422498091B5049091B60485
:10AF5000813491050CF444CC2FCC4091A305509141
:10AF6000A40557FD37C2559547955595479580914E
:10AF7000270390912803209100013327489FF00177
:10AF8000499FF00D589FF00D1124CF01B9010E9487
:10AF90008067ADCE80938105C9CC87B5853F08F029
:10AFA00059C18091170481500C94984F8093820569
:10AFB0000C943A3FC301AA2797FDA095BA2FBC0174
:10AFC000CD0128A939A94AA95BA90E9441674B0173
:10AFD0005C010E94B5673093F3042093F204109251
:10AFE00084050C94334D80819181855B9F4F0CF0DB
:10AFF00035C1809180058F5F80938005893C10F476
:10B000000C94BB422C3008F0BDC32998A4E0B0E0FA
:10B010008FEF082E0E94DD671092D90410928005F0
:10B020001092B4041092B3040E941138A4E0B0E06E
:10B0300080913C0590913D0597FD9BC4892F990F08
:10B04000990B082E0E94DD67A5E0B0E080913C05D9
:10B0500090913D05082E0E94DD67A6E0B0E080914A
:10B060003A0590913B0597FD51C4892F990F990B93
:10B07000082E0E94DD67A7E0B0E080913A0590912C
:10B080003B05082E0E94DD6708E010E08091340542
:10B0900090913505A0913605B0913705BC01CD01E1
:10B0A0000E94AA66DC01CB019C0197FD55C4832F49
:10B0B000992787FD9A95D801082E0E94DD6709E03F
:10B0C00010E08091340590913505A0913605B0913E
:10B0D0003705BC01CD010E94AA66DC01CB01D80175
:10B0E000082E0E94DD670E945F0568E770E00E94FD
:10B0F000CA2C3091E8080C94BB4281E08093EF04A5
:10B1000088EC8093CB0357CC6C016ACD80912E05DF
:10B1100090912F05A0913005B09131058CA79DA786
:10B12000AEA7BFA7C0902605D0902705E0902805C0
:10B13000F0902905C9AEDAAEEBAEFCAEE090A909FD
:10B14000F090AA09FBA6EAA6ADCE882799278C190C
:10B150009D096817790714F00C94C54DBC010C9437
:10B16000C54DF095E195FF4F0C9475490894210861
:10B1700031083092AB032092AA030C94E54D615044
:10B180007E4F8F4F9F4F0C943549673971050CF4F2
:10B1900045C086E990E09093C8038093C703B1CD82
:10B1A0000196A11DB11D0C9452490196A11DB11D1E
:10B1B0000C945E4981E08093840510926A05109298
:10B1C0006B0510926C0510926D051092FE041092A2
:10B1D000FF0410920005109201050C94C4410091E7
:10B1E0002E0510912F0520913005309131050CA7C7
:10B1F0001DA72EA73FA72091260530912705409136
:10B2000028055091290529AF3AAF4BAF5CAF40916B
:10B21000A9095091AA095BA74AA744CE7093C80315
:10B220006093C7036ECD095F1F4F0C94824D0F963C
:10B23000A11DB11DB0CA0F96A11DB11D9FCAF095E9
:10B24000E195FF4FDCCA7093A2056093A1055E876C
:10B250004D875FCD81E08093AC0544CB4093800562
:10B260000C94BB42FDADF093AB05F093AC053ACB2B
:10B2700060912E0570912F058091300590913105D8
:10B280006CA77DA78EA79FA7809126059091270583
:10B29000A0912805B091290589AF9AAFABAFBCAF9B
:10B2A000A091A909B091AA09BBA7AAA7FBCD30928A
:10B2B00092052092910520911A0A2CA30C944E46D7
:10B2C000809380050C94BB42B090A8092B2D3327A6
:10B2D000220F331F220F331F20553040241735070C
:10B2E0000CF0EFCCA901B901ECCC109293050C94B1
:10B2F000B8462093890530938A0540938B05509377
:10B300008C05109295050C94174822962CAD3DADF6
:10B310004EAD5FAD2297209385053093860540930F
:10B32000870550938805109294050C9424476F3F2D
:10B33000710509F00CF42CCC2FEF30E029CC1092E1
:10B3400096050C9489482F3F310509F00CF473CC15
:10B350002FEF30E070CC6F3F710509F00CF4EACBB1
:10B360002FEF30E0E7CB121613060CF4B1CB229F7F
:10B37000C001239F900D329F900D112497FD80C333
:10B38000959587959595879520911504309116048C
:10B39000281B390BB1CB0E945F0545E666EE78E0CD
:10B3A0000E9407058091EE0880FF10C080911D0368
:10B3B00090911E03875B934038F480911D03909118
:10B3C0001E038E5E924010F40E945B180E9411389A
:10B3D000579A89CE4D5F5F4FC6CD609285057092BA
:10B3E00086058092870590928805109292051092AA
:10B3F000910588EE282E83E0382E3092AB03209200
:10B40000AA030C9424472093890530938A0540931E
:10B410008B0550938C051092920510929105A8EE21
:10B420002A2EA3E03A2E3092AB032092AA030C946A
:10B430008948299A0C94F241F090E7080C941E4236
:10B440007093CE046093CD045092D0044092CF0408
:10B45000CB0177FD60C2BC0175956795C20157FCB1
:10B4600058C22C01559447940C9476458091B204AF
:10B4700081FFA5C12091C7033091C803C9010F9670
:10B480004091DA045091DB04841795070CF0C2C197
:10B490008091AB05882309F0BDC18091AD0581FF86
:10B4A000F6C28D7FE090D504F090D6040091D704C9
:10B4B0001091D804E092D104F092D2040093D30406
:10B4C0001093D40481608093AD05421B530B9A0105
:10B4D0002F50304037FDE4C280919F059091A00528
:10B4E000280F391F3093A00520939F0520919F05B9
:10B4F0003091A005C90137FDC5C2815092400CF4BE
:10B50000BEC18091F3089927829FB001839F700D7F
:10B51000929F700D1124CB0160E075E00E9480675E
:10B52000CB01AA2797FDA095BA2F2091D104309185
:10B53000D2044091D3045091D404820F931FA41FCE
:10B54000B51F8093D1049093D204A093D304B093F9
:10B55000D4041092A00510929F0571FE06C08BE4E2
:10B5600090E090930104809300048091F708882371
:10B5700009F085C1E091A305F091A405AF01F7FDA5
:10B5800098C2559547955595479580912703909179
:10B590002803209100013327489FD001499FB00D17
:10B5A000589FB00D1124CD01B9010E948067663407
:10B5B00071050CF05FC226E430E03093C80320939D
:10B5C000C7038091480590914905892B09F4BAC1B8
:10B5D000D801C701E092D104F092D2040093D304C1
:10B5E0001093D4046F013ACA81E08093AB057AC905
:10B5F000AFE0803A9A0708F0C7C0D801C701FAE067
:10B60000B695A79597958795FA95D1F7E81AF90A0F
:10B610000A0B1B0BDA01C901880F991FAA1FBB1F58
:10B62000880F991FAA1FBB1FEFCB1092A60510927F
:10B63000A5058FEF93E09093CA038093C9032091EF
:10B640002E0530912F0540913005509131052CA7E2
:10B650003DA74EA75FA74091260550912705609111
:10B6600028057091290549AF5AAF6BAF7CAF609147
:10B67000A9097091AA097BA76AA714CCB095A095D7
:10B68000909581959F4FAF4FBF4F0C947A47815053
:10B690009F4FAF4FBF4F0C94484581509F4FAF4FC6
:10B6A000BF4F0C943B45909581959F4F67CB882762
:10B6B0009927DC018E199F09A00BB10B0C941C4635
:10B6C00061507F4F8F4F9F4F0C94074561507F4FC4
:10B6D0008F4F9F4F0C94F14481509F4FAF4FBF4FFE
:10B6E0000C94C94481509F4FAF4FBF4F0C94AF444F
:10B6F0002093890530938A0540938B0550938C05E0
:10B7000081E0809395050C94174881E0809396051D
:10B710000C94894881E0809393050C94B846229656
:10B720008CAD9DADAEADBFAD229780938505909356
:10B730008605A0938705B093880581E080939405E2
:10B740000C9424472D5F3F4FA6CA615E7F4F8F4FF9
:10B750009F4F0FCA2FE730E040E050E0E20EF31EAB
:10B76000041F151FF3C961587F4F8F4F9F4F54CA55
:10B7700061587F4F8F4F9F4FCEC9295F3F4F9CC964
:10B780000F968AC9299A42CC80549F4108F0C8C0BC
:10B79000D801C7017BE0B695A795979587957A95CF
:10B7A000D1F7E81AF90A0A0B1B0BDA01C901820F5B
:10B7B000931FA41FB51F28CB2D5F3F4F93C9E09067
:10B7C000D504F090D6040091D7041091D804D80184
:10B7D000C70180599140A040B0408093D10490931C
:10B7E000D204A093D304B093D4042091F708222369
:10B7F00009F493C033273093C8032093C703E09123
:10B80000A305F091A4056F0129C96150704E8F4FB7
:10B810009F4FCACAC9010F97481759070CF04DC06E
:10B820008091AC05882309F048C08091AD0580FF68
:10B8300018C18E7FE090D504F090D6040091D70413
:10B840001091D804E092D104F092D2040093D30472
:10B850001093D40482608093AD05421B530B9A0170
:10B86000215F3F4F37FD28C180919F059091A00532
:10B87000821B930B9093A00580939F0537CEE09198
:10B88000A305F091A4059DCEF095E195FF4F0C9492
:10B890009D422093890530938A0540938B055093F0
:10B8A0008C050C9471482093890530938A05409348
:10B8B0008B0550938C050C94FF472091AD05822F8A
:10B8C000992783709070892B09F456C02C7F2093A0
:10B8D000AD051092A00510929F05E090D504F09060
:10B8E000D6040091D7041091D804E092D104F092CC
:10B8F000D2040093D3041093D40471FEF7CD84EFE7
:10B9000091E09093010480930004F0CD81509F4F0B
:10B91000ACCB0196A6CD01969ECD28E730E06BCF4B
:10B92000D801C7016CE0B695A795979587956A955C
:10B93000D1F7E81AF90A0A0B1B0BE20EF31E041FDB
:10B94000151F66CA8091D1049091D204A091D304AE
:10B95000B091D4046F0182C821503F4FA8CBF0951D
:10B96000E195FF4F0C941A42F095E195FF4F0C942E
:10B970006E4581509F4F62CBE090D504F090D60485
:10B980000091D7041091D804B1CD295F3F4F4F4F9C
:10B990005F4F0C94E24781509E4FAF4FBF4F0C94C6
:10B9A000CD47295F3F4F4F4F5F4F0C945448815014
:10B9B0009F4FAF4FBF4F0C941847B095A0959095EF
:10B9C00081959F4FAF4FBF4F0C94C947295F3F4FA1
:10B9D0004F4F5F4F0C94F04621503E4F4F4F5F4FFB
:10B9E0000C94D94681509F4FAF4FBF4F0C94B04637
:10B9F00081509F4FAF4FBF4F0C940B4881509F4FCA
:10BA0000AF4FBF4F0C947D4888279927DC018E19D2
:10BA10009F09A00BB10B0C946946295F3F4F4F4F14
:10BA20005F4F0C94864621503E4F4F4F5F4F0C9412
:10BA30006F4688279927DC018E199F09A00BB10B4F
:10BA40000C94D34621503E4F4F4F5F4F0C943B48D0
:10BA5000B095A095909581959F4FAF4FBF4F0C9497
:10BA60003548E090D504F090D6040091D7041091A9
:10BA7000D804F0CE67397105BCF026E930E09DCDE1
:10BA800003967ECC88279927821B930B36CDE090B6
:10BA9000D504F090D6040091D7041091D80412CDAB
:10BAA000309521953F4F18CD7093C8036093C7031D
:10BAB00088CD4D5F5F4F65CD309521953F4FD4CEFA
:10BAC000AD8CBE8CB0924308A0924208CF8CD8A017
:10BAD000D0924508C0924408EB8CFC8CF092470849
:10BAE000E092460830934908209348080F89188D42
:10BAF0001093370800933608C75BDF4F0FB6F894F2
:10BB0000DEBF0FBECDBFDF91CF911F910F91FF9090
:10BB1000EF90DF90CF90BF90AF909F908F907F90ED
:10BB20006F905F904F903F902F9008958091BA054D
:10BB30009091BB05A091BC05B091BD058093B20565
:10BB40009093B305A093B405B093B5058091B60565
:10BB50009091B705A091B805B091B9058093AE0555
:10BB60009093AF05A093B005B093B10508951092DE
:10BB7000C5051092C4051092C3051092C205089520
:10BB800084B1806A84B93D9A82E58CBD1DBC459A1A
:10BB900081E08093BA098AEA8093BE0983E88093A2
:10BBA000BF099AE09093C0091092C2091092C1098E
:10BBB0001092C4091092C30910921C0A1092E00955
:10BBC0001092E1098CE48093E20986E08093E30916
:10BBD0009093E4090895EF92FF920F931F93809141
:10BBE000FD089927880F991F880F991F7C0100274E
:10BBF000F7FC0095102F80912E0590912F05A091B4
:10BC00003005B0913105BC01CD01A80197010E941A
:10BC1000B5673093C2092093C109809126059091A0
:10BC20002705A0912805B0912905BC01CD01A801E7
:10BC300097010E94B5673093C4092093C3092091EE
:10BC4000B0093091B1094091B2095091B309DA01BC
:10BC5000C901E3E0880F991FAA1FBB1FEA95D1F71E
:10BC6000820F931FA41FB51F820F931FA41FB51F20
:10BC70002091860330918703409188035091890376
:10BC8000BC01CD010E94B5673093CA092093C90950
:10BC9000E0913805F091390580917209909173090E
:10BCA000BF010E948067CB019B01220F331F220F2F
:10BCB000331F280F391F280F391F37FD1CC1359539
:10BCC0002795359527953093C6092093C50980910E
:10BCD000AC099091AD09BF010E9480679B01220FC2
:10BCE000331F220F331F260F371F260F371F37FD35
:10BCF000FFC035952795359527953093C809209332
:10BD0000C7091092390510923805109273091092E4
:10BD100072091092AD091092AC098091C00999275F
:10BD20008C30910509F4A1C08D3091050CF069C0EB
:10BD30008A30910509F4A4C10B9709F410C18091D0
:10BD4000E009882309F4CBC02091E6093091E70986
:10BD5000C90181509E4F8F5F9340C8F44091E8091C
:10BD60005091E909CA0181509E4F8F5F934078F44A
:10BD70008091EE0885FF0BC03093C5052093C40564
:10BD80005093C3054093C2058AEF8093C705809105
:10BD9000EC099091ED0921E0893692070CF056C12B
:10BDA0009C019093F5048093F4048091F2049091A7
:10BDB000F304281B390BC901845E9D4F68E671E0CE
:10BDC0000E948067845B90409093F1048093F0041C
:10BDD0002091F0093091F1098091000490910104C3
:10BDE0008217930740F480918307882321F43093CE
:10BDF0000104209300048091E509873609F0ADC164
:10BE00002AC18E30910509F476C18E3091050CF46B
:10BE100075C00F9709F093CF809115098093D109D0
:10BE200080913D098093D209809192038093D30938
:10BE300080910E098093D40980910F098093D509D0
:10BE4000809110098093D609809191038093D7093E
:10BE5000809112098093D809809113098093D909A0
:10BE6000809114098093DA096ACF80918307863024
:10BE700018F01092830785E08093D10980913A09E8
:10BE80008093D20980913408909135089093D40919
:10BE90008093D3098091D1049091D204A091D304CE
:10BEA000B091D404BC01CD0125E030E040E050E089
:10BEB0000E94B5673093D6092093D5098091300947
:10BEC0008093D709809131098093D80980913209F4
:10BED0008093D9098091E009882309F035CF109229
:10BEE000C5051092C4051092C3051092C20535C154
:10BEF0002D5F3F4FFECE2D5F3F4FE1CE80912B094E
:10BF00008093D10980912C098093D20980912D09C9
:10BF10008093D30980912E098093D40980912F09B1
:10BF20008093D509809133098093D6098091340993
:10BF30008093D709809135098093D8098091380979
:10BF40008093D909809136098093DA098091370965
:10BF50008093DB09809139098093DC09F0CEF89455
:10BF60008091E808E82FFF27EE0FFF1FEC54F74FF2
:10BF70000190F081E02DE038F1050CF0D1C02FEFF9
:10BF8000E138F20714F4E1E8FFEFE093D109809182
:10BF9000E908E82FFF27EE0FFF1FEC54F74F019041
:10BFA000F081E02DE038F1050CF4CDC0EFE7F0E0D2
:10BFB000E093D2098091E708E82FFF27EE0FFF1FDB
:10BFC000EC54F74F0190F081E02DE038F1050CF4CE
:10BFD000B2C0EFE7F0E0E093D3098091E608E82FE4
:10BFE000FF27EE0FFF1FEC54F74F0190F081E02D7B
:10BFF000E038F1050CF497C0EFE7F0E07894E093B7
:10C00000D4098091EA048093D5098091E804809353
:10C01000D6098091E6048093D7098091E404809347
:10C02000D8098091E3048093D9098091E204809338
:10C03000DA09809138089091390897FD8CC0959560
:10C040008795959587958093DB0979CE2091F404A7
:10C050003091F504AACE8091F2098093190A80915B
:10C06000F30980931B0A8091F40980931A0A809146
:10C07000F50980931C0A8091F60980931D0A6DC012
:10C080008091C6048093D1098091C5048093D20920
:10C090008091C4048093D3098091C3048093D40910
:10C0A0008091C2048093D5098091C1048093D60900
:10C0B0008091C0048093D7098091BF048093D809F0
:10C0C0008091B2048093D9098091B204837F8093D8
:10C0D000B20480912703909128038093DA0980911C
:10C0E00000018093DB09A2E0B0E00E94D067802DC0
:10C0F0008093DC0924CE8091E1098093D10980915D
:10C10000E2098093D2098091E3098093D309809159
:10C11000E4098093D409809102018093D5090FCE60
:10C12000EFE7F0E032CF8FEFE138F8070CF066CFA1
:10C13000E1E8FFEF63CF6FEFE138F6070CF04BCF8C
:10C14000E1E8FFEF48CF4FEFE138F4070CF030CFD4
:10C15000E1E8FFEF2DCF039672CF1F910F91FF9073
:10C16000EF9008958091BA09882309F43BC045985F
:10C170008EEB99E09093BC098093BB098091C60532
:10C18000E82FFF27E453FC4F982F9F5F8081809317
:10C19000C009973008F027C09093C6051092BA09DD
:10C1A0000E94EB5D81E08093BD090000000000006B
:10C1B000000000000000000000000000000000007F
:10C1C000000000000000000000000000000000006F
:10C1D000000000000000000000008091BE09809374
:10C1E000DD098EBD08951092C605D8CF2091BA09F9
:10C1F000222309F045C00DB407FE42C084E08093BD
:10C20000FF03459A3EB58091C80599278130910575
:10C2100009F437C0823091050CF451C0029709F43B
:10C2200039C02091BD09203208F030C04598000087
:10C2300000000000000000000000000000000000FE
:10C2400000000000000000000000000000000000EE
:10C250000000000000000000000000000000E0916D
:10C26000BB09F091BC09E20FF11D80818EBD809168
:10C27000DD099081890F8093DD092F5F2093BD092F
:10C280000895353551F12093C805CBCF81E08093D7
:10C29000BA09F3CF8091DF09E82FFF27E150F64F6D
:10C2A00030838F5F8093DF098A3100F18091C90567
:10C2B000381711F12093E0091092C805B2CF892BED
:10C2C00009F0AFCF2093DF093093C905313809F069
:10C2D000A8CF81E08093C805A4CF8091C905830FC2
:10C2E0008093C90582E08093C8059BCF8091C905E2
:10C2F000830F8093C90595CF8AE1EFEFF9E0A5EEB2
:10C30000B9E001900D928A95E1F781E08093E00910
:10C310001092C80586CF87B18C6087B94298439840
:10C320001092CB0580E88093D4031092CA058093C5
:10C33000D30308958091D00581508F3F19F08093E9
:10C34000D005089584E08093D0058091B20485FFE4
:10C3500016C0409129094093D10560912A09609344
:10C36000D20550913C09252F332724FF13C080911B
:10C37000D904882379F425FF17C0429A33C08091ED
:10C38000E304882334F7409125094093D105609157
:10C390002709E5CF909126099B3FB8F08091740959
:10C3A0008D3D98F047FDE9CF4298252F332724FD96
:10C3B0001DC0909128099B3F08F18091A709873EF5
:10C3C000E8F067FD19C0439808959B3F20F08091E5
:10C3D00074098A3008F18091CB0581508F3F21F19B
:10C3E0008093CB05252F332724FFE3CF8091D904F9
:10C3F0008823F9F626FFE7CF439A08959B3F20F064
:10C400008091A7098A3060F08091CA0581508F3FE2
:10C41000E1F08093CA05089547FDC6CF429AE2CF66
:10C4200067FDD1CF439A089580917409815080931C
:10C43000CB058091D4038130C9F086958093D403D5
:10C44000842309F4B1CF429ACDCF8091A7098150BE
:10C450008093CA058091D303813051F086958093F3
:10C46000D303862309F4AFCF439A089580E8E6CF3B
:10C4700080E8F5CF8091C9008F778093C9008091C3
:10C48000C9008F7B8093C9008091C9008F7D809304
:10C49000C9005A9A52981092CD0084E190E080939E
:10C4A000CC008091C80082608093C80080E18093B6
:10C4B000C9008091CA008F778093CA008091CA001A
:10C4C0008F7B8093CA008091CA008F7D8093CA00C1
:10C4D0008091CA008F7E8093CA008091CA00877FB6
:10C4E0008093CA008091C9008B7F8093C90080919E
:10C4F000CA0084608093CA008091CA0082608093E1
:10C50000CA008091C80087FF0CC08091CE00809146
:10C51000C800882334F48091CE008091C80088231D
:10C52000A4F38091C90080688093C90008951F9387
:10C53000CF93DF9380E197E20E94FD16EC0110E0BB
:10C540008091C9008F778093C9008091C9008F7E48
:10C550008093C9005A988DE797E09F938F931F931C
:10C560000E947E130F900F900F90CE010E9406172D
:10C57000882309F066C04A9BF8CF8AE590E00E94C4
:10C58000FD16EC0183EB97E09F938F931F920E941F
:10C590007E13529A0F900F900F90CE010E940617B3
:10C5A0008823D9F383E690E05A9A019797FFFCCF4E
:10C5B0008FE891E05A98019797FFFCCF89E090E0CF
:10C5C0005A9A019797FFFCCF89E090E05A9801971B
:10C5D00097FFFCCF8FE891E05A9A019797FFFCCF25
:10C5E0008FE891E05A98019797FFFCCF89E090E09F
:10C5F0005A9A019797FFFCCF89E090E05A980197EB
:10C6000097FFFCCF8FE891E05A9A019797FFFCCFF4
:10C610008FE891E05A98019797FFFCCF89E090E06E
:10C620005A9A019797FFFCCF89E090E05A980197BA
:10C6300097FFFCCF8FE891E05A9A019797FFFCCFC4
:10C640000AC089EB97E09F938F931F930E947E13FC
:10C650000F900F900F9052985A980E943A62DF9173
:10C66000CF911F9108951F920F920FB60F92112430
:10C67000EF92FF920F931F932F933F934F935F93EC
:10C680006F937F938F939F93AF93BF93CF93DF93DA
:10C69000EF93FF932091CE008091D503813009F470
:10C6A0004BC08091D3058823C9F040E050E08091D1
:10C6B000D4058823C9F4452B09F44AC081E080934E
:10C6C000D4058091D5058F5F8093D50543E0809197
:10C6D000D5058031E8F44093D30504C141E050E032
:10C6E0008091D405882339F3813009F44AC082301F
:10C6F000B9F1833009F44AC081E08093D5031092E8
:10C70000D5051092D70544E48091D505803118F302
:10C710008091D705882331F48091D503882311F4C3
:10C72000809384031092D5051092D7051092D405FA
:10C7300084E48093D305D6C01092D50384E480931B
:10C74000D3051092D5051092D4051092D605CAC013
:10C7500044E48093D5058093D4058093D605D4CF47
:10C76000452B51F643E02093D6059091D5059230A4
:10C7700009F492C083E08093D4059F5F9093D50520
:10C78000C3CF452B09F0B8CF82E099CF452B09F0F4
:10C79000B3CF482F82E08093D4058091D5058F5F79
:10C7A0008093D5059091D605892F86958695E82F9B
:10C7B000FF27EF70F0703196892F9927982F8827DF
:10C7C0003327822B932B93708050924063E070E06C
:10C7D0000E948067EB30F10508F057C07F01EE0E34
:10C7E000FF1EF701EC54F74F808191819B01281BBC
:10C7F000390BC90137FD6EC0069754F48091E304EC
:10C80000883C08F05BC08091E304865F8093E3047A
:10C81000F701EC54F74F808191819C01220F331F67
:10C82000280F391F260F371F37FD51C0E901D59555
:10C83000C795D595C795CB0101968C179D07BCF57B
:10C8400021978091E304843B60F187010653174FE1
:10C85000F701EC54F74F80819181FE01E81BF90B41
:10C86000CF0163E070E00E948067CB01880F991FC1
:10C87000860F971FF8019183808324EB38E0E20E46
:10C88000F31EF701D183C0833FCF729708F43CCFEA
:10C8900081E08093D50338CF27FD20C01092D705C3
:10C8A00069CFF701E653F74F11821082E6CF61504E
:10C8B0007040C617D7072CF62196C3CF88EC80931B
:10C8C000E30480916F008F7D80936F00A1CF2D5F77
:10C8D0003F4FACCF909581959F4F8ECF81E0809355
:10C8E000D70548CFFF91EF91DF91CF91BF91AF91E5
:10C8F0009F918F917F916F915F914F913F912F9178
:10C900001F910F91FF90EF900F900FBE0F901F900F
:10C910001895CF93FC0197FD21C0C1E028E631E0D6
:10C92000CF01B9010E948067FC018B35910554F05D
:10C930008B5590408A35910538F484EB90E08E1B3E
:10C940009F0BFC0141E013C0CF01855B90408A350D
:10C95000910548F4E45BF0404FEF09C0CFEFF0954C
:10C96000E195FF4FDBCF2E1B3F0BF9014FEFEE0F91
:10C97000FF1FE25EF64F259134918C2F992787FD9A
:10C980009095829FB001839F700D929F700D11242E
:10C99000842F992787FD9095689FA001699F500D6E
:10C9A000789F500D1124CA01CF9108952AE530E0F7
:10C9B000281B390BC9010E94896408951F93CF93E6
:10C9C000DF93EB016115710519F4009709F494C028
:10C9D00097FD3EC011E0209729F48AE51802B001C6
:10C9E00011248AC0AA2797FDA095BA2F26E0880FA8
:10C9F000991FAA1FBB1F2A95D1F79E01442737FD17
:10CA00004095542FBC01CD010E94B567F90137FD57
:10CA10002CC081E0EA35F807ACF08CE1E73AF80782
:10CA2000CCF02AE530E01C161D061CF5812F992755
:10CA300087FD9095829FB001839F700D929F700D2E
:10CA400011245AC0EC53F84F8491282F3327EBCF91
:10CA50001FEFC1CF89E0ED38F8078CF485E0EA3BA1
:10CA6000F80784F028E530E0DECFF095E195FF4F40
:10CA7000D0CFD7FD0EC0B901645B70403DC029E541
:10CA800030E0D1CF84E0E731F80754F027E530E01B
:10CA9000CACF111684F764EB70E0621B730B2CC0D5
:10CAA00083E0EE32F8071CF026E530E0BCCF82E0F0
:10CAB000E939F8071CF025E530E0B5CF82E0E23334
:10CAC000F8071CF024E530E0AECF81E0E73EF80740
:10CAD0001CF023E530E0A7CF81E0ED3AF8071CF029
:10CAE00022E530E0A0CFEF57F1401CF021E530E027
:10CAF0009ACF20E530E097CFCB01DF91CF911F9106
:10CB00000895EF92FF920F931F93CF93DF937B01D2
:10CB10008C0120E030E040E050E0FA01E9016FE0F4
:10CB20000BC0C21BD30BE40BF50B2F5F3F4F4F4FD6
:10CB30005F4F615067FD31C0220F331F441F551FE7
:10CB4000CC0FDD1FEE1FFF1FCC0FDD1FEE1FFF1FE1
:10CB5000D801C7017EE1B695A795979587957A95F7
:10CB6000D1F7C80FD91FEA1FFB1FEE0CFF1C001FD7
:10CB7000111FEE0CFF1C001F111F2F5F3F4F4F4F67
:10CB80005F4FC217D307E407F50758F6215030402E
:10CB900040405040615067FFCFCF5695479537953D
:10CBA0002795CA01B901DF91CF911F910F91FF9095
:10CBB000EF900895002422273327442751E0BB2714
:10CBC000EE27FF27A0E1660F771F881F991F001C23
:10CBD000221F331F441F660F771F881F991F001CD9
:10CBE000221F331F441F2AF4050E2B1F3E1F4F1F09
:10CBF00004C0051A2B0B3E0B4F0B550FBB1FEE1F2E
:10CC0000587F556047FD5250AA95E9F6E695B795CD
:10CC10005795E695B7955795852F9B2F0895222711
:10CC2000332741E0552768E0880F991F221F331FE3
:10CC3000880F991F221F331F1AF4240F351F02C0BB
:10CC4000241B350B440F551F487F456037FD42506C
:10CC50006A9551F75695479556954795842F0895AF
:10CC6000AA2797FF04C0809590958A1F9A1F77FF87
:10CC700004C0609570956A1F7A1F669F9001779F28
:10CC8000A001679F300D411D5A1F300D411D5A1FD5
:10CC9000889FF001999F2E0F3F1F401D511D899FB6
:10CCA000300D411D5A1F300D411D5A1FCA01B901D7
:10CCB000112480CFFC014150504030F00190061605
:10CCC000D1F73197CF0108958827992708955058B3
:10CCD000192EA6D001D08CC0BA176207730784073B
:10CCE0009507B1F188F40EF410940B2EBA2FA02DF5
:10CCF000062E622F202D072E732F302D082E842F05
:10CD0000402D092E952F502DFF275523B9F0591B83
:10CD100049F0573E98F0469537952795A795F040EE
:10CD20005395C9F776F0BA0F621F731F841F30F452
:10CD3000879577956795B795F040939517FA0F2EDD
:10CD40000895BF1BBB27BA0B620B730B840BF6CF86
:10CD5000DEF692C097FB70D09F3738F0FEE9F91BE2
:10CD6000982F872F762F6B2F05C083C096958795B8
:10CD700077956795F150D0F73EF490958095709532
:10CD800061957F4F8F4F9F4F0895E89403C097FBA5
:10CD90000EF4F3DFB62F672F782F892F9EE900243A
:10CDA00027C00ED05EF004C00BD026F001C008D022
:10CDB00019F020F48FEF089580E0089581E0089540
:10CDC00097FB092E052600F868942DD0E89407FCFF
:10CDD00007C0621773078407950721F008F40094D1
:10CDE0000794989408959A95BB0F661F771F881F24
:10CDF00011249923A1F08823B2F79F3F59F0BB0F6C
:10CE000048F421F4002011F460FF04C06F5F7F4FED
:10CE10008F4F9F4F881F9795879597F9089529C041
:10CE2000052E092607FA440F551F5F3F79F0AA2700
:10CE3000A51708F051E04795880F991F9F3F31F0E3
:10CE4000BB27B91708F091E0879508959F919F91AE
:10CE5000112414C097FB880F991F9F3F31F0BB2707
:10CE6000B91708F091E0879508959F919F9111243B
:10CE700005C0662777278827992708959FEF80ECBC
:10CE80000895629FD001739FF001829FE00DF11D14
:10CE9000649FE00DF11D929FF00D839FF00D749F34
:10CEA000F00D659FF00D9927729FB00DE11DF91FE0
:10CEB000639FB00DE11DF91FBD01CF01112408953D
:10CEC000991B79E004C0991F961708F0961B881FDC
:10CED0007A95C9F780950895AA1BBB1B51E107C03D
:10CEE000AA1FBB1FA617B70710F0A61BB70B881FFA
:10CEF000991F5A95A9F780959095BC01CD01089589
:10CF000097FB092E07260AD077FD04D0E5DF06D06F
:10CF100000201AF4709561957F4F0895F6F790956B
:10CF200081959F4F0895A1E21A2EAA1BBB1BFD01FC
:10CF30000DC0AA1FBB1FEE1FFF1FA217B307E407F8
:10CF4000F50720F0A21BB30BE40BF50B661F771F50
:10CF5000881F991F1A9469F7609570958095909530
:10CF60009B01AC01BD01CF01089597FB092E052659
:10CF70000ED057FD04D0D7DF0AD0001C38F45095EE
:10CF80004095309521953F4F4F4F5F4F0895F6F7ED
:10CF900090958095709561957F4F8F4F9F4F089525
:10CFA000F999FECFB2BDA1BDF89A119600B40895CB
:10CFB000F7DF01921A94E1F70895F999FECFB2BD17
:10CFC000A1BD00BC11960FB6F894FA9AF99A0FBE5B
:0CCFD00008950190F2DF1A94E1F7089533
:10CFDC005E010A0151756164726F0000416E676CED
:10CFEC00654E69636B20202020202020416E676CE9
:10CFFC0065526F6C6C202020202020204163634EF2
:10D00C0069636B2020202020202020204163635264
:10D01C006F6C6C2020202020202020204779726FFC
:10D02C0047696572202020202020202048696768ED
:10D03C00742056616C756520202020204163635A52
:10D04C002020202020202020202020204761732019
:10D05C00202020202020202020202020436F6D70B5
:10D06C006173732056616C7565202020566F6C744B
:10D07C00616765202020202020202020456D7066CF
:10D08C00616E672020202020202020204779726F9D
:10D09C00204B6F6D70617373202020204D6F746F67
:10D0AC00722046726F6E7420202020204D6F746F9A
:10D0BC007220526561722020202020204D6F746FE9
:10D0CC0072204C6566742020202020204D6F746FD8
:10D0DC007220526967687420202020202020202094
:10D0EC002020202020202020202020202020202034
:10D0FC002020202020202020202020205661726912
:10D10C006F4D657465722020202020204D4B334DCF
:10D11C0061672043616C537461746520536572764A
:10D12C006F2020202020202020202020486F6F7688
:10D13C006572676173202020202020202020202071
:10D14C0020202020202020202020202020202020D3
:10D15C0020202020202020202020202020202020C3
:10D16C0020202020202020202020202020202020B3
:10D17C0020202020202020202020202020202020A3
:10D18C002020202020202020202020202020202093
:10D19C002020202020202020202020204932432D18
:10D1AC004572726F72202020202020202020202009
:10D1BC002020202020202020202020204750535F9A
:10D1CC004E69636B20202020202020204750535F85
:10D1DC00526F6C6C2020202020202020C80001647D
:10D1EC00FF01FFFF01FC01FC0101737373FF0300DE
:10D1FC007D0000C409C40964000E48616C6C6F208A
:10D20C0057656C7400000000000000000000000076
:10D21C000000000000000000000000000000000002
:10D22C0000000000000000000000000000000000F2
:10D23C0000000000000000000000000000000000E2
:10D24C0000000000000000000000010203040506BD
:10D25C000708090A01040B050000ECFF6440415A61
:10D26C004664640A02969696960840403A10FB3043
:10D27C00380190D0030090D00300F4016400537087
:10D28C006F727400004E6F726D616C0000426567C6
:10D29C00696E6E657200007800FF03640A0B0D0B5B
:0CD2AC000C0E0F0101017F7F7F7F7F7F50
:00000001FF
